:1000000000800010F500000000000000D1DF0000BB
:1000100055DF00008DDF0000A9DF000000000000B8
:1000200000000000000000000000000000000000D0
:100030000000000000000000C9CD010061E10000E7
:10004000E5CD010001CE01001DCE010039CE010039
:1000500055CE010071CE01008DCE0100A9CE010068
:10006000C5CE0100E1CE0100FDCE010019CF010097
:1000700035CF010051CF01006DCF010089CF0100C4
:10008000A5CF0100C1CF0100DDCF0100F9CF0100F4
:1000900015D0010031D001004DD0010069D0010020
:1000A00085D00100A1D00100BDD00100D9D0010050
:1000B000F5D0010011D101002DD1010049D101007D
:1000C00065D1010040F62013C1F200031A780AB985
:1000D00001221A70704700BF40F61C10C1F20000E8
:1000E00008B503682BB140F20003C0F2000303B16E
:1000F000984708BD684620F007018D4681B583B05A
:1001000000AF2EF0EDFD43F20042C0F2050240F2D6
:100110000003C1F200039A421DD043F20043C0F233
:1001200005033B6040F20003C1F200037B600BE07B
:100130003B681A687B681A607B6803F104037B6084
:100140003B6803F104033B607A6840F61C13C1F27C
:1001500000039A42ECD34DF2E002C0F2040240F2F6
:100160000003C1F200039A421DD04DF2E003C0F239
:1001700004033B6040F20003C1F200037B600BE02C
:100180003B681A687B681A607B6803F104037B6034
:100190003B6803F104033B607A6840F20003C1F25C
:1001A00000039A42ECD340F62013C1F200037B60B7
:1001B00007E07B684FF000021A607B6803F10403DC
:1001C0007B607A6841F24C43C1F200039A42F0D35B
:1001D0003AF05AFB0FF068FBFEE700BF80B487B02F
:1001E00000AFF860B9607A60FB687B61BB683B6117
:1001F0000BE03B691A787B691A707B6903F1010394
:100200007B613B6903F101033B617B68002B0CBF01
:1002100000230123DBB27A6802F1FF327A60002BFF
:10022000E7D107F11C07BD4680BC704780B487B09A
:1002300000AFF860B9607A60FB687B6107E0BB687B
:10024000DAB27B691A707B6903F101037B617B6819
:10025000002B0CBF00230123DBB27A6802F1FF32CE
:100260007A60002BEBD107F11C07BD4680BC7047BC
:1002700080B489B000AFF860B9607A60FB68FB6158
:10028000BB68BB614FF000037B6100BF7B68002B44
:100290000CBF00230123DBB27A6802F1FF327A60DF
:1002A000002B16D0FB691B781A46BB691B78D31A42
:1002B0007B617B69002B14BF00230123DBB2FA6949
:1002C00002F10102FA61BA6902F10102BA61002B7E
:1002D000DCD17B69184607F12407BD4680BC704716
:1002E00080B483B000AF7860396003E07B6803F1CD
:1002F00001037B607B681B78002B05D07B681B7833
:100300001A463B689A42F1D17B681B78184607F180
:100310000C07BD4680BC704780B584B000AF7860E4
:1003200039607B68DB6AFB60FA683B689A4255D0AB
:100330007B681B79002B39D07B685A787B6803F186
:10034000300310461946FA684FF0010315F01EFEFF
:100350000346002B02D04FF0010341E07B684FF0D1
:1003600000021A717B681A6A7B68DB69D218FB6825
:100370009A421BD97B68DB78FB7214E07B68DB69EF
:10038000FA68D318FB607B685A787B6803F1300306
:1003900010461946FA684FF0010315F0F7FDFB7A95
:1003A00003F1FF33FB72FB7A012BE7D83B68002B8C
:1003B00014D07B685A787B6803F1300310461946E5
:1003C0003A684FF0010315F0CBFD0346002B02D035
:1003D0004FF0010304E07B683A68DA624FF00003F3
:1003E000184607F11007BD4680BD00BF80B584B038
:1003F00000AF786078684FF00001FFF78DFF03468B
:10040000FB73FB7B002B40F0D2807B681B78032BB7
:1004100040F0BE807B685B79002B00F0B9807B6880
:100420004FF00002DA627B6803F1300318464FF0A8
:1004300000014FF40072FFF7F9FE7B6803F50A73C1
:1004400003F106034FF055021A707B6803F50A7337
:1004500003F107034FF0AA021A707B684FF05202B3
:1004600083F830207B6803F131034FF052021A7099
:100470007B6803F132034FF061021A707B6803F16D
:1004800033034FF041021A707B6803F505734FF098
:1004900072021A707B6803F5047303F105034FF0D1
:1004A00072021A707B6803F5047303F106034FF0C0
:1004B00041021A707B6803F5047303F107034FF0E0
:1004C00061021A707B6803F506737A681269D2B20A
:1004D0001A707B6803F5067303F101037A681269E9
:1004E00092B24FEA122292B2D2B21A707B6803F52E
:1004F000067303F102037A6812694FEA1242D2B21C
:100500001A707B6803F5067303F103037A681269B6
:100510004FEA1262D2B21A707B6803F507737A68E9
:10052000D268D2B21A707B6803F5067303F1050333
:100530007A68D26892B24FEA122292B2D2B21A709C
:100540007B6803F5067303F106037A68D2684FEA05
:100550001242D2B21A707B6803F5067303F10703E7
:100560007A68D2684FEA1262D2B21A707B68597800
:100570007B6803F130027B685B69084611461A46C6
:100580004FF0010315F002FD7B684FF000025A7135
:100590007B685B7818464FF000014FF0000215F0C1
:1005A000C9FC0346002B02D04FF00103FB73FB7B19
:1005B000184607F11007BD4680BD00BF80B483B068
:1005C00000AF786039603B68A3F102033B607B6851
:1005D0009B69A3F102023B689A4202D84FF00003E4
:1005E00007E07B689B783A6802FB03F27B689B6AB2
:1005F000D318184607F10C07BD4680BC704700BFF2
:1006000080B586B000AF786039603B68012B04D9B3
:100610007B689A693B689A4202D84FF00103BCE0BC
:100620007B681B78022B54D0032B79D0012B40F030
:10063000B2803B687B617B694FEA53037A69D318C8
:100640007B617B681A6A7B694FEA5323D318786809
:100650001946FFF761FE0346002B40F095807B6949
:100660004FEAC3534FEAD3537A68D31893F8303024
:100670003B617B6903F101037B617B681A6A7B69DB
:100680004FEA5323D31878681946FFF745FE03460F
:10069000002B7BD17B694FEAC3534FEAD3537A686F
:1006A000D31893F830304FEA03233A6942EA030340
:1006B0003B613B6803F00103DBB2002B03D03B69D5
:1006C0004FEA131304E03B694FEA03534FEA135315
:1006D00063E07B681A6A3B684FEA1323D318786893
:1006E0001946FFF719FE0346002B51D17B6803F131
:1006F00030023B684FEA43034FEAC3534FEAD353F8
:10070000D318FB60FB6803F101031B784FEA032356
:100710009AB2FB681B7842EA03039BB29BB23CE0AF
:100720007B681A6A3B684FEAD313D3187868194676
:10073000FFF7F2FD0346002B2CD17B6803F130025A
:100740003B684FEA83034FEAC3534FEAD353D318AE
:10075000FB60FB6803F103031B784FEA0362FB684D
:1007600003F102031B784FEA03431A43FB6803F1CA
:1007700001031B784FEA03231A43FB681B7842EA04
:10078000030323F0704308E000BF04E000BF02E071
:1007900000BF00E000BF4FF0FF33184607F1180715
:1007A000BD4680BD80B588B000AFF860B9607A60A2
:1007B000BB68012B04D9FB689A69BB689A4203D8CD
:1007C0004FF00203FB7718E1FB681B78022B00F067
:1007D0008380032B00F0AA80012B40F0FF80BB68D0
:1007E000BB61BB694FEA5303BA69D318BB61FB68AD
:1007F0001A6ABB694FEA5323D318F8681946FFF702
:100800008BFD0346FB77FB7F002B40F0EB80FB6802
:1008100003F13002BB694FEAC3534FEAD353D318F5
:100820007B61BB6803F00103DBB2002B0FD07B6957
:100830001B78DBB203F00F03DAB27B68DBB24FEA5E
:100840000313DBB242EA0303DBB2DBB201E07B68F5
:10085000DBB27A691370BB6903F10103BB61FB680A
:100860004FF001021A71FB681A6ABB694FEA532301
:10087000D318F8681946FFF74FFD0346FB77FB7F57
:10088000002B40F0B180FB6803F13002BB694FEAF6
:10089000C3534FEAD353D3187B61BB6803F0010302
:1008A000DBB2002B04D07B684FEA1313DBB210E0FD
:1008B0007B691B78DBB223F00F03DAB27B684FEA67
:1008C0001323DBB203F00F03DBB242EA0303DBB214
:1008D000DBB27A6913708CE0FB681A6ABB684FEA76
:1008E0001323D318F8681946FFF716FD0346FB7764
:1008F000FB7F002B7AD1FB6803F13002BB684FEA23
:1009000043034FEAC3534FEAD353D3187B617B6849
:10091000DAB27B691A707B6903F101037A6892B2DB
:100920004FEA122292B2D2B21A7062E0FB681A6ADF
:10093000BB684FEAD313D318F8681946FFF7ECFCED
:100940000346FB77FB7F002B52D1FB6803F130029B
:10095000BB684FEA83034FEAC3534FEAD353D3181C
:100960007B617B6903F103031B784FEA03627B69B8
:1009700003F102031B784FEA03431A437B6903F137
:1009800001031B784FEA03231A437B691B7842EA71
:10099000030303F070437A6842EA03037B607B68D9
:1009A000DAB27B691A707B6903F101037A6892B24B
:1009B0004FEA122292B2D2B21A707B6903F102039B
:1009C0007A684FEA1242D2B21A707B6903F10303CC
:1009D0007A684FEA1262D2B21A700AE04FF002034C
:1009E000FB7706E000BF04E000BF02E000BF00E0CC
:1009F00000BFFB684FF001021A71FB7F184607F138
:100A00002007BD4680BD00BF80B584B000AF7860D0
:100A100039603B68012B04D97B689A693B689A422C
:100A200003D84FF00203FB733FE04FF00003FB736A
:100A300032E078683968FFF7E3FDB860BB68002BE7
:100A400030D0BB68012B03D14FF00203FB732CE0C5
:100A5000BB68B3F1FF3F03D14FF00103FB7324E008
:100A6000786839684FF00002FFF79CFE0346FB737D
:100A7000FB7B002B18D17B681B69B3F1FF3F09D0CA
:100A80007B681B6903F101027B681A617B684FF088
:100A900001025A71BB683B607B689A693B689A4265
:100AA000C7D802E000BF00E000BFFB7B184607F19B
:100AB0001007BD4680BD00BF80B586B000AF78602E
:100AC00039603B68002B0ED17B68DB683B613B697A
:100AD000002B04D07B689A693B699A4217D84FF083
:100AE00001033B6113E078683968FFF789FDB8605E
:100AF000BB68012B02D84FF001036DE07B689A6957
:100B0000BB689A4201D9BB6866E03B683B613B69C0
:100B10007B6100E000BF7B6903F101037B617B68BF
:100B20009A697B699A4209D84FF002037B617A691E
:100B30003B699A4202D94FF000034DE07868796929
:100B4000FFF75EFDB860BB68002B0BD17868796950
:100B50006FF07042FFF726FE0346FB73FB7B002B12
:100B600010D019E0BB68B3F1FF3F02D0BB68012B86
:100B700001D1BB6830E07A693B699A42CAD14FF033
:100B8000000329E03B68002B06D0786839687A6951
:100B9000FFF708FE0346FB73FB7B002B12D17B683B
:100BA0007A69DA607B681B69B3F1FF3F13D07B6819
:100BB0001B6903F1FF327B681A617B684FF0010209
:100BC0005A7108E0FB7B012B02D14FF0FF3301E0AB
:100BD0004FF001037B617B69184607F11807BD469A
:100BE00080BD00BF80B584B000AF78600B467B80CD
:100BF0007B687A88DA807B689B68FB60FB68012BE6
:100C000005D07B681B689A69FB689A4202D84FF04E
:100C100002036DE0FB68002B08D17B681B681B7822
:100C2000032B03D17B681B685B6AFB60FB68002BAE
:100C300016D17B68FA68DA607B681B681B897A8842
:100C40009A4202D34FF0020352E07B681B685A6A53
:100C50007B884FEA13139BB2D2187B681A6139E084
:100C60007B681B689B784FEA03137B811DE07B68E0
:100C70001B681846F968FFF7C3FCF860FB68B3F11E
:100C8000FF3F02D14FF0010332E0FB68012B05D991
:100C90007B681B689A69FB689A4202D84FF002038E
:100CA00026E07A887B89D31A7B807A887B899A426E
:100CB000DDD27B68FA68DA607B681B681846F968E1
:100CC000FFF77CFC02467B884FEA13139BB2D218D5
:100CD0007B681A617B681B6803F130027B8803F034
:100CE0000F034FEA4313D2187B685A614FF0000399
:100CF000184607F11007BD4680BD00BF90B585B00E
:100D000000AF786039607B68DB8803F101033B81C9
:100D10003B89002B03D07B681B69002B02D14FF06D
:100D20000403D4E03B8903F00F039BB2002B40F097
:100D3000BD807B681B6903F101027B681A617B68D7
:100D4000DB68002B09D17B681B681B893A899A42B2
:100D5000C0F0AC804FF00403B9E03B894FEA1313B5
:100D60009BB21A467B681B689B7803F1FF3302EA4B
:100D70000303002B40F09A807B681A687B68DB686D
:100D800010461946FFF73CFCF860FB68012B02D8BF
:100D90004FF002039BE0FB68B3F1FF3F02D14FF03D
:100DA000010394E07B681B689A69FB689A4271D8DA
:100DB0003B68002B02D14FF0040388E07B681A687F
:100DC0007B68DB6810461946FFF776FEF860FB6823
:100DD000002B02D14FF0070379E0FB68012B02D111
:100DE0004FF0020373E0FB68B3F1FF3F02D14FF015
:100DF00001036CE07B681B6818464FF00001FFF7A9
:100E00008BFA0346002B02D04FF001035FE07B68B2
:100E10001B6803F1300318464FF000014FF40072D5
:100E2000FFF704FA7B681C687B681B681846F96842
:100E3000FFF7C4FB0346E3624FF00003FB721BE0C5
:100E40007B681B684FF001021A717B681B681846AB
:100E50004FF00001FFF760FA0346002B02D04FF07D
:100E6000010334E07B681B68DA6A02F10102DA628E
:100E7000FB7A03F10103FB727B681B689B78FA7AAB
:100E80009A42DDD37B681B687A681268D16AFA7A65
:100E90008A1ADA627B68FA68DA607B681B6818462F
:100EA000F968FFF78BFB02467B681A617B683A8919
:100EB000DA807B681B6803F130023B8903F00F0383
:100EC0004FEA4313D2187B685A614FF0000318466B
:100ED00007F11407BD4690BD80B485B000AF7860BF
:100EE00039603B6803F11B031B784FEA03239AB276
:100EF0003B6803F11A031B7842EA03039BB29BB2DF
:100F0000FB607B681B78032B14D13B6803F115034E
:100F10001B784FEA03239AB23B6803F114031B7852
:100F200042EA03039BB29BB24FEA0343FA6842EAE8
:100F30000303FB60FB68184607F11407BD4680BC3D
:100F4000704700BF80B483B000AF786039607B68C1
:100F500003F11A033A68D2B21A707B6803F11B03DB
:100F60003A6892B24FEA122292B2D2B21A707B68F9
:100F700003F114033A684FEA1242D2B21A707B6846
:100F800003F115033A684FEA124292B24FEA122275
:100F900092B2D2B21A7007F10C07BD4680BC7047FE
:100FA00080B586B000AF786039603B681B7823F06D
:100FB000400303F1FF3213464FEA43039B184FEA05
:100FC00083039B187B614FF000033B614FF00103EB
:100FD000FB8148F65023C0F204033A699B181B7842
:100FE00003F101033A68D3181B784FEA03239AB23E
:100FF00048F65023C0F2040339695B181B7839683E
:10100000CB181B7842EA03039BB2BB81FB89002B00
:101010001CD0BB89184602F005FD0346FB817B69A5
:10102000FE2B10D87B694FEA43037A68D3181B88DC
:101030007A6902F101027A61184602F0F3FC034674
:10104000FA899A420AD04FF0000324E0BA894FF699
:10105000FF739A4202D04FF000031CE03B6903F19A
:1010600001033B613B690C2BB3D93B681B7803F050
:101070004003002B0DD0FB89002B0AD07B694FEA7F
:1010800043037A68D3181B88002B02D04FF000036B
:1010900001E04FF00103184607F11807BD4680BD77
:1010A00080B487B000AF786039603B681B7803F08C
:1010B0003F0303F1FF3213464FEA43039B184FEA05
:1010C00083039B187B614FF000033B614FF00103EA
:1010D000FB8148F65023C0F204033A699B181B7841
:1010E00003F101033A68D3181B784FEA03239AB23D
:1010F00048F65023C0F2040339695B181B7839683D
:10110000CB181B7842EA03039BB2BB81FB89002BFF
:1011100013D07B69FE2B02D94FF0000332E07B69CC
:101120004FEA43037A68D318BA89FA81FA891A8098
:101130007B6903F101037B6107E0BA894FF6FF7316
:101140009A4202D04FF000031CE03B6903F1010317
:101150003B613B690C2BBCD93B681B7803F0400317
:10116000002B0DD07B69FE2B02D94FF0000309E064
:101170007B694FEA43037A68D3184FF000021A8064
:101180004FF00103184607F11C07BD4680BC7047AD
:1011900080B489B000AFF860B960FA71BB71BB6808
:1011A00003F10D03BA791A70BB6803F10B034FF01A
:1011B0000F021A70BB6803F10C034FF000021A70A3
:1011C000BB6803F11A034FF000021A70BB6803F109
:1011D0001B034FF000021A70FB7903F1FF32134634
:1011E0004FEA43039B184FEA83039B18FB614FF0C0
:1011F0000003FB824FF00003BB61FA8A4FF6FF73D6
:101200009A420AD0FB694FEA4303FA68D3181B8855
:10121000FB82FB6903F10103FB6148F65023C0F236
:101220000403BA699B181B78BA68D318FA8AD2B239
:101230001A7048F65023C0F20403BA699B181B7851
:1012400003F10103BA68D318FA8A4FEA122292B264
:10125000D2B21A70FB8A002B02D14FF6FF73FB82C9
:10126000BB6903F10103BB61BB690C2BC5D9FA8AC9
:101270004FF6FF739A4207D0FB694FEA4303FA68BF
:10128000D3181B88002B03D1FB7943F04003FB717B
:10129000BB68FA791A7007F12407BD4680BC704715
:1012A00080B58AB000AFF860B9607A607B80F8687A
:1012B000B9684FF00B02FEF791FF7B88052B14D91C
:1012C0007B884FEAC3329BB24FEA530342EA0303DF
:1012D0009AB27B681B88D3187B807B6803F102037A
:1012E0007B607B681B88002BEAD14FF007033B62D1
:1012F0007B88DBB203F00F03DBB203F1300387F826
:10130000273097F82730392B05D997F8273003F184
:10131000070387F8273007F114023B6AD31897F8C0
:1013200027201A703B6A03F1FF333B627B884FEA48
:1013300013137B807B88002BDAD107F114023B6A00
:10134000D3184FF07E021A704FF00003FB6103E0E8
:10135000FB6903F10103FB61FA693B6A9A4205D21A
:10136000FA68FB69D3181B78202BF1D1FA68FB6966
:10137000D2183B6A072B09D807F114013B6ACB1836
:101380001B78396A01F10101396201E04FF0200355
:101390001370FB6903F10103FB61FB69072BE5D9BE
:1013A00007F12807BD4680BD80B485B000AF7860E6
:1013B0004FF00003FB734FF00B03BB60FB7B4FEA66
:1013C000C312DBB24FEA530342EA0303DAB27B688B
:1013D0001B78D318FB737B6803F101037B60BB6848
:1013E00003F1FF33BB60BB68002BE7D1FB7B1846E2
:1013F00007F11407BD4680BC704700BF80B586B0BA
:1014000000AF786078684FF00001FFF7EBFB034610
:10141000FB75FB7D002B01D0FB7DA4E04FF0FF03AB
:101420003B753B7D7B757B681A687B681B69104642
:101430001946FEF771FF0346FB75FB7D002B40F05C
:101440008C807B685B693B613B691B78BB75BB7DAE
:10145000002B03D14FF00403FB7583E03B6903F1DC
:101460000B031B7803F03F03FB73BB7DE52B07D019
:10147000FB7B03F00803002B06D0FB7B0F2B03D074
:101480004FF0FF037B755CE0FB7B0F2B34D17B6857
:10149000DB69002B55D0BB7D03F04003002B0ED041
:1014A0003B6903F10D031B783B75BB7D23F04003C3
:1014B000BB75BB7D7B757B68DA887B681A84BA7DD7
:1014C0007B7D9A4214D13B6903F10D031B783A7D71
:1014D0009A420DD17B68DB6918463969FFF760FDD8
:1014E0000346002B04D07B7D03F1FF33DBB201E028
:1014F0004FF0FF037B7524E07B7D002B06D138691C
:10150000FFF752FF03463A7D9A4228D04FF0FF037F
:101510007B757B684FF6FF721A847B689B6903F1C9
:101520000B031B7803F00103002B0AD17B689B6936
:10153000386919464FF00B02FEF79AFE0346002B5E
:101540000FD078684FF00001FFF7D8FB0346FB751A
:10155000FB7D002B3FF467AF04E000BF02E000BF5B
:1015600000E000BFFB7D184607F11807BD4680BDAF
:1015700080B586B000AF78604FF0FF037B754FF009
:10158000FF033B754FF00403FB757FE07B681A682F
:101590007B681B6910461946FEF7BEFE0346FB75C5
:1015A000FB7D002B78D17B685B693B613B691B78D5
:1015B000BB75BB7D002B03D14FF00403FB7570E0BE
:1015C0003B6903F10B031B7803F03F03FB73BB7D07
:1015D000E52B0AD0BB7D2E2B07D0FB7B03F0080345
:1015E000002B06D0FB7B0F2B03D04FF0FF037B7546
:1015F00042E0FB7B0F2B30D1BB7D03F04003002B7F
:101600000ED03B6903F10D031B783B75BB7D23F0C6
:101610004003BB75BB7D7B757B68DA887B681A8469
:10162000BA7D7B7D9A4214D13B6903F10D031B788F
:101630003A7D9A420DD17B68DB6918463969FFF71C
:101640002FFD0346002B04D07B7D03F1FF33DBB27B
:1016500001E04FF0FF037B750EE07B7D002B06D190
:101660003869FFF7A1FE03463A7D9A4216D07B689F
:101670004FF6FF721A8414E078684FF00001FFF70C
:101680003DFB0346FB75FB7D002B09D17B681B6985
:10169000002B7FF47BAF04E000BF02E000BF00E05E
:1016A00000BFFB7D002B03D07B684FF000021A6166
:1016B000FB7D184607F11807BD4680BD80B58CB08C
:1016C00000AF78607B689B697B627B68DB693B620B
:1016D00007F10C031846796A4FF00C02FEF77EFD05
:1016E000FB7D03F00103DBB2002B3DD07B6A03F1ED
:1016F0000B034FF000021A707B684FF00002DA61B2
:101700004FF00103BB8515E007F10C02BB8D786A31
:1017100011463A6AFFF7C4FD7868FFF76FFE03468B
:1017200087F82F3097F82F30002B07D1BB8D03F1AE
:101730000103BB85BB8D632BE6D900E000BFBB8DE9
:10174000642B02D14FF007030BE197F82F30042BE5
:1017500002D097F82F3004E17B6A03F10B03FA7D86
:101760001A707B683A6ADA61FB7D03F00203002B92
:101770001FD04FF000037B8503E07B8D03F1010355
:101780007B857B8D4FEA43033A6AD3181B88002B75
:10179000F3D17B8D03F119024EF64F43C4F6C463B7
:1017A00083FB02134FEAA3014FEAE273CB1A7B8556
:1017B00002E04FF001037B8578684FF00001FFF7EE
:1017C00011FA034687F82F3097F82F30002B02D0FC
:1017D00097F82F30C5E04FF000033B853B8DBB856C
:1017E0007B681A687B681B6910461946FEF794FDF2
:1017F000034687F82F3097F82F30002B28D17B68CD
:101800005B691B78FB77FB7FE52B02D0FB7F002B0E
:101810000ED1BB8D002B02D17B68DB883B85BB8D55
:1018200003F10103BB85BA8D7B8D9A4203D110E091
:101830004FF00003BB8578684FF00101FFF75EFAB7
:10184000034687F82F3097F82F30002BC8D000E0E0
:1018500000BF97F82F30002B4BD17B8D012B48D93F
:101860003B8D78681946FFF7BDF9034687F82F309E
:1018700097F82F30002B3CD17B689B691846FFF707
:1018800093FD0346BB777B8D03F1FF337B857B683C
:101890001A687B681B6910461946FEF73DFD034632
:1018A00087F82F3097F82F30002B21D17B68D8692B
:1018B0007B6859697B8DDAB2BB7FFFF769FC7B6877
:1018C0001B684FF001021A7178684FF00001FFF7B2
:1018D00015FA034687F82F3097F82F30002B08D1E0
:1018E0007B8D03F1FF337B857B8D002BCFD100E017
:1018F00000BF97F82F30002B31D17B681A687B68C6
:101900001B6910461946FEF707FD034687F82F307E
:1019100097F82F30002B22D17B685B69BB61B869D7
:101920004FF000014FF02002FEF780FC7B689B69BE
:10193000B86919464FF00B02FEF750FCBB6903F182
:101940000C037A68926902F10B02127802F0180215
:10195000D2B21A707B681B684FF001021A7197F8B7
:101960002F30184607F13007BD4680BD80B584B0E2
:1019700000AF78607B68DB88BB817B681A8C4FF690
:10198000FF739A4202D07B681B8C00E0BB897868A9
:101990001946FFF727F90346FB73FB7B002B2FD17A
:1019A0007B681A687B681B6910461946FEF7B4FC11
:1019B0000346FB73FB7B002B19D17B685B694FF0FF
:1019C000E5021A707B681B684FF001021A717B6890
:1019D000DB88BA899A420CD978684FF00001FFF78A
:1019E0008DF90346FB73FB7B002BD9D002E000BFCF
:1019F00000E000BFFB7B042B02D14FF00203FB731E
:101A0000FB7B184607F11007BD4680BD80B58AB044
:101A100000AF786039603B681B683B6103E03B695D
:101A200003F101033B613B691B782F2BF7D03B6926
:101A30001B785C2BF3D07B68DB69FB604FF0000305
:101A40007B617B69BB613A69BB69D3181B78BB8436
:101A5000BB6903F10103BB61BB8C1F2B3AD9BB8C63
:101A60002F2B37D0BB8C5C2B34D07B69FE2B02D95B
:101A70004FF00603A7E1BB8C03F0FF03BB84BB8CD4
:101A800018464FF0010101F087FF0346BB84BB8C71
:101A9000002B02D14FF0060395E1BB8C7F2B0DD8B4
:101AA000BB8C48F66020C0F204001946FEF718FC13
:101AB0000346002B02D04FF0060384E17B694FEA16
:101AC0004303FA68D318BA8C1A807B6903F10103C7
:101AD0007B61B8E73A69BB69D2183B681A60BB8C76
:101AE0001F2B02D84FF0040301E04FF0000387F8EA
:101AF000263012E07B6903F1FF334FEA4303FA68B3
:101B0000D3181B88BB84BB8C202B02D0BB8C2E2B04
:101B100007D17B6903F1FF337B617B69002BE9D13E
:101B200000E000BF7B69002B02D14FF006034AE1C1
:101B30007B694FEA4303FA68D3184FF000021A801A
:101B40007B689B6918464FF020014FF00B02FEF7AF
:101B50006DFB4FF00003BB6103E0BB6903F10103C0
:101B6000BB61BB694FEA4303FA68D3181B88202B7B
:101B7000F3D0BB694FEA4303FA68D3181B882E2BB6
:101B8000EBD0BB69002B0AD097F8263043F0030353
:101B900087F8263003E07B6903F1FF337B617B69C3
:101BA000002B09D07B6903F1FF334FEA4303FA6846
:101BB000D3181B882E2BEED14FF000033B624FF061
:101BC000000387F827304FF00803FB61BB694FEA39
:101BD0004303FA68D3181B88BB84BB6903F1010374
:101BE000BB61BB8C002B00F09F80BB8C202B06D0F0
:101BF000BB8C2E2B0AD1BA697B699A4206D097F822
:101C0000263043F0030387F826308CE03A6AFB69FC
:101C10009A4203D2BA697B699A4226D1FB690B2B9F
:101C200006D197F8263043F0030387F826307EE08C
:101C3000BA697B699A4205D097F8263043F00303CE
:101C400087F82630BA697B699A426FD87B69BB6195
:101C50004FF008033B624FF00B03FB6197F827300E
:101C60004FEA830387F827305DE0BB8C7F2B19D9BF
:101C7000BB8C18464FF0000101F08EFE0346BB847A
:101C8000BB8C002B08D0BB8CA3F1800248F67423D8
:101C9000C0F204039B5CBB8497F8263043F0020338
:101CA00087F82630BB8C002B0AD0BB8C48F66C2002
:101CB000C0F204001946FEF713FB0346002B09D0BF
:101CC0004FF05F03BB8497F8263043F0030387F897
:101CD00026301CE0BB8C402B09D9BB8C5A2B06D874
:101CE00097F8273043F0020387F827300FE0BB8CCA
:101CF000602B0CD9BB8C7A2B09D897F8273043F08E
:101D0000010387F82730BB8CA3F12003BB847B68D9
:101D10009A693B6AD318BA8CD2B21A703B6A03F143
:101D200001033B6252E751E700BF00E000BF7B6860
:101D30009B691B78E52B04D17B689B694FF00502FA
:101D40001A70FB69082B05D197F827304FEA8303F7
:101D500087F8273097F8273003F00C030C2B05D0B9
:101D600097F8273003F00303032B05D197F82630AB
:101D700043F0020387F8263097F8263003F0020379
:101D8000002B17D197F8273003F00303012B05D15F
:101D900097F8263043F0100387F8263097F827305D
:101DA00003F00C03042B05D197F8263043F0080309
:101DB00087F826307B689B6903F10B0397F8262090
:101DC0001A704FF00003184607F12807BD4680BD82
:101DD00080B584B000AF786039603B681B782F2BEA
:101DE00003D03B681B785C2B03D13B6803F10103F4
:101DF0003B607B684FF000029A603B681B781F2BAA
:101E00000BD878684FF00001FEF7ECFE0346FB7339
:101E10007B684FF000025A6148E03B4678681946FB
:101E2000FFF7F4FD0346FB73FB7B002B37D178688B
:101E3000FFF7E4FA0346FB737B689B6903F10B032E
:101E40001B78BB73FB7B002B0BD0FB7B042B28D1B7
:101E5000BB7B03F00403002B25D14FF00503FB737C
:101E600024E0BB7B03F00403002B1ED17B685B697D
:101E7000BB60BB6803F10B031B7803F01003002B5E
:101E800003D14FF00503FB7310E07B681B68184615
:101E9000B968FFF721F802467B689A60BDE700BF8A
:101EA00004E000BF02E000BF00E000BFFB7B18467B
:101EB00007F11007BD4680BD80B582B000AF7860E5
:101EC00039607B685A787B6803F130031046194605
:101ED0003A684FF0010314F043F80346002B02D098
:101EE0004FF0030367E07B6803F50A7303F1070310
:101EF0001B784FEA03239AB27B6803F50A7303F158
:101F000006031B7842EA03039BB21AB24AF6552332
:101F1000CFF6FF739A4202D04FF002034BE07B688A
:101F200003F169031B784FEA03627B6803F16803DE
:101F30001B784FEA03431A437B6803F167031B785E
:101F40004FEA03231A437B6803F166031B7842EAD6
:101F5000030323F07F4244F24613C0F254039A4233
:101F600002D14FF0000326E07B6803F185031B7864
:101F70004FEA03627B6803F184031B784FEA034353
:101F80001A437B6803F183031B784FEA03231A4348
:101F90007B6803F182031B7842EA030323F07F424C
:101FA00044F24613C0F254039A4202D14FF00003A8
:101FB00001E04FF00103184607F10807BD4680BD58
:101FC00080B592B000AFF860B9601346FB71FB6852
:101FD0001B68FB62FB6A1B78A3F130033B643B6C1C
:101FE000092B0DD8FB6A03F101031B783A2B07D1AB
:101FF000FB6A03F10203FB62FB68FA6A1A6002E003
:102000004FF000033B64BB684FF000021A603B6C6A
:10201000022B02D94FF00B031CE340F62413C1F24C
:1020200000033A6C53F82230BB62BB6A002B02D12A
:102030004FF00C030EE3BB68BA6A1A60BB6A1B78E8
:10204000002B1CD0BB6A5B78184613F063FF034675
:1020500087F8273097F8273003F00103002B0ED1C3
:10206000FB79002B08D097F8273003F00403002BEE
:1020700002D04FF00A03EDE24FF00003EAE2BB6A40
:102080004FF000021A703B6CDAB2BB6A5A70BB6A3E
:102090005B78184613F02EFF034687F8273097F831
:1020A000273003F00103DBB2002B02D04FF0030313
:1020B000D0E2FB79002B08D097F8273003F0040317
:1020C000002B02D04FF00A03C4E24FF00003FB6381
:1020D000B86AF96BFFF7F0FE034687F8473097F8C8
:1020E0004730012B40D14FF0000387F8463097F876
:1020F0004630002B05D097F8463003F1FF3387F8C0
:102100004630BB6A03F1300297F846304FEA0313BA
:1021100003F5DF73D3183B623B6A03F104031B78BA
:10212000002B21D03B6A03F10B031B784FEA0362BB
:102130003B6A03F10A031B784FEA03431A433B6AE5
:1021400003F109031B784FEA03231A433B6A03F1A7
:1021500008031B7842EA0303FB63B86AF96BFFF7D5
:10216000ABFE034687F8473097F84730032B02D180
:102170004FF001036EE297F84730002B02D04FF08A
:102180000D0367E2BB6A03F13C031B784FEA0323AC
:102190009AB2BB6A03F13B031B7842EA03039BB28A
:1021A0001BB2B3F5007F02D04FF00D0352E2BB6AC1
:1021B00003F147031B784FEA03239AB2BB6A03F18A
:1021C00046031B7842EA03039BB29BB2BB63BB6B23
:1021D000002B1AD1BB6A03F157031B784FEA036245
:1021E000BB6A03F156031B784FEA03431A43BB6AE9
:1021F00003F155031B784FEA03231A43BB6A03F12B
:1022000054031B7842EA0303BB63BB6ABA6BDA610F
:10221000BB6A93F84030FB77BB6AFA7FDA70FB7FCA
:10222000012B05D0FB7F022B02D04FF00D0311E2F2
:10223000FA7FBB6B02FB03F3BB63BB6A93F83D30D1
:10224000FB77BB6AFA7F9A70FB7F002B07D0FA7F7F
:10225000FB7F03F1FF3302EA0303002B02D04FF0B0
:102260000D03F7E1BB6A03F142031B784FEA032336
:102270009AB2BB6A03F141031B7842EA03039BB2A3
:102280009AB2BB6A1A81BB6A1B8903F00F039BB227
:10229000002B02D04FF00D03DCE1BB6A03F14403D5
:1022A0001B784FEA03239AB2BB6A03F143031B78FE
:1022B00042EA03039BB29BB27B637B6B002B1AD178
:1022C000BB6A03F153031B784FEA0362BB6A03F155
:1022D00052031B784FEA03431A43BB6A03F15103CD
:1022E0001B784FEA03231A43BB6A03F150031B78A0
:1022F00042EA03037B63BB6A03F13F031B784FEAA7
:1023000003239AB2BB6A03F13E031B7842EA03033C
:102310009BB2BB83BB8B002B02D14FF00D0399E125
:10232000BA8BBB6BD218BB6A1B894FEA13139BB2E3
:10233000D318BB617A6BBB699A4202D24FF00D038E
:1023400088E17A6BBB69D21ABB6A9B78B2FBF3F364
:102350007B617B69002B02D14FF00D037AE14FF0D6
:10236000010387F847307A6940F6F5739A4203D93A
:102370004FF0020387F847307A694FF6F5739A42B7
:1023800003D94FF0030387F847307B6903F102025A
:10239000BB6A9A61FA6BBB69D218BB6A9A62BA8B44
:1023A000FB6BD218BB6A1A6297F84730032B27D110
:1023B000BB6A1B89002B02D04FF00D034AE1BB6AB8
:1023C00003F15F031B784FEA0362BB6A03F15E030C
:1023D0001B784FEA03431A43BB6A03F15D031B7882
:1023E0004FEA03231A43BB6A03F15C031B781A43C9
:1023F000BB6A5A62BB6A9B694FEA83033B6323E073
:10240000BB6A1B89002B02D14FF00D0322E1BB6A8E
:102410001A6ABB6BD218BB6A5A6297F84730022B14
:1024200004D1BB6A9B694FEA43030CE0BB6A9A691B
:1024300013464FEA43039B184FEA5302BB6A9B695A
:1024400003F00103D3183B63BB6ADA693B6B03F506
:10245000FE7303F103034FEA53239A4202D24FF073
:102460000D03F7E0BB6A4FF0FF321A61BB6A4FF011
:102470000002DA6097F84730032B40F0C980BB6A4E
:102480004FF000025A71BB6A03F161031B784FEAF7
:1024900003239AB2BB6A03F160031B7842EA030389
:1024A0009BB29BB21A46FB6BD218BB6A5A61BB6ADD
:1024B0005978BB6A03F13002BB6A5B690846114672
:1024C0001A464FF0010313F04BFD0346002B40F07A
:1024D0009F80BB6A03F50A7303F107031B784FEA79
:1024E00003239AB2BB6A03F50A7303F106031B7850
:1024F00042EA03039BB21AB24AF65523CFF6FF73A2
:102500009A4240F08580BB6A03F133031B784FEA9F
:102510000362BB6A03F132031B784FEA03431A4399
:10252000BB6A03F131031B784FEA03231A43BB6AEA
:1025300093F830301A4345F25223C4F261139A42A1
:1025400066D1BB6A03F5047303F107031B784FEAF6
:102550000362BB6A03F5047303F106031B784FEAB9
:1025600003431A43BB6A03F5047303F105031B78A5
:102570004FEA03231A43BB6A03F505731B781A431A
:1025800047F27223C6F241139A4241D1BB6A03F566
:10259000067303F107031B784FEA0362BB6A03F576
:1025A000067303F106031B784FEA03431A43BB6A21
:1025B00003F5067303F105031B784FEA03231A435F
:1025C000BB6A03F507731B781A43BB6ADA60BB6A00
:1025D00003F5067303F103031B784FEA0362BB6A3A
:1025E00003F5067303F102031B784FEA03431A4312
:1025F000BB6A03F5067303F101031B784FEA03235B
:102600001A43BB6A03F506731B781A43BB6A1A6147
:10261000BB6A97F847201A7040F63013C1F20003E6
:102620001B8803F101039AB240F63013C1F2000394
:102630001A8040F63013C1F200031A88BB6ADA80B0
:10264000BB6A4FF00002DA62BB6A4FF000021A71F7
:102650004FF00003184607F14807BD4680BD00BF94
:1026600080B584B000AF78607B68FB60FB681B6856
:10267000002B0BD0FB681B681B78002B06D0FB6877
:102680001B68DA88FB689B889A4202D04FF00903E6
:1026900010E0FB681B685B78184613F03BFC0346B0
:1026A00003F00103DBB2002B02D04FF0030301E083
:1026B0004FF00003184607F11007BD4680BD00BF6C
:1026C00080B485B000AF03463960FB71FB79022B03
:1026D00002D94FF00B031FE0FA7940F62413C1F240
:1026E000000353F82230FB60FB68002B03D0FB682B
:1026F0004FF000021A703B68002B03D03B684FF08C
:1027000000021A70FA7940F62413C1F20003396806
:1027100043F822104FF00003184607F11407BD4696
:1027200080BC704780B5ADF5147D00AF07F10C0398
:10273000186007F10803196007F1080303F1FF337C
:102740001A7007F10C031B68002B02D14FF009032C
:10275000D3E107F10C031B684FF000021A6007F188
:10276000080303F1FF3307F1080202F1FF32127888
:1027700002F01F021A7007F1080303F1FF331B7800
:1027800023F00103DBB207F1080107F507720846E1
:1027900011461A46FFF714FC034687F84F3297F8A4
:1027A0004F32002B40F0A78107F50473C7F834328D
:1027B00007F11003C7F8383207F108031B6807F563
:1027C000077210461946FFF703FB034687F84F329E
:1027D000D7F83032C7F8483297F84F32002B07D17C
:1027E000D7F84832002B03D14FF0060387F84F3259
:1027F00007F1080303F1FF331B7803F01C03002BE0
:1028000000F0D78097F84F32002B1CD097F84F324A
:10281000042B07D107F507731846FEF74FFF034651
:1028200087F84F3207F1080303F1FF3307F108027D
:1028300002F1FF32127842F008021A70D7F83032F3
:10284000C7F848321AE0D7F8483203F10B031B7877
:1028500003F01103002B04D04FF0070387F84F3229
:102860000CE007F1080303F1FF331B7803F00403C6
:10287000002B03D04FF0080387F84F3297F84F3200
:10288000002B40F0BF8007F1080303F1FF331B78F2
:1028900003F00803002B00F0B58013F08DFBC7F8A0
:1028A0004402D7F8483203F10E03D7F84422D2B2DB
:1028B0001A70D7F8483203F10F03D7F8442292B2C6
:1028C0004FEA122292B2D2B21A70D7F8483203F10C
:1028D0001003D7F844224FEA1242D2B21A70D7F846
:1028E000483203F11103D7F844224FEA1262D2B200
:1028F0001A70D7F8483203F10B034FF000021A7038
:10290000D7F8483203F11C034FF000021A70D7F8D1
:10291000483203F11D034FF000021A70D7F8483215
:1029200003F11E034FF000021A70D7F8483203F18A
:102930001F034FF000021A70D7F81C321846D7F860
:102940004812FEF7C9FAC7F84002D7F848024FF01C
:102950000001FEF7F7FAD7F81C324FF001021A71A6
:10296000D7F84032002B4DD0D7F81C32DB6AC7F8BD
:102970004432D7F81C321846D7F84012FEF744F814
:10298000034687F84F3297F84F32002B3AD1D7F8E9
:102990001C32D7F8402202F1FF32DA60D7F81C323D
:1029A0001846D7F84412FDF7B7FC034687F84F32B4
:1029B00028E097F84F32002B24D1D7F8483203F1A2
:1029C0000B031B7803F01003002B04D04FF004031B
:1029D00087F84F3216E007F1080303F1FF331B7845
:1029E00003F00203002B0DD0D7F8483203F10B039C
:1029F0001B7803F00103DBB2002B03D04FF0070379
:102A000087F84F3297F84F32002B21D107F1080396
:102A100003F1FF331B7803F00803002B0BD007F101
:102A2000080303F1FF3307F1080202F1FF321278C5
:102A300042F020021A70D7F81C32DA6A07F10C0350
:102A40001B68DA6107F10C031B68D7F848221A6289
:102A500097F84F32002B4ED107F10C031A6807F19B
:102A6000080303F1FF331B789371D7F81C32184623
:102A7000D7F84812FEF730FA024607F10C031B683C
:102A80001A61D7F8483203F11F031B784FEA03623B
:102A9000D7F8483203F11E031B784FEA03431A4369
:102AA000D7F8483203F11D031B784FEA03231A437A
:102AB000D7F8483203F11C031B781A4307F10C03C3
:102AC0001B68DA6007F10C031B684FF000029A6084
:102AD00007F10C031B684FF000029A61D7F81C2223
:102AE00007F10C031B681A60D7F81C32DA8807F16B
:102AF0000C031B689A8097F84F32184607F5147735
:102B0000BD4680BD80B58CB000AFF860B9607A601A
:102B10003B60BB683B623B684FF000021A60F8689C
:102B2000FFF79EFD0346FB77FB7F002B01D0FB7F69
:102B300055E1FB689B79DBB25BB2002B02DA4FF008
:102B400002034CE1FB689B7903F00103002B02D1E7
:102B50004FF0070343E1FB68DA68FB689B68D31A10
:102B6000BB617A68BB699A4240F23381BB697B6082
:102B70002FE1FB689B684FEAC3534FEAD353002B06
:102B800040F0F580FB689B684FEA5323DAB2FB689C
:102B90001B689B7803F1FF33DBB202EA0303FB758A
:102BA000FB7D002B2ED1FB689B68002B03D1FB68BB
:102BB0001B69FB6208E0FB681A68FB685B691046EA
:102BC0001946FDF71DFDF862FB6A012B09D8FB6869
:102BD0009B7963F07F03DAB2FB689A714FF00203CE
:102BE000FDE0FB6AB3F1FF3F09D1FB689B7963F01D
:102BF0007F03DAB2FB689A714FF00103EFE0FB68E4
:102C0000FA6A5A61FB681A68FB685B6910461946E4
:102C1000FDF7D4FC38613B69002B09D1FB689B7937
:102C200063F07F03DAB2FB689A714FF00203D6E0DB
:102C3000FB7D3A69D3183B617B684FEA53237B6283
:102C40007B6A002B48D0FA7D7B6AD218FB681B6830
:102C50009B789A4206D9FB681B689B781A46FB7DD5
:102C6000D31A7B62FB681B685A787B6ADBB210461A
:102C7000396A3A6913F074F90346002B09D0FB68EE
:102C80009B7963F07F03DAB2FB689A714FF001031E
:102C9000A5E0FB689B7903F04003002B17D0FB688D
:102CA0009A693B69D21A7B6A9A4210D2FB689A6988
:102CB0003B69D31A4FEA43233A6AD218FB6803F1FF
:102CC0002403104619464FF40072FDF787FA7B6A19
:102CD0004FEA4323BB6268E0FB689A693B699A420A
:102CE00042D0FB689B7903F04003002B22D0FB68A5
:102CF0001B685978FB6803F12402FB689B6908464E
:102D000011461A464FF0010313F040F90346002B19
:102D100009D0FB689B7963F07F03DAB2FB689A7194
:102D20004FF001035BE0FB689B7923F04003DAB2CC
:102D3000FB689A71FB681B685A78FB6803F12403EF
:102D4000104619463A694FF0010313F009F903469A
:102D5000002B09D0FB689B7963F07F03DAB2FB6834
:102D60009A714FF001033AE0FB683A699A61FB6897
:102D70009B684FEAC3534FEAD353C3F50073BB625A
:102D8000BA6A7B689A4201D97B68BB62FB6803F12F
:102D90002402FB689B684FEAC3534FEAD353D3180E
:102DA000386A1946BA6AFDF719FA3A6ABB6AD31843
:102DB0003B62FB689A68BB6AD218FB689A603B6802
:102DC0001A68BB6AD2183B681A607A68BB6AD31A61
:102DD0007B607B68002B7FF4CCAE4FF0000318467D
:102DE00007F13007BD4680BD80B58AB000AFF860FE
:102DF000B9607A603B60BB68BB613B684FF0000222
:102E00001A60F868FFF72CFC0346FB75FB7D002B6E
:102E100001D0FB7D87E1FB689B79DBB25BB2002BC5
:102E200002DA4FF002037EE1FB689B7903F00203B4
:102E3000002B02D14FF0070375E1FB68DA687B686D
:102E4000D218FB68DB689A4280F054814FF000038F
:102E50007B604FE1FB689B684FEAC3534FEAD35353
:102E6000002B40F00E81FB689B684FEA5323DAB2D7
:102E7000FB681B689B7803F1FF33DBB202EA0303B4
:102E8000BB75BB7D002B40D1FB689B68002B11D12B
:102E9000FB681B697B627B6A002B14D1FB681B6893
:102EA00018464FF00001FDF707FE7862FB687A6A6A
:102EB0001A6108E0FB681A68FB685B6910461946EE
:102EC000FDF7FAFD78627B6A002B00F018817B6ABF
:102ED000012B09D1FB689B7963F07F03DAB2FB68B1
:102EE0009A714FF002031EE17B6AB3F1FF3F09D1F3
:102EF000FB689B7963F07F03DAB2FB689A714FF04D
:102F0000010310E1FB687A6A5A61FB689B7903F060
:102F10004003002B22D0FB681B685978FB6803F143
:102F20002402FB689B69084611461A464FF00103CC
:102F300013F02CF80346002B09D0FB689B7963F053
:102F40007F03DAB2FB689A714FF00103EBE0FB6894
:102F50009B7923F04003DAB2FB689A71FB681A6828
:102F6000FB685B6910461946FDF728FB38613B6931
:102F7000002B09D1FB689B7963F07F03DAB2FB6811
:102F80009A714FF00203CEE0BB7D3A69D3183B61E2
:102F90007B684FEA5323FB61FB69002B49D0BA7D64
:102FA000FB69D218FB681B689B789A4206D9FB68BC
:102FB0001B689B781A46BB7DD31AFB61FB681B68B4
:102FC0005A78FB69DBB21046B9693A6912F0DEFF44
:102FD0000346002B09D0FB689B7963F07F03DAB2CC
:102FE000FB689A714FF001039DE0FB689A693B69A9
:102FF000D21AFB699A4217D2FB6803F12402FB68DC
:1030000099693B69CB1A4FEA4323B969CB1810463B
:1030100019464FF40072FDF7E1F8FB689B7923F045
:103020004003DAB2FB689A71FB694FEA43233B62C3
:103030004CE0FB689A693B699A421FD0FB689A682A
:10304000FB68DB689A4219D2FB681B685A78FB68F8
:1030500003F12403104619463A694FF0010312F0B8
:103060007FFF0346002B09D0FB689B7963F07F0349
:10307000DAB2FB689A714FF0010354E0FB683A69D9
:103080009A61FB689B684FEAC3534FEAD353C3F579
:1030900000733B623A6A7B689A4201D97B683B6263
:1030A000FB6803F12402FB689B684FEAC3534FEAB5
:1030B000D353D3181846B9693A6AFDF78FF8FB68FD
:1030C0009B7943F04003DAB2FB689A71BA693B6AB4
:1030D000D318BB61FB689A683B6AD218FB689A6098
:1030E0003B681A683B6AD2183B681A607A683B6A88
:1030F000D31A7B607B68002B7FF4ACAE00E000BF8E
:10310000FB689A68FB68DB689A4203D9FB689A6897
:10311000FB68DA60FB689B7943F02003DAB2FB6856
:103120009A714FF00003184607F12807BD4680BD8D
:1031300080B586B000AF78607868FFF791FA0346F3
:10314000FB75FB7D002B40F0B0807B689B7903F022
:103150002003002B00F0A9807B689B7903F04003DB
:10316000002B1BD07B681B6859787B6803F1240215
:103170007B689B69084611461A464FF0010312F01E
:1031800005FF0346002B02D04FF001038EE07B6861
:103190009B7923F04003DAB27B689A717B681A68E6
:1031A0007B68DB6910461946FDF7B6F80346FB75E8
:1031B000FB7D002B79D17B681B6A3B613B6903F186
:1031C0000B033A6902F10B02127842F02002D2B2EC
:1031D0001A703B6903F11C037A68D268D2B21A7084
:1031E0003B6903F11D037A68D26892B24FEA12225A
:1031F00092B2D2B21A703B6903F11E037A68D268A8
:103200004FEA1242D2B21A703B6903F11F037A6887
:10321000D2684FEA1262D2B21A707B681B693869B1
:103220001946FDF78FFE12F0C7FEF8603B6903F107
:103230001603FA68D2B21A703B6903F11703FA68F1
:1032400092B24FEA122292B2D2B21A703B6903F1E3
:103250001803FA684FEA1242D2B21A703B6903F1BE
:103260001903FA684FEA1262D2B21A703B6903F18D
:1032700012034FF000021A703B6903F113034FF081
:1032800000021A707B689B7923F02003DAB27B6816
:103290009A717B681B684FF001021A717B681B688A
:1032A0001846FDF7A3F80346FB75FB7D184607F1AA
:1032B0001807BD4680BD00BF80B584B000AF786000
:1032C0007868FFF735FF0346FB73FB7B002B03D1C8
:1032D0007B684FF000021A60FB7B184607F110076D
:1032E000BD4680BD80B588B000AF78603960786831
:1032F000FFF7B6F90346FB75FB7D002B01D0FB7D84
:1033000057E17B689B79DBB25BB2002B02DA4FF0AE
:1033100002034EE17B68DA683B689A4208D27B6818
:103320009B7903F00203002B02D17B68DB683B60D2
:103330007B689B683B614FF00003BB617B68BA69A7
:103340009A603B68002B00F0CF807B681B689B78FD
:103350004FEA4323FB603B69002B1FD03B6803F11E
:10336000FF32FB68B2FBF3F23B6903F1FF31FB680C
:10337000B1FBF3F39A4211D33B6903F1FF32FB68CF
:10338000C3F100031A407B689A607B689B683A68C7
:10339000D31A3B607B685B69FB612EE07B681B692D
:1033A000FB61FB69002B25D17B681B6818464FF039
:1033B0000001FDF781FBF861FB69012B09D17B68F6
:1033C0009B7963F07F03DAB27B689A714FF0020356
:1033D000EFE0FB69B3F1FF3F09D17B689B7963F0B4
:1033E0007F03DAB27B689A714FF00103E1E07B68FA
:1033F000FA691A617B68FA695A61FB69002B73D01C
:1034000047E07B689B7903F00203002B0CD07B68BC
:103410001B681846F969FDF74FFBF861FB69002B43
:1034200009D1FB683B6038E07B681B681846F96986
:10343000FDF7E6F8F861FB69B3F1FF3F09D17B685E
:103440009B7963F07F03DAB27B689A714FF00103D6
:10345000AFE0FB69012B05D97B681B689A69FB69A2
:103460009A4209D87B689B7963F07F03DAB27B6864
:103470009A714FF002039CE07B68FA695A617B689D
:103480009A68FB68D2187B689A603A68FB68D31A1E
:103490003B603A68FB689A42B3D87B689A683B689D
:1034A000D2187B689A603B684FEAC3534FEAD35304
:1034B000002B19D07B681B681846F969FDF77EF868
:1034C000B861BB69002B09D17B689B7963F07F03EE
:1034D000DAB27B689A714FF002036AE03B684FEA08
:1034E0005323BA69D318BB617B689B684FEAC35307
:1034F0004FEAD353002B4AD07B689A69BB699A4242
:1035000045D07B689B7903F04003002B22D07B6879
:103510001B6859787B6803F124027B689B69084625
:1035200011461A464FF0010312F030FD0346002BFE
:1035300009D07B689B7963F07F03DAB27B689A716C
:103540004FF0010335E07B689B7923F04003DAB24A
:103550007B689A717B681B685A787B6803F1240347
:1035600010461946BA694FF0010312F0F9FC034600
:10357000002B09D07B689B7963F07F03DAB27B680C
:103580009A714FF0010314E07B68BA699A617B6815
:103590009A687B68DB689A420AD97B689A687B687C
:1035A000DA607B689B7943F02003DAB27B689A711A
:1035B000FB7D184607F12007BD4680BD80B5ADF5FF
:1035C0001A7D00AF07F10403186007F1040207F544
:1035D0000E73104619464FF00102FEF7F1FC034648
:1035E00087F8673297F86732002B40F0B18007F513
:1035F0000273C7F8503207F10803C7F8543207F1D5
:1036000004031B6807F50E7210461946FEF7E0FB2F
:10361000034687F8673297F86732002B40F09880AE
:10362000D7F84C32C7F86032D7F86032002B04D19B
:103630004FF0060387F867320DE0D7F8603203F1E8
:103640000B031B7803F00103DBB2002B03D04FF018
:10365000070387F86732D7F838321846D7F8601270
:10366000FDF73AFCC7F85C0297F86732002B45D1AA
:10367000D7F8603203F10B031B7803F01003002B23
:103680003CD0D7F85C32012B04D84FF0020387F806
:10369000673233E007F5057207F50E7310461946D9
:1036A0004FF02402FCF79AFDD7F85C32C7F81C32C1
:1036B00007F5057318464FF00201FDF793FA03462C
:1036C00087F8673297F86732002B17D107F5057333
:1036D0001846FDF74DFF034687F8673297F86732C3
:1036E000002B03D14FF0070387F8673297F8673252
:1036F000042B03D14FF0000387F8673297F8673245
:10370000002B25D107F50E731846FEF72FF9034657
:1037100087F8673297F86732002B19D1D7F85C32F7
:10372000002B09D0D7F838321846D7F85C12FDF7CD
:103730006BF9034687F8673297F86732002B07D199
:10374000D7F838321846FCF751FE034687F867323F
:1037500097F86732184607F51A77BD4680BD00BF57
:1037600090B5ADF5217D00AF07F1040318603B462D
:10377000196007F1040207F51473104619464FF05B
:103780000102FEF71DFC034687F87F3297F87F326F
:10379000002B40F0FA80D7F85032C7F82C3207F5EA
:1037A0000273C7F8683207F10803C7F86C3207F1F3
:1037B00004031B6807F5147210461946FEF708FB50
:1037C000034687F87F3297F87F32002B40F0DD8088
:1037D000D7F86432002B04D14FF0040387F87F320E
:1037E000D3E0D7F8643203F10B0307F505721046F6
:1037F00019464FF01502FCF7F1FC07F50B7207F5BF
:103800001473104619464FF02402FCF7E7FC07F545
:103810000B723B4610461968FEF7DAFA034687F842
:103820007F3297F87F32002B03D14FF0080387F8DF
:103830007F3297F87F32042B40F0A78007F50B7397
:103840001846FDF73BFF034687F87F3297F87F3233
:10385000002B40F09A80D7F84032C7F87832D7F87A
:10386000783203F10D0207F5057303F102031046E8
:1038700019464FF01302FCF7B1FCD7F8783203F188
:103880000B0397F8142242F02002D2B21A70D7F834
:1038900050324FF001021A71D7F85822D7F834325B
:1038A0009A425AD0D7F8783203F10B031B7803F011
:1038B0001003002B51D0D7F85042D7F85032184699
:1038C000D7F87812FDF708FB034620461946FCF7A7
:1038D00075FEC7F87402D7F87432002B04D14FF08C
:1038E000020387F87F3238E0D7F850321846D7F80D
:1038F0007412FCF711FD034687F87F32D7F8503277
:1039000003F15003C7F8783297F87F32002B24D1A7
:10391000D7F8783203F101031B782E2B1DD1D7F88D
:1039200050321B78032B06D1D7F83422D7F8503207
:103930005B6A9A4202D0D7F8343201E04FF00003BC
:10394000C7F87432D7F87802D7F87412FDF7FAFA8C
:10395000D7F850324FF001021A7197F87F32002BDE
:1039600013D107F514731846FEF700F8034687F8DD
:103970007F3297F87F32002B07D1D7F850321846A4
:10398000FCF734FD034687F87F3297F87F321846FC
:1039900007F52177BD4690BD80B485B000AF0346E2
:1039A0003960FB80FB887F2B02D8FB88FB8131E0EC
:1039B0003B68002B10D0FB88FF2B09D8FB88A3F1B4
:1039C000800248F6F423C0F2040333F8123001E019
:1039D0004FF00003FB811DE04FF00003FB810DE081
:1039E000FA8948F6F423C0F2040333F81230FA8857
:1039F0009A4207D0FB8903F10103FB81FB897F2BEE
:103A0000EED900E000BFFB8903F180039BB203F015
:103A1000FF03FB81FB89184607F11407BD4680BCF4
:103A2000704700BF80B485B000AF0346FB804FF005
:103A30000003FB6003E0FB6803F10103FB6048F651
:103A4000F433C0F20403FA6833F81230002B09D0C3
:103A500048F6F433C0F20403FA6833F81230FA88F7
:103A60009A42E8D148F6F433C0F20403FA6833F816
:103A70001230002B07D048F6D453C0F20403FA6882
:103A800033F8123000E0FB88184607F11407BD46F2
:103A900080BC704780B582B000AF7860786819F05C
:103AA000BBF80346184607F10807BD4680BD00BFB6
:103AB00080B584B000AFF860B9607A603B60FB68A5
:103AC000BA681A60FB687A685A60FB683A689A605C
:103AD000FB683A7F5A73FB683A7E9A7378684FF0B6
:103AE000000118F0B7FF38684FF0000118F0B2FF7E
:103AF000F86800F013F8FB68184607F11007BD4698
:103B000080BD00BF80B582B000AF7860786800F0FB
:103B100005F807F10807BD4680BD00BF80B584B039
:103B200000AF78604FF00003FB737B685B6818465A
:103B30004FF0010118F08EFF7B689B6818464FF02C
:103B4000010118F087FF4FF00803BB7330E04FF01E
:103B500001000BF07BFE7B685B6818464FF00001AC
:103B600018F078FF4FF001000BF070FE7B685B6887
:103B700018464FF0010118F06DFF4FF001000BF0F7
:103B800065FE7B681B681846FFF784FF0346002B21
:103B90000AD0BB7B03F1FF334FF0010202FA03F3BB
:103BA000DAB2FB7BD318FB73BB7B03F1FF33BB7330
:103BB000BB7B002B0CBF00230123DBB2002BC6D143
:103BC0007B689B6818464FF0000118F043FF7B6844
:103BD0005B6818464FF0000118F03CFF7B68FA7BE9
:103BE0001A7307F11007BD4680BD00BF80B483B0D3
:103BF00000AF78607B681B7B184607F10C07BD4659
:103C000080BC704780B582B000AF78607868FFF7FD
:103C1000EDFF03461A467B685B7B82EA0303DBB257
:103C2000DAB27B689B7B6FEA0303DBB2DBB202EAAA
:103C30000303DBB2DBB2184607F10807BD4680BDBF
:103C400080B483B000AF78607B681B78184607F1BA
:103C50000C07BD4680BC704780B483B000AF78606D
:103C60007B685B78184607F10C07BD4680BC70473F
:103C700080B483B000AF786039603B68184607F1C4
:103C80000C07BD4680BC704780B582B000AF78603D
:103C90007B68184600F0A2F97B6803F10C03184614
:103CA00000F0CCF97B68184607F10807BD4680BDD7
:103CB0007B68184600F0A0F92CF034F890B58BB072
:103CC00002AFF860B9607A60FB68BA681A60FB6896
:103CD0007A685A60FB6803F108031846796819F09E
:103CE000F5FEFB684FF00002DA62FB684FF000025D
:103CF0001A6343F6DD63C0F200037B614FF00003FB
:103D0000BB61BB6900937B6978684FF01501FA6865
:103D100000F0A2F9B868FFF793FF03461C46B868A5
:103D2000FFF79AFF03464FF0010202FA03F3204621
:103D300019464FF0000227F0ABFBB868FFF780FF91
:103D400003461C46B868FFF787FF03464FF00102A1
:103D500002FA03F3204619464FF0010227F098FBC0
:103D60004FF01503FB774FF46143CEF2000397F950
:103D70001F204FEA5212F97F01F01F014FF001009E
:103D800000FA01F143F82210FB68184607F12407F6
:103D9000BD4690BDFB6803F10803184619F05CFFAF
:103DA0002BF0C0FF80B584B000AF7860786800F079
:103DB00051F80346FB60FB68002B01D10C4B12E06D
:103DC000F86833F04DF9034618460A4933F054FABF
:103DD00003460948194633F04FFA03461846074987
:103DE00033F096F90346184607F11007BD4680BD2B
:103DF00000000000002474490000803F0000704271
:103E000090B585B000AF7860786800F023F803467D
:103E1000FB60786800F040F80346BB60FB68002B4D
:103E200002D0BB68002B01D1094B0CE0B86833F01D
:103E300017F90446F86833F013F90346204619468B
:103E400033F01AFA0346184607F11407BD4690BD31
:103E50000000000080B582B000AF78607B6803F19D
:103E6000080318461AF0ACF903461A464AF2201322
:103E7000C0F207039A4294BF00230123DBB2002B58
:103E800002D04FF0000301E07B68DB6A184607F1BF
:103E90000807BD4680BD00BF80B582B000AF786026
:103EA0007B6803F1080318461AF08AF903461A469C
:103EB0004AF22013C0F207039A4294BF0023012361
:103EC000DBB2002B02D04FF0000301E07B681B6BDC
:103ED000184607F10807BD4680BD00BF90B585B004
:103EE00000AF78607B681B681846FFF7A9FE0346A1
:103EF0001C467B681B681846FFF7AEFE034620464B
:103F000019464FF0010227F08FFB0346002B0CBF30
:103F100000230123DBB2002B03D04FF00003FB731F
:103F20001DE07B681B681846FFF78AFE03461C46A7
:103F30007B681B681846FFF78FFE0346204619462C
:103F40004FF0000227F070FB0346002B0CBF00234C
:103F50000123DBB2002B3CD04FF00103FB737B68E5
:103F60001B681846FFF76CFE03461C467B681B68FF
:103F70001846FFF771FE03464FF0010202FA03F301
:103F80002046194627F0B0FBFB7B83F00103DBB230
:103F9000002B10D07B6803F1080318461AF010F9C3
:103FA00003461A467B68DA627B6803F10803184609
:103FB0001AF032F80EE0FB7B002B0BD07B6803F18C
:103FC000080318461AF0FCF803461A467B681A6381
:103FD00000E000BF07F11407BD4690BD80B582B078
:103FE00000AF78607B68184600F0A4F87B6818463C
:103FF00007F10807BD4680BDB0B582B000AF78605C
:104000007B681D687B685C687B68184600F0C4F8B4
:104010000346284621461A4600F0CAF87B6818462F
:1040200000F096F87B68184607F10807BD46B0BD5A
:104030007B68184600F08CF82BF074FE80B582B0D7
:1040400000AF78607B68184600F0C0F87B681846BF
:1040500007F10807BD4680BD82B090B585B000AFBE
:10406000F8607A607B620B46FB727B6A002B04D19E
:10407000BB6A03F00103002B43D07B68002B42D0C6
:10408000FA6897F90B304FEA8303D3181B68002BAB
:1040900023D14FF018002CF0DBFC03461C462346CE
:1040A0004FF000021A604FF000025A604FF0000219
:1040B0009A604FF00002DA604FF000021A614FF090
:1040C00000025A611846FFF7DFFDFA6897F90B30D6
:1040D0004FEA8303D31822461A60FA6897F90B3027
:1040E0004FEA8303D3181B681846796807F1240345
:1040F0000CCB00F015F907E020462BF0B7FD2BF0B4
:1041000011FE00BF00E000BF07F11407BD46BDE887
:10411000904002B0704700BF80B582B000AF7860B9
:104120007B68184600F048F97B68184607F10807D5
:10413000BD4680BD80B582B000AF78607B68184610
:1041400000F020F97B68184607F10807BD4680BDDE
:1041500080B582B000AF78607B681A687B689B6826
:1041600019467B681B68CB1A4FEAA303786811468F
:104170001A4600F02FF97B681846FFF7CDFF7B68E1
:10418000184607F10807BD4680BD7B681846FFF753
:10419000C3FF2BF0C7FD00BF80B483B000AF7860D1
:1041A0007B68184607F10C07BD4680BC704700BF0E
:1041B00080B584B000AFF860B9607A60F868B9681B
:1041C00000F01CF907F11007BD4680BD80B582B034
:1041D00000AF78607B68184600F01EF97B681846CF
:1041E00007F10807BD4680BD80B483B000AF78609A
:1041F0007B685B681A467B681B68D31A4FEAA30387
:10420000184607F10C07BD4680BC704780B483B0E8
:1042100000AF786039607B681A683B684FEA8303B7
:10422000D318184607F10C07BD4680BC704700BF85
:1042300080B584B000AF78607B6807F10C0210464F
:10424000194600F003F9FB68184607F11007BD4650
:1042500080BD00BF80B584B000AF786039607B68F6
:104260001A683B681B684FEA8303D318FB6007F1A9
:10427000080207F10C031046194600F0E7F8BB6886
:10428000184607F11007BD4680BD00BF90B587B046
:1042900000AF786039604FF00103FB603A4607F1E8
:1042A0000C0310461946FFF7D5FF0346BB6078683C
:1042B00000F0DCF803463B6107F1080207F1100348
:1042C0001046194600F0E6F80346002B13D04FF0D5
:1042D00001037B613A4607F1140310461946FFF7C4
:1042E000B9FF0446786800F0C1F803462046194635
:1042F0003A6800F0E9F87B685B68A3F104027B6828
:104300005A607B681A467B685B681046194600F065
:10431000F5F83B68184607F11C07BD4690BD00BF85
:1043200090B587B000AFF860B960394681E80C00FD
:10433000BB68002B21D03B68002B04D17B6803F0C5
:104340000103002B19D04FF010002CF081FB034625
:104350001C462346184600F0EBF87C617869B96882
:104360003B460CCB00F004F9FA687B693B6107F12E
:1043700010031046194600F01FF907F11C07BD464F
:1043800090BD00BF80B582B000AF78607B681846F2
:1043900000F03AF97B684FF000021A607B684FF03A
:1043A00000025A607B684FF000029A607B681846F2
:1043B00007F10807BD4680BD80B582B000AF7860C8
:1043C0007B68184600F02EF97B68184607F108074D
:1043D000BD4680BD80B584B000AFF860B9607A603A
:1043E000BB68002B05D0FB681846B9687A6800F0F6
:1043F00025F907F11007BD4680BD00BF80B582B02A
:1044000000AF786039607868396800F025F907F105
:104410000807BD4680BD00BF80B582B000AF7860A0
:104420007B68184600F022F97B684FF000021A60A2
:104430007B684FF000025A607B684FF000029A6080
:104440007B68184607F10807BD4680BD80B483B07D
:1044500000AF786039603B681A687B681A607B68D7
:10446000184607F10C07BD4680BC704780B584B084
:1044700000AF78607B6803F1040307F10C0210467B
:104480001946FFF7E3FFFB68184607F11007BD4622
:1044900080BD00BF90B583B000AF786039607868A8
:1044A00000F0F2F803461C68386800F0EDF80346A7
:1044B0001B689C420CBF00230123DBB2184607F1A6
:1044C0000C07BD4690BD00BF90B585B000AFF86049
:1044D000B9607A60F86800F0E3F80446B86800F064
:1044E000DFF80346204619467A6800F0E7F80346ED
:1044F000184607F11407BD4690BD00BF80B483B0D5
:1045000000AF7860396007F10C07BD4680BC70478A
:1045100080B483B000AF78607B68044A1A607B681F
:10452000184607F10C07BD4680BC7047E88F0400B1
:1045300080B582B000AF78607B681846FFF7E8FF6F
:104540007B680A4A1A607B684FF000025A607B68F9
:104550004FF000029A607B684FF00002DA607B68DF
:10456000184607F10807BD4680BD00BFD88F04007C
:1045700080B485B000AFF860B960394681E80C00BE
:10458000BB68002B12D03B68002B04D17B6803F082
:104590000103002B0AD0FB68BA685A60FB6803F17C
:1045A00008033A4692E8030083E8030007F1140782
:1045B000BD4680BC704700BF80B582B000AF786058
:1045C00039607B685A687B689B689A420FD07B6829
:1045D0001A467B685B68104619463A6800F098F8FE
:1045E0007B685B6803F104027B685A6008E07868C6
:1045F000FFF73CFF0346786819463A6800F0A0F8D8
:1046000007F10807BD4680BD80B582B000AF786075
:104610007B68184600F08CF97B68184607F108079C
:10462000BD4680BD80B483B000AF78607B6818461B
:1046300007F10C07BD4680BC704700BF80B584B051
:1046400000AFF860B9607A60B8682BF00FFB07F133
:104650001007BD4680BD00BF80B483B000AF786056
:10466000396007F10C07BD4680BC704780B582B049
:1046700000AF78607B68184600F066F97B681846E2
:1046800007F10807BD4680BD80B483B000AF7860F5
:104690007B68184607F10C07BD4680BC704700BF19
:1046A00080B582B000AF7860786800F06DF903469D
:1046B000184607F10807BD4680BD00BFB0B586B0FB
:1046C00000AFF860B9607A60F86800F069F90346F5
:1046D0001D46B86800F064F903461C46786800F08F
:1046E0005FF90346284621461A4600F067F903465B
:1046F0007B6107F1100207F1140310461946FFF71A
:10470000A5FE3B69184607F11807BD46B0BD00BFBE
:1047100080B584B000AFF860B9607A60BB684FF0D4
:1047200004001946FFF7A4FA03461A46002A02D0ED
:104730007A6812681A6007F11007BD4680BD00BF95
:10474000B0B58AB000AFF860B9607A60FB685A68AB
:10475000FB689B689A4232D0FB681946FB685A682E
:10476000FB685B68A3F10403084611461A46FFF78D
:10477000CFFFFB685B6803F10402FB685A607B684B
:104780001B683B6207F108031846FFF77DFF0346ED
:104790001968FB685B68A3F10802FB685B68A3F11A
:1047A0000403084611461A4600F01CF907F10803F5
:1047B000184600F031F903463A6A1A60B4E0F86826
:1047C0004FF0010148F6B472C0F2040200F030F973
:1047D0000346FB61F868FFF72BFD03463B6107F1D9
:1047E000080207F110031046194600F06BF9034662
:1047F000BB61FB681846F96900F07CF903467B61F0
:104800007B697B62FB681A46BB694FEA830379695F
:10481000CB18104619467A68FFF77AFF4FF000036D
:104820007B62FB681D6807F108031846FFF72CFF41
:1048300003461C68FB681846FFF7AEFC0346284693
:1048400021467A6900F06EF903467B627B6A03F1C8
:1048500004037B6207F108031846FFF715FF0346C0
:104860001D68FB685C68FB681846FFF795FC03460B
:10487000284621467A6A00F055F903467B62FB68B8
:104880001D68FB685C68FB681846FFF785FC0346FB
:10489000284621461A46FFF78BFCF968FB681A6820
:1048A000FB689B681846FB681B68C31A4FEAA303A2
:1048B000084611461A46FFF78DFDFB687A691A60B3
:1048C000FB687A6A5A60FB694FEA83037A69D218F7
:1048D000FB689A6028E02BF027FC2BF023FA0346B4
:1048E00018462BF0D7FB7B6A002B0BD1FB681A46CE
:1048F000BB694FEA83037969CB1810461946FFF765
:10490000FDFD09E0FB681846FFF746FC03467869A1
:10491000796A1A46FFF74CFCFB6818467969FA6910
:10492000FFF758FD2BF0E8FF07F12807BD46B0BDA3
:1049300080B483B000AF78607B68184607F10C073D
:10494000BD4680BC704700BF80B483B000AF7860C4
:104950007B68184607F10C07BD4680BC704700BF56
:1049600080B483B000AF786039607B681A683B68B8
:104970001B689A4201D23B6800E07B68184607F149
:104980000C07BD4680BC704780B483B000AF786030
:104990007B68184607F10C07BD4680BC704700BF16
:1049A00080B582B000AF7860786800F0CFF8034639
:1049B000184607F10807BD4680BD00BF80B586B028
:1049C00000AFF860B9607A604FF00103FB75F868DA
:1049D000B9687A6800F0CAF80346184607F1180764
:1049E000BD4680BD90B585B000AFF860B9607A6013
:1049F000F86800F0DDF803461C46B86800F0D8F807
:104A00000346204619467A6800F0E0F80346184647
:104A100007F11407BD4690BD80B483B000AF786045
:104A20007B681B68184607F10C07BD4680BC7047C1
:104A300090B587B000AFF860B9607A60F86800F0B0
:104A4000E3F803461C46F868FFF7CEFB0346E21A7C
:104A5000BB689A422CBF00230123DBB2002B02D09B
:104A600078682AF0CBFAF868FFF7BEFB0446F868CE
:104A7000FFF7BAFB03463B6107F1100207F1080399
:104A800010461946FFF76CFF03461B68E3187B616D
:104A9000F868FFF7A9FB02467B699A4207D8F868D5
:104AA00000F0B2F803461A467B699A4204D2F868CD
:104AB00000F0AAF8034600E07B69184607F11C07DE
:104AC000BD4690BD90B583B000AF7860396078681E
:104AD000FFF7DAFD03461B681C463868FFF7D4FD74
:104AE00003461B68E31A4FEAA303184607F10C07B5
:104AF000BD4690BD80B582B000AF786039603B683C
:104B0000002B08D07B68184639684FF0000200F08F
:104B10008DF8034601E04FF00003184607F108073F
:104B2000BD4680BD80B584B000AFF860B9607A60E2
:104B30003B60F868B9687A683B6800F097F803460C
:104B4000184607F11007BD4680BD00BF80B582B092
:104B500000AF786007F104031846FFF795FD0346A0
:104B60001B68184607F10807BD4680BD80B586B0B2
:104B700000AFF860B9607A60BA68FB68D31A4FEA90
:104B8000A3037B617B69002B07D07B694FEA83031A
:104B90007868F9681A4636F02DFE7B694FEA830380
:104BA0007A68D318184607F11807BD4680BD00BFC4
:104BB00080B582B000AF7860786800F069F803468D
:104BC000184607F10807BD4680BD00BFB0B584B0E8
:104BD00000AFF860B9607A60F86800F065F80546E3
:104BE000B86800F061F80446786800F05DF80346A4
:104BF000284621461A4600F065F80346184607F194
:104C00001007BD46B0BD00BF80B582B000AF786070
:104C10007B68184600F06AF80346184600F072F800
:104C20000346184607F10807BD4680BD80B584B02D
:104C300000AFF860B9607A60F86800F063F8024687
:104C4000BB689A422CBF00230123DBB2002B01D0AA
:104C50002AF090F9BB684FEA830318462BF0F8FE60
:104C60000346184607F11007BD4680BD80B584B0E5
:104C700000AFF860B9607A603B60F868B9687A683C
:104C800000F04CF80346184607F11007BD4680BDFA
:104C900080B483B000AF78607B68184607F10C07DA
:104CA000BD4680BC704700BF80B582B000AF786061
:104CB0007868FFF7EDFF0346184607F10807BD4681
:104CC00080BD00BF80B586B000AFF860B9607A6083
:104CD0004FF00103FB75F868B9687A6800F030F8A6
:104CE0000346184607F11807BD4680BD80B483B05F
:104CF00000AF78607B68184607F10C07BD4680BCA2
:104D0000704700BF80B483B000AF78606FF040435D
:104D1000184607F10C07BD4680BC704780B584B0CB
:104D200000AFF860B9607A60F868B9687A6800F036
:104D300031F80346184607F11007BD4680BD00BF95
:104D400080B586B000AFF860B9607A60BA68FB6879
:104D5000D31A4FEAA3037B617B69002B0ED07B69DA
:104D60004FEA8303C3F100037A68D2187B694FEAE4
:104D700083031046F9681A4636F03CFD7B694FEA1A
:104D80008303C3F100037A68D318184607F11807A4
:104D9000BD4680BD80B584B000AFF860B9607A6070
:104DA000F868B9687A6800F007F80346184607F112
:104DB0001007BD4680BD00BF90B585B000AFF8605C
:104DC000B9607A60F868FFF7F3FE03461C46B868DE
:104DD000FFF7EEFE0346204619467A6800F006F813
:104DE0000346184607F11407BD4690BDB0B584B020
:104DF00000AFF860B9607A60F868FFF755FF0546C4
:104E0000B868FFF751FF04467868FFF74DFF034687
:104E1000284621461A46FFF7D1FD0346184607F1FA
:104E20001007BD46B0BD00BF80B582B000AF78604E
:104E30007B685B68002B28D07B689B68002B05D1C2
:104E40007B68DB6803F00103002B1ED07B68DB6806
:104E500003F00103DBB2002B0CD07B685A687B683F
:104E6000DB684FEA6303D3181A687B689B68D31822
:104E70001B6801E07B689B687A6851687A68D26831
:104E80004FEA62028A181046984707F10807BD46A4
:104E900080BD00BF90B58BB002AFF860B9607A609A
:104EA000FB68BA681A60FB687A685A60FB6803F1AD
:104EB0000803184618F0F6FDFB6803F12C031846AA
:104EC00018F0F0FDFB684FF00002A3F8502044F604
:104ED0009173C0F200037B614FF00003BB61BB69BB
:104EE00000937B6978684FF01501FA6800F0B8F913
:104EF000B868FEF7A5FE03461C46B868FEF7ACFE90
:104F000003464FF0010202FA03F3204619464FF020
:104F1000000226F0BDFAB868FEF792FE03461C4672
:104F2000B868FEF799FE03464FF0010202FA03F358
:104F3000204619464FF0010226F0AAFA4FF0150359
:104F4000FB774FF46143CEF2000397F91F204FEA3D
:104F50005212F97F01F01F014FF0010000FA01F138
:104F600043F82210FB68184607F12407BD4690BDA0
:104F7000FB6803F12C03184618F06EFEFFE7FB6890
:104F800003F10803184618F067FE2AF0CBFE00BFB5
:104F900090B587B000AF78607B681B681846FEF755
:104FA0004FFE03461C467B681B681846FEF754FEFE
:104FB0000346204619464FF0010226F035FB034612
:104FC000002B0CBF00230123DBB2002B03D04FF0DA
:104FD0000003FB751EE07B681B681846FEF730FE79
:104FE00003461C467B681B681846FEF735FE0346E1
:104FF000204619464FF0000226F016FB0346002B10
:105000000CBF00230123DBB2002B00F023814FF003
:105010000103FB757B681B681846FEF711FE03460B
:105020001C467B681B681846FEF716FE03464FF0C9
:10503000010202FA03F32046194626F055FB7B686D
:1050400003F12C03184619F0BBF803463B617B685B
:1050500003F12C03184618F0DFFF3A694EF65F2380
:105060009A4206D940F63213C1F200034FF0000213
:105070001A7040F63213C1F200031B7883F001036B
:10508000DBB2002B1CD040F63213C1F200034FF00C
:1050900001021A7040F63313C1F200034FF0000210
:1050A0001A7040F63413C1F200034FF000021A7078
:1050B00040F63613C1F200034FF000021A80CAE036
:1050C00040F63413C1F200031B78002B09D040F6E0
:1050D0003413C1F200031A7840F63413C1F200030E
:1050E0001A7040F63313C1F200031B78002B02D074
:1050F0004FF0010301E04FF00003FB7326E0F97B62
:1051000040F63413C1F200031A78134601FA03F390
:1051100099B240F63613C1F200031B88CB1899B23E
:1051200040F63613C1F20003198002F10103DAB22E
:1051300040F63413C1F200031A703A6940F69F73C7
:105140009A420ED93B69A3F57A633B613A6940F212
:10515000CF739A4294BF00230123DBB2002BCED140
:1051600000E000BF40F63413C1F200031B780C2BA3
:1051700026D1FB7D002B02D04FF0010301E04FF060
:105180000003FB73F97B40F63413C1F200031A7875
:10519000134601FA03F399B240F63613C1F2000345
:1051A0001B88CB1899B240F63613C1F20003198060
:1051B00002F10103DAB240F63413C1F200031A70AF
:1051C00040F63413C1F200031B780D2B2DD140F6AD
:1051D0003613C1F200031B8803F48053002B0CBF6D
:1051E00000230123BB7340F63613C1F200031B8872
:1051F00023F4C0539AB240F63613C1F200031A806A
:1052000040F63613C1F200031B884FEA63039AB2DB
:1052100040F63613C1F200031A8040F63613C1F28D
:1052200000031A887B68A3F8502040F63413C1F2BB
:1052300000031B780C2B06D940F63213C1F2000391
:105240004FF000021A7040F63313C1F20003FA7DEA
:105250001A7000E000BF07F11C07BD4690BD00BFFB
:1052600082B090B585B000AFF8607A607B620B4683
:10527000FB727B6A002B04D1BB6A03F00103002B95
:1052800043D07B68002B42D0FA6897F90B304FEA85
:105290008303D3181B68002B23D14FF018002BF089
:1052A000D7FB03461C4623464FF000021A604FF01E
:1052B00000025A604FF000029A604FF00002DA607C
:1052C0004FF000021A614FF000025A611846FEF7D3
:1052D000DBFCFA6897F90B304FEA8303D3182246B8
:1052E0001A60FA6897F90B304FEA8303D3181B68EA
:1052F0001846796807F124030CCB00F011F807E099
:1053000020462AF0B3FC2AF00DFD00BF00E000BFEC
:1053100007F11407BD46BDE8904002B0704700BFDA
:1053200090B587B000AFF860B960394681E80C00ED
:10533000BB68002B21D03B68002B04D17B6803F0B5
:105340000103002B19D04FF010002BF081FB034616
:105350001C462346184600F015F87C617869B96848
:105360003B460CCB00F02EF8FA687B693B6107F1F5
:10537000100310461946FFF71FF907F11C07BD4639
:1053800090BD00BF80B582B000AF78607B681846E2
:10539000FFF7BEF87B680A4A1A607B684FF000028C
:1053A0005A607B684FF000029A607B684FF0000201
:1053B000DA607B68184607F10807BD4680BD00BF6C
:1053C0005090040080B485B000AFF860B9603946F1
:1053D00081E80C00BB68002B12D03B68002B04D185
:1053E0007B6803F00103002B0AD0FB68BA685A609F
:1053F000FB6803F108033A4692E8030083E80300E0
:1054000007F11407BD4680BC704700BF80B582B06D
:1054100000AF78607B685B68002B28D07B689B6856
:10542000002B05D17B68DB6803F00103002B1ED045
:105430007B68DB6803F00103DBB2002B0CD07B68D8
:105440005A687B68DB684FEA6303D3181A687B6885
:105450009B68D3181B6801E07B689B687A68516879
:105460007A68D2684FEA62028A181046984707F1B4
:105470000807BD4680BD00BF80B582B000AF786030
:105480000B46FB70FA787B6802F10C0253F822306D
:10549000002B08D0FA787B6802F10C0253F8223016
:1054A000184600F04DFD07F10807BD4680BD00BF5E
:1054B00080B582B000AF78607B68184600F014FEBB
:1054C0007B6803F10C03184600F03EFE7B6818462B
:1054D00007F10807BD4680BD7B68184600F012FE44
:1054E0002AF020FC90B58BB002AFF860B9607A600A
:1054F0003B60FB68BA681A60FB687A685A60FB68B0
:105500003A689A60FB683A6BDA60FB687A6B1A61FA
:10551000FB68BA6B5A61FB68FA6B9A61FB683A6C7C
:10552000DA61FB687A6C1A62FB68BA6C5A62FB68D3
:1055300003F178031846FFF7BBFFBB681B6803F154
:1055400008031B68B8684FF0010198477B681B6827
:1055500003F108031B6878684FF0010198473B6826
:105560001B6803F108031B6838684FF00101984776
:105570003B6B1B6803F108031B68386B4FF001019C
:1055800098477B6B1B6803F108031B68786B4FF02F
:1055900001019847B8684FF0000117F05BFA78688E
:1055A0004FF0000117F056FA38684FF0000117F07D
:1055B00051FA386B4FF0000117F04CFA786B4FF04E
:1055C000000117F047FAB86B17F05CFBF86B17F0A7
:1055D00059FB386C17F056FB786C17F053FB4FF003
:1055E0000003FB610BE0FB68FA6902F10C024FF06B
:1055F000000143F82210FB6903F10103FB61FB6921
:10560000112B8CBF00230123DBB2002BEBD14FF019
:1056100024002BF01DFA03461C4623461846B96C9D
:1056200018F054FA2246FB689A624FF024002BF0DF
:105630000FFA03461C4623461846B96C18F046FA82
:105640002246FB68DA62FB684FF00002C3F8902044
:1056500045F63143C0F200033B614FF000037B612C
:105660007B6900933B69B86C4FF01501FA6800F054
:10567000D1FDB86BFEF7E4FA03461C46B86BFEF7A3
:10568000EBFA03464FF0010202FA03F320461946F3
:105690004FF0010225F0FCFEF86BFEF7D1FA03464D
:1056A0001C46F86BFEF7D8FA03464FF0010202FAE7
:1056B00003F3204619464FF0010225F0E9FE386C4D
:1056C000FEF7BEFA03461C46386CFEF7C5FA0346E1
:1056D0004FF0010202FA03F3204619464FF001028F
:1056E00025F0D6FE786CFEF7ABFA03461C46786CC4
:1056F000FEF7B2FA03464FF0010202FA03F3204626
:1057000019464FF0010225F0C3FEB86BFEF798FA78
:1057100003461C46B86BFEF79FFA03464FF00102A2
:1057200002FA03F3204619464FF0000225F0B0FEBE
:10573000F86BFEF785FA03461C46F86BFEF78CFA09
:1057400003464FF0010202FA03F3204619464FF0D8
:10575000000225F09DFE386CFEF772FA03461C46E7
:10576000386CFEF779FA03464FF0010202FA03F3B0
:10577000204619464FF0000225F08AFE786CFEF7AD
:105780005FFA03461C46786CFEF766FA03464FF054
:10579000010202FA03F3204619464FF0000225F0F9
:1057A00077FE4FF01503FB764FF46143CEF2000312
:1057B00097F91B204FEA5212F97E01F01F014FF0BA
:1057C000010000FA01F143F82210FB68184607F1C6
:1057D0002407BD4690BD20462AF048FA03E0204643
:1057E0002AF044FAFFE7FB6803F17803184600F05B
:1057F000DBFC2AF097FA00BF80B58EB000AF78606E
:105800007B681B68BB617B685B68FB617B689B682E
:105810003B627B68DB687B627B681B69BB627B6881
:105820005B69BB607B689B69FB607B68DB693B6194
:105830007B681B6A7B614FF000037B634FF00003C2
:105840003B634FF0000387F82F3013E097F82F30B9
:105850004FEA830307F13802D31853F8203C184667
:105860004FF0010117F0F6F897F82F3003F101031C
:1058700087F82F3097F82F30042B8CBF002301239B
:10588000DBB2002BE2D14FF0000387F82E3053E05B
:1058900097F82E304FEA830307F13802D31853F8F4
:1058A000203C18464FF0000117F0D4F84FF00003E9
:1058B00087F82D3023E097F82D304FEA830307F166
:1058C0003802D31853F8303C1846FEF7E3F8034685
:1058D00083F00103DBB2002B07D03B6B4FF00102DA
:1058E00002FA03F37A6BD3187B633B6B03F101037A
:1058F0003B6397F82D3003F1010387F82D3097F8BB
:105900002D30032B8CBF00230123DBB2002BD2D11F
:1059100097F82E304FEA830307F13802D31853F873
:10592000203C18464FF0010117F094F897F82E30FC
:1059300003F1010387F82E3097F82E30042B8CBF2B
:1059400000230123DBB2002BA2D14FF0000387F824
:105950002C3013E097F82C304FEA830307F138021C
:10596000D31853F8203C18464FF0000117F072F896
:1059700097F82C3003F1010387F82C3097F82C307E
:10598000042B8CBF00230123DBB2002BE2D17B6B05
:10599000184607F13807BD4680BD00BF80B58AB004
:1059A00002AF78607868FFF727FF0346FB617B68EA
:1059B000D3F89030002B2AD1FB69002B27D07B68CD
:1059C000DA6A45F69D13C0F20003FB604FF0000356
:1059D0003B614FF0320300931046796807F10C03E6
:1059E0000CCB00F077FC7B68DB6A184618F014FBE0
:1059F0007B68FA69C3F890207B6803F178027B68C2
:105A0000D3F890301046194600F07EFC56E07B68D3
:105A1000D3F89030002B3AD0FB69002B37D07B684D
:105A2000DA6A45F69D13C0F200037B614FF0000374
:105A3000BB614FF0320300931046796807F11403FD
:105A40000CCB00F047FC7B68DB6A184618F0E4FAE0
:105A50007B68D3F890306FEA0303FA6902EA030324
:105A6000FB617B68D3F89020FB691A437B68C3F81D
:105A70009020FB69002B21D07B6803F178027B68C2
:105A8000D3F890301046194600F03EFC16E07B68D3
:105A9000D3F89030002B11D0FB69002B0ED17B681E
:105AA0004FF00002C3F890207B6803F178027B6816
:105AB000D3F890301046194600F026FCFB69B3F588
:105AC000807F00F08780B3F5807F18D8082B00F026
:105AD0009380082B06D8022B58D0042B62D0012BC0
:105AE0003CD0A1E0202B4BD0202B02D8102B2FD064
:105AF0009AE0402B5CD0802B00F0848094E0B3F5DA
:105B0000004F00F08B80B3F5004F10D8B3F5805FE5
:105B10002AD0B3F5805F03D8B3F5006F3CD083E0A3
:105B2000B3F5005F4AD0B3F5804F5FD07CE0B3F5AA
:105B3000003F49D0B3F5003F03D8B3F5803F19D0FB
:105B400072E0B3F5802F4BD0B3F5002F60D06BE03F
:105B500078684FF00001FFF78FFC65E078684FF040
:105B60000101FFF789FC5FE078684FF00201FFF761
:105B700083FC59E078684FF00301FFF77DFC53E0A8
:105B800078684FF00401FFF777FC4DE078684FF03C
:105B90000501FFF771FC47E078684FF00601FFF759
:105BA0006BFC41E078684FF00701FFF765FC3BE0D4
:105BB00078684FF00801FFF75FFC35E078684FF038
:105BC0000901FFF759FC2FE078684FF00A01FFF751
:105BD00053FC29E078684FF00B01FFF74DFC23E000
:105BE00078684FF00C01FFF747FC1DE078684FF034
:105BF0000D01FFF741FC17E078684FF00E01FFF749
:105C00003BFC11E078684FF00F01FFF735FC0BE02B
:105C100078684FF01001FFF72FFC05E078684FF02F
:105C20001101FFF729FC00BF07F12007BD4680BD29
:105C300090B583B000AF78607B685B691846FDF76C
:105C4000FFFF03461C467B685B691846FEF704F8B5
:105C50000346204619464FF0010225F0E5FC0346B5
:105C6000002B41D17B689B691846FDF7E9FF03468D
:105C70001C467B689B691846FDF7EEFF03462046ED
:105C800019464FF0010225F0CFFC0346002B2BD123
:105C90007B68DB691846FDF7D3FF03461C467B682B
:105CA000DB691846FDF7D8FF0346204619464FF03A
:105CB000010225F0B9FC0346002B15D17B681B6A55
:105CC0001846FDF7BDFF03461C467B681B6A184655
:105CD000FDF7C2FF0346204619464FF0010225F0AA
:105CE000A3FC0346002B02D04FF0010301E04FF06C
:105CF0000003002B68D07B689B6A184618F008FAEE
:105D00000346132B94BF00230123DBB2002B02D0E8
:105D10007868FFF743FE7B689B6A184618F07CF9A9
:105D20007B685B691846FDF78BFF03461C467B6862
:105D30005B691846FDF790FF03464FF0010202FA37
:105D400003F32046194625F0CFFC7B689B69184673
:105D5000FDF776FF03461C467B689B691846FDF7F6
:105D60007BFF03464FF0010202FA03F32046194677
:105D700025F0BAFC7B68DB691846FDF761FF034636
:105D80001C467B68DB691846FDF766FF03464FF04B
:105D9000010202FA03F32046194625F0A5FC7B68B0
:105DA0001B6A1846FDF74CFF03461C467B681B6ABE
:105DB0001846FDF751FF03464FF0010202FA03F3C4
:105DC0002046194625F090FC7B685B691846FDF774
:105DD00037FF03461C467B685B691846FDF73CFFAE
:105DE0000346204619464FF0000225F01DFC0346ED
:105DF000002B41D17B689B691846FDF721FF0346C4
:105E00001C467B689B691846FDF726FF0346204623
:105E100019464FF0000225F007FC0346002B2BD15A
:105E20007B68DB691846FDF70BFF03461C467B6861
:105E3000DB691846FDF710FF0346204619464FF070
:105E4000000225F0F1FB0346002B15D17B681B6A8D
:105E50001846FDF7F5FE03461C467B681B6A18468C
:105E6000FDF7FAFE0346204619464FF0000225F0E2
:105E7000DBFB0346002B02D04FF0010301E04FF0A3
:105E80000003002B58D07B689B6A184618F0C4F8B2
:105E90007B685B691846FDF7D3FE03461C467B68AA
:105EA0005B691846FDF7D8FE03464FF0010202FA7F
:105EB00003F32046194625F017FC7B689B691846BA
:105EC000FDF7BEFE03461C467B689B691846FDF73E
:105ED000C3FE03464FF0010202FA03F320461946BF
:105EE00025F002FC7B68DB691846FDF7A9FE034636
:105EF0001C467B68DB691846FDF7AEFE03464FF093
:105F0000010202FA03F32046194625F0EDFB7B68F7
:105F10001B6A1846FDF794FE03461C467B681B6A05
:105F20001846FDF799FE03464FF0010202FA03F30B
:105F30002046194625F0D8FB07F10C07BD4690BD59
:105F400080B586B000AF78607B6803F10C0318461B
:105F500000F040FA78617B69012B1BD17B6803F16B
:105F60000C0318464FF0000100F046FA03461B6888
:105F700098474DE07B69002B14BF00230123FB737E
:105F80007B6803F10C031846796900F035FA034683
:105F90001B6898477B69002B0CBF00230123DBB2F1
:105FA0007A6902F1FF327A61002BE3D17B681846EF
:105FB000FEF71AF938613B69012B1DD17B68184641
:105FC0004FF00001FEF722F903461B681A681268B9
:105FD000184690471CE03B69002B14BF00230123A7
:105FE000BB737B6818463969FEF710F903461B68D6
:105FF0001A681268184690473B69002B0CBF0023B3
:106000000123DBB23A6902F1FF323A61002BE2D19F
:1060100007F11807BD4680BD90B589B000AF786024
:106020007B681846FEF7E0F8F86123E0FB6903F1AE
:10603000FF33FB617B681846F969FEF7E7F8034612
:106040001B68184629F012FE7C687B681846FEF72C
:10605000EFF80346BB60FB69FB6007F1080207F13C
:106060000C0310461946FEF7F5F80346204619467C
:10607000FEF70CF9FB69002B0CBF00230123DBB2F8
:10608000002BD3D17B6803F10C03184600F0A2F972
:10609000B8611DE0BB6903F1FF33BB617B6803F1AD
:1060A0000C047B6803F10C03184600F0B7F90346B3
:1060B0003B61BB697B6107F1100207F114031046D5
:1060C000194600F0BDF903462046194600F0D4F900
:1060D000BB69002B0CBF00230123DBB2002BD9D1FD
:1060E00007F12407BD4690BD80B582B000AF78604F
:1060F0007B68184600F018FA7B68184607F1080715
:10610000BD4680BDB0B582B000AF78607B681D68C9
:106110007B685C687B68184600F038FA03462846BE
:1061200021461A4600F03EFA7B68184600F00AFA4B
:106130007B68184607F10807BD46B0BD7B68184666
:1061400000F000FA29F0EEFD80B582B000AF786073
:106150007B68184600F042FA7B68184607F108078A
:10616000BD4680BDB0B582B000AF78607B681D6869
:106170007B685C687B68184600F062FA0346284634
:1061800021461A4600F068FA7B68184600F034FA97
:106190007B68184607F10807BD46B0BD7B68184606
:1061A00000F02AFA29F0BEFD80B584B000AF786017
:1061B0007B68184600F05EFAF8600DE0FB6803F1BA
:1061C000FF33FB607B681846F96800F065FA034608
:1061D0001B68184629F04AFDFB68002B0CBF002302
:1061E0000123DBB2002BE9D17B6803F10C031846D5
:1061F000FFF7B8FF7B681846FFF784FF7B681846F7
:1062000007F11007BD4680BD7B681846FFF77AFF8F
:1062100029F088FD82B090B585B000AFF8607A6053
:106220007B620B46FB727B6A002B04D1BB6A03F0D6
:106230000103002B43D07B68002B42D0FA6897F90A
:106240000B304FEA8303D3181B68002B23D14FF088
:1062500018002AF0FDFB03461C4623464FF00002BF
:106260001A604FF000025A604FF000029A604FF03F
:106270000002DA604FF000021A614FF000025A612A
:106280001846FDF701FDFA6897F90B304FEA8303D2
:10629000D31822461A60FA6897F90B304FEA830345
:1062A000D3181B681846796807F124030CCB00F05B
:1062B00005FA07E0204629F0D9FC29F033FD00BF9C
:1062C00000E000BF07F11407BD46BDE8904002B0F2
:1062D000704700BF80B586B002AFF860B96039463C
:1062E00081E80C00BB694FF47A7202FB03F3009360
:1062F000F868B9683B460CCB00F012FA184607F173
:106300001007BD4680BD00BF80B584B000AF786087
:1063100039607B6803F10C03184600F04BFAF86013
:10632000FB68012B17D17B6803F10C0318464FF073
:10633000000100F051FA03461B683868984744E0B2
:106340007B6803F10C031846F96800F045FA034630
:106350001B6838689847FB68002B0CBF002301239B
:10636000DBB2FA6802F1FF32FA60002BE8D17B68F9
:10637000184600F07FF9B860BB68012B19D17B6823
:1063800018464FF0000100F087F903461B681A68B1
:10639000126818463968904717E07B681846B96854
:1063A00000F07AF903461B681A68126818463968C3
:1063B0009047BB68002B0CBF00230123DBB2BA68F7
:1063C00002F1FF32BA60002BE7D107F11007BD469A
:1063D00080BD00BF80B483B000AF78607B685B682D
:1063E0001A467B681B68D31A4FEAA303184607F1C5
:1063F0000C07BD4680BC704780B483B000AF7860A6
:1064000039607B681A683B684FEA8303D3181846E3
:1064100007F10C07BD4680BC704700BF80B584B053
:1064200000AF78607B6807F10C021046194600F057
:10643000F9F9FB68184607F11007BD4680BD00BF9B
:1064400080B584B000AF786039607B681A683B68BB
:106450001B684FEA8303D318FB6007F1080207F1BA
:106460000C031046194600F0DDF9BB68184607F129
:106470001007BD4680BD00BF90B587B000AF786003
:1064800039604FF00103FB603A4607F10C031046F8
:106490001946FFF7D5FF0346BB60786800F0AEF9F8
:1064A00003463B6107F1080207F110031046194645
:1064B00000F0C8F90346002B13D04FF001037B61B5
:1064C0003A4607F1140310461946FFF7B9FF044690
:1064D000786800F093F90346204619463A6800F0C0
:1064E000CBF97B685B68A3F104027B685A607B6828
:1064F0001A467B685B681046194600F0D7F93B687E
:10650000184607F11C07BD4690BD00BF80B582B09C
:1065100000AF78607B68184600F0ECF97B6818469D
:1065200007F10807BD4680BD80B582B000AF786036
:106530007B68184600F0C4F97B68184607F1080725
:10654000BD4680BD80B582B000AF78607B681A68B8
:106550007B689B6819467B681B68CB1A4FEAA303CC
:10656000786811461A4600F0D3F97B681846FFF7A1
:10657000CDFF7B68184607F10807BD4680BD7B68E4
:106580001846FFF7C3FF29F0CDFB00BF80B483B0EE
:1065900000AF78607B68184607F10C07BD4680BCE9
:1065A000704700BF80B584B000AFF860B9607A6012
:1065B000F868B96800F0C0F907F11007BD4680BD62
:1065C00080B582B000AF78607B68184600F0DCF9D7
:1065D0007B68184607F10807BD4680BD80B582B0CC
:1065E00000AF78607B68184600F0B4F97B68184605
:1065F00007F10807BD4680BD80B582B000AF786066
:106600007B681A687B689B6819467B681B68CB1A95
:106610004FEAA303786811461A4600F0C3F97B6875
:106620001846FFF7CDFF7B68184607F10807BD46FF
:1066300080BD7B681846FFF7C3FF29F073FB00BFDE
:1066400080B483B000AF78607B68184607F10C0710
:10665000BD4680BC704700BF80B584B000AFF86015
:10666000B9607A60F868B96800F0B0F907F110070E
:10667000BD4680BD80B483B000AF78607B685B6846
:106680001A467B681B68D31A4FEAA303184607F122
:106690000C07BD4680BC704780B483B000AF786003
:1066A00039607B681A683B684FEA8303D318184641
:1066B00007F10C07BD4680BC704700BF90B587B09E
:1066C00000AFF860B960394681E80C00BB68002B68
:1066D00021D03B68002B04D17B6803F00103002B21
:1066E00019D04FF010002AF0B3F903461C46234698
:1066F000184600F079F97C617869B9683B460CCBA3
:1067000000F092F9FA687B693B6107F110031046CB
:106710001946FDF751FF07F11C07BD4690BD00BFAC
:1067200080B586B002AFF860B960394681E80C00E8
:10673000FB689B68002B18D140F25843C1F200035C
:106740001B68DA6849F21C13C0F204030093104678
:1067500049F28401C0F2040149F2B002C0F204021D
:106760004FF0400332F048FFFEE73B68002B04D1B6
:106770007B6803F00103002B17D0BB68002B14D0FB
:10678000FB681B691846FFF747FCFB681B69184646
:10679000B9683B460CCBFFF791FFF868B96917F071
:1067A000B7FDFB684FF001021A77184607F1100792
:1067B000BD4680BD80B483B000AF78607B685B6805
:1067C0001A467B681B68D31A4FEAA303184607F1E1
:1067D0000C07BD4680BC704780B483B000AF7860C2
:1067E00039607B681A683B684FEA8303D318184600
:1067F00007F10C07BD4680BC704700BF80B584B070
:1068000000AF78607B6803F1040307F10C021046C7
:10681000194600F007F8FB68184607F11007BD4657
:1068200080BD00BF80B483B000AF786039603B6842
:106830001A687B681A607B68184607F10C07BD462A
:1068400080BC704790B583B000AF786039607868DD
:1068500000F00EF903461C68386800F009F9034699
:106860001B689C420CBF00230123DBB2184607F1D2
:106870000C07BD4690BD00BF90B585B000AFF86075
:10688000B9607A60F86800F0FFF80446B86800F074
:10689000FBF80346204619467A6800F003F90346E0
:1068A000184607F11407BD4690BD00BF80B483B001
:1068B00000AF7860396007F10C07BD4680BC7047B7
:1068C00080B582B000AF78607B68184600F014F99C
:1068D0007B684FF000021A607B684FF000025A603C
:1068E0007B684FF000029A607B68184607F1080742
:1068F000BD4680BD80B582B000AF78607B68184629
:1069000000F008F97B68184607F10807BD4680BD0E
:1069100080B584B000AFF860B9607A60BB68002BC6
:1069200005D0FB681846B9687A6800F0FFF807F1EF
:106930001007BD4680BD00BF80B582B000AF786053
:1069400039607868396800F0FFF807F10807BD463C
:1069500080BD00BF80B582B000AF78607B6818460C
:1069600000F0FCF87B684FF000021A607B684FF083
:1069700000025A607B684FF000029A607B681846FC
:1069800007F10807BD4680BD80B582B000AF7860D2
:106990007B68184600F0F0F87B68184607F1080796
:1069A000BD4680BD80B584B000AFF860B9607A6044
:1069B000BB68002B05D0FB681846B9687A6800F000
:1069C000E7F807F11007BD4680BD00BF80B582B073
:1069D00000AF786039607868396800F0E7F807F14F
:1069E0000807BD4680BD00BF80B582B000AF7860AB
:1069F0007B681846FDF78CFD7B680A4A1A607B6845
:106A00004FF000025A607B684FF000029A607B688A
:106A10004FF00002DA607B68184607F10807BD46B0
:106A200080BD00BFE890040080B485B000AFF8607E
:106A3000B960394681E80C00BB68002B12D03B6876
:106A4000002B04D17B6803F00103002B0AD0FB6804
:106A5000BA685A60FB6803F108033A4692E80300FB
:106A600083E8030007F11407BD4680BC704700BFF0
:106A700080B483B000AF78607B68184607F10C07DC
:106A8000BD4680BC704700BF80B582B000AF786063
:106A9000786800F095F80346184607F10807BD46E8
:106AA00080BD00BFB0B586B000AFF860B9607A6055
:106AB000F86800F091F803461D46B86800F08CF8BD
:106AC00003461C46786800F087F8034628462146AE
:106AD0001A4600F08FF803467B6107F1100207F1B8
:106AE000140310461946FFF79DFE3B69184607F14F
:106AF0001807BD46B0BD00BF80B582B000AF78605A
:106B00007B68184600F08AF87B68184607F108078A
:106B1000BD4680BD80B483B000AF78607B68184606
:106B200007F10C07BD4680BC704700BF80B584B03C
:106B300000AFF860B9607A60B86829F097F807F19B
:106B40001007BD4680BD00BF80B483B000AF786041
:106B5000396007F10C07BD4680BC704780B582B034
:106B600000AF78607B68184600F064F87B681846D0
:106B700007F10807BD4680BD80B483B000AF7860E0
:106B80007B68184607F10C07BD4680BC704700BF04
:106B900080B584B000AFF860B9607A60B86829F059
:106BA00065F807F11007BD4680BD00BF80B483B013
:106BB00000AF7860396007F10C07BD4680BC7047B4
:106BC00080B483B000AF78607B68184607F10C078B
:106BD000BD4680BC704700BF80B582B000AF786012
:106BE000786800F033F80346184607F10807BD46F9
:106BF00080BD00BF80B586B000AFF860B9607A6034
:106C00004FF00103FB75F868B9687A6800F02EF858
:106C10000346184607F11807BD4680BD80B483B00F
:106C200000AF78607B68184607F10C07BD4680BC52
:106C3000704700BF80B483B000AF78607B681846AF
:106C400007F10C07BD4680BC704700BF80B582B01D
:106C500000AF786007F104031846FFF709FF034609
:106C60001B68184607F10807BD4680BD80B586B091
:106C700000AFF860B9607A60BA68FB68D31A4FEA6F
:106C8000A3037B617B69002B07D07B694FEA8303F9
:106C90007868F9681A4634F0ADFD7B694FEA8303E2
:106CA0007A68D318184607F11807BD4680BD00BFA3
:106CB00080B582B000AF78607B685B68002B28D01D
:106CC0007B689B68002B05D17B68DB6803F00103C0
:106CD000002B1ED07B68DB6803F00103DBB2002BC6
:106CE0000CD07B685A687B68DB684FEA6303D31873
:106CF0001A687B689B68D3181B6801E07B689B68F7
:106D00007A6851687A68D2684FEA62028A18104637
:106D1000984707F10807BD4680BD00BF80B584B025
:106D200000AFF860B9607A603B60FB68BA681A60CF
:106D3000FB687A685A60FB683A689A60FB68BA69CF
:106D4000DA60FB68FA691A61FB683A6A5A61FB68A3
:106D50005B6818464FF0010115F07CFEFB689B68EC
:106D600018464FF0000115F075FEFB68DB68184609
:106D70004FF0010115F06EFEFB681B6918464FF0DD
:106D8000000115F067FEFB684FF000021A76FB6801
:106D90004FF0000283F82D20FB68184607F110071A
:106DA000BD4680BD0EB480B585B000AF786007F1F8
:106DB0002003FB607B6803F1180318464FF01501B0
:106DC000FA69FB683BF084FF786800F043F807F14C
:106DD0001407BD46BDE8804003B070470EB480B5CF
:106DE00085B000AF786007F12003FB607B6803F19A
:106DF0002D0318464FF00501FA69FB683BF068FF68
:106E0000786800F027F807F11407BD46BDE8804018
:106E100003B0704780B582B000AF7860786849F2FF
:106E20002C11C0F20401FFF7BDFF07F10807BD46B2
:106E300080BD00BF80B582B000AF7860786849F24D
:106E40002C11C0F20401FFF7C9FF07F10807BD4686
:106E500080BD00BF80B586B000AF78607B681A68DF
:106E60007B685B691046194616F066FD7B685B68B7
:106E700018464FF0000115F0EDFD7B6803F1180393
:106E8000184636F035FD0346C3F11403FB60FB687A
:106E90004FEA53037B61FB6803F00103DBB2002B75
:106EA00003D07B6903F101037B617B69FB740AE01A
:106EB0007B681B6818464FF0200116F0BFFDFB7C75
:106EC00003F1FF33FB74FB7C002B0CBF0023012379
:106ED000DBB2002BECD14FF00003BB7415E0BB7CA0
:106EE0007A68D3181B7E002B01D100BF20E07B689D
:106EF0001A68BB7C7968CB181B7E1046194616F0C1
:106F00009DFDBB7C03F10103BB74BA7C7B69C3F1BB
:106F100014039A422CBF00230123DBB2002BDED1E5
:106F200006E07B681B6818464FF0200116F086FDCE
:106F3000BA7C7B69C3F114039A422CBF002301235E
:106F4000DBB2BA7C02F10102BA74002BE9D14FF036
:106F50000003BB7417E0BB7C7A68D31893F82D301C
:106F6000002B01D100BF1EE07B681A68BB7C7968EA
:106F7000CB1893F82D301046194616F05FFDBB7CF8
:106F800003F10103BB74BB7C032B8CBF00230123E3
:106F9000DBB2002BDFD106E07B681B6818464FF0A0
:106FA000200116F04BFDBB7C032B8CBF002301237B
:106FB000DBB2BA7C02F10102BA74002BECD17B681F
:106FC0001B6818464FF0000116F038FD7B681B68FF
:106FD00018464FF0200116F031FD7B681B681846FB
:106FE0004FF0200116F02AFD7B681B6818464FF011
:106FF000200116F023FD7B689B6818464FF00101C5
:1070000015F028FD4FF0010008F020FC7B689B681C
:1070100018464FF0000115F01DFD7B685B681846AF
:107020004FF0010115F016FD07F11807BD4680BDB0
:1070300080B483B000AF78607A6840F2FF139A4260
:1070400005D84FF400727B68B2FBF3F301E04FF018
:107050000103184607F10C07BD4680BC704700BF0E
:1070600080B483B000AF78607B6803F120031846DA
:1070700007F10C07BD4680BC704700BF80B483B0E9
:1070800000AF78607B6803F13503184607F10C0701
:10709000BD4680BC704700BF80B483B000AF78604D
:1070A0007B68DB6B184607F10C07BD4680BC704758
:1070B00080B483B000AF78600B46FB707B68FA78D1
:1070C00083F83A2007F10C07BD4680BC704700BF2B
:1070D00080B483B000AF786039607B683A681A6426
:1070E00007F10C07BD4680BC704700BF80B483B079
:1070F00000AF78607B681B6C184607F10C07BD4633
:1071000080BC704790B58DB000AFF860B9607A6010
:107110003B60FB68184618F0C1FBFB683A689A6749
:10712000FB68BA68DA67FB687A68C3F88020FB6896
:1071300003F18403184600F079FDFB6803F19C031A
:10714000184616F0AFFCFB6803F1C003184600F0C8
:107150009DFDFB684FF00002C3F89020FB684FF0E4
:107160000002C3F8942007F11803184628F07EF9AE
:1071700007F1140207F11803104649F23011C0F26A
:1071800004011A4628F044FC07F1100207F1140329
:10719000104639681A4613F093FE07F1100318469B
:1071A00049F24411C0F2040100F0AAFD03461C4656
:1071B00007F11003184628F0C5F907F11403184623
:1071C00028F0C0F907F11803184628F051F9002CEF
:1071D00005D0FB684FF0000283F8982065E007F1C6
:1071E0002403184628F042F907F1200207F124038E
:1071F000104649F23011C0F204011A4628F008FC8A
:1072000007F11C0207F12003104639681A4613F0F3
:1072100057FE07F11C03184649F24C11C0F2040155
:1072200000F06EFD03461C4607F11C03184628F0CB
:1072300089F907F12003184628F084F907F124039F
:10724000184628F015F9002C05D0FB684FF0010214
:1072500083F8982029E007F12C03184628F006F956
:1072600007F1280207F12C03104649F23011C0F251
:1072700004011A4628F0CCFB07F1280338681946A8
:1072800049F25812C0F2040214F014F807F128036E
:10729000184628F057F907F12C03184628F0E8F8AB
:1072A000FB684FF0020283F89820FB68184607F14C
:1072B0003407BD4690BD07F11003184628F042F987
:1072C000FFE707F11403184628F03CF9FFE707F140
:1072D0001803184628F0CCF81CE007F11C031846E8
:1072E00028F030F9FFE707F12003184628F02AF9C3
:1072F000FFE707F12403184628F0BAF80AE007F17F
:107300002803184628F01EF9FFE707F12C0318465A
:1073100028F0AEF8FB6803F1C003184600F0C4FC87
:10732000FFE7FB6803F19C03184616F095FCFFE7A6
:10733000FB6803F18403184600F086FCFFE7FB6856
:10734000184618F0D3FA28F0EDFC00BFB0B584B0B1
:1073500000AF78607B68184618F04AFB7B6803F141
:107360008403184600F0E0FC0346BB6019E007F117
:107370000803184600F02AFD03461B68184602F071
:10738000B5FD07F10803184600F020FD03461B6811
:107390001A6812681846904707F10803184600F06B
:1073A00003FD7B6803F18403184600F0CFFC03461D
:1073B000FB6007F1080207F10C031046194600F0C4
:1073C000D9FC0346002BD2D17B68D3F89030002B38
:1073D0002FD07B68D3F890301846FFF787FE03461E
:1073E0001846AC4930F028F80346002B21D17B68C1
:1073F00003F19C03184616F049FE03461D467B68C0
:10740000D3F890301846FFF771FE03464FF00102A3
:1074100014462846194630F02DF80346002B02D1B9
:107420004FF000031C46E3B2002B02D04FF00103E3
:1074300001E04FF00003002B3BD07B68D3F8903085
:1074400018464FF00001FFF733FE7B6803F1C003DD
:10745000184600F0C7FC7B6803F1C003184600F033
:10746000E1FC034683F00103DBB2002B13D07B6801
:1074700003F1C003184600F0E9FC03461A687B6874
:10748000C3F890207B68D3F8903018464FF0010184
:10749000FFF70EFE0DE07B684FF00002C3F890206E
:1074A0007B68DB6F184649F26011C0F20401FFF7F8
:1074B00079FC40F63813C1F200031B6803F00103A6
:1074C000002B2AD140F63810C1F2000029F07CFAD6
:1074D0000346002B0CBF00230123DBB2002B1CD082
:1074E0004FF0000440F64010C1F2000016F0DAFA46
:1074F00040F63810C1F2000029F088FA4DF65943E1
:10750000C0F2010340F64010C1F20000194640F2FB
:107510000002C1F2000228F00BFB7B68D3F8903028
:10752000002B21D040F64010C1F2000016F0AEFD55
:1075300003461D467B68D3F890301846FFF7ACFD34
:1075400003464FF001021446284619462FF092FFD9
:107550000346002B02D14FF000031C46E3B2002B80
:1075600002D04FF0010301E04FF00003002B16D0D2
:1075700040F64010C1F2000016F04EFD7B68DC6F53
:107580007B68D3F890301846FFF76AFD0346204623
:1075900049F26411C0F204011A46FFF703FC40F6F9
:1075A0003C13C1F200031B6803F00103002B2AD136
:1075B00040F63C10C1F2000029F006FA0346002B09
:1075C0000CBF00230123DBB2002B1CD04FF00004C2
:1075D00040F66410C1F2000016F064FA40F63C1068
:1075E000C1F2000029F012FA4DF65943C0F201032E
:1075F00040F66410C1F20000194640F20002C1F2E8
:10760000000228F095FA7B68D3F89430002B0BD059
:1076100040F66410C1F2000016F07AFD0346632BB9
:1076200002D94FF0010301E04FF00003002B2BD0F3
:1076300040F66410C1F2000016F0EEFC7B68DC6FCF
:107640007B68D3F894301846FFF718FD03462046B0
:1076500049F26411C0F204011A46FFF7BFFB14E0BF
:10766000002C05D140F63810C1F2000029F0CAF90B
:1076700028F058FB002C05D140F63C10C1F2000068
:1076800029F0C0F928F04EFB00BF07F11007BD46F6
:10769000B0BD00BF0000000080B582B000AF7860D0
:1076A00039603B68002B08D07B6803F184023B46BD
:1076B0001046194600F0E4FB00E000BF07F10807A0
:1076C000BD4680BD90B5A1B000AFF861B9617A61E7
:1076D000BB69002B0ED1FB69DB6F184649F26011C4
:1076E000C0F20401FFF75EFBFB694FF00002C3F834
:1076F00090208DE0BB6918464FF00101FFF7D8FCE0
:10770000FB69D3F89030002B07D0FB69D3F8903099
:1077100018464FF00001FFF7CBFCBA69FB69C3F8CC
:107720009020FB69DC6FFB69D3F890301846FFF7B7
:1077300097FC0346204649F26411C0F204011A4640
:10774000FFF730FB07F12003184600F0C1FB12E001
:10775000FB6903F1C00407F1700207F12003104632
:10776000194600F0F9FB3A4607F17003104621462E
:107770001A4600F049FCFB6903F1C00307F140021F
:107780001046194600F0C0FBFB6903F1C00307F186
:1077900050021046194600F0CBFB07F1300007F10C
:1077A000400107F1500207F1180300F0F1FB07F167
:1077B000200407F130030FCB84E80F00FB6903F1CD
:1077C000C00307F160021046194600F0B1FB07F153
:1077D000200207F160031046194600F003FC03463F
:1077E000002BB5D1FB6903F1C00207F11803104665
:1077F000194600F0AFFCFB69D3F890301846796960
:10780000FFF766FCFB6903F19C03184616F004FCC5
:1078100007F18407BD4690BD90B59BB000AF78617D
:1078200039617B6903F1C003184600F0B9FC0346D7
:10783000002B14BF00230123DBB2002B02D04FF03A
:1078400000037AE03B69002B08D17B6903F1C00398
:10785000184600F0FBFA03461B683B617B6903F1A5
:10786000C00307F128021046194600F04DFB7B6962
:1078700003F1C00307F138021046194600F058FB27
:1078800007F1180007F1280107F1380207F110038A
:1078900000F07EFB7B6903F1C00307F1480210464C
:1078A000194600F045FB07F1180207F1480310469E
:1078B000194600F089FC0346002B02D04FF000036C
:1078C0003BE07B6903F1C00407F1580207F118039C
:1078D0001046194600F040FB3A4607F1580310469F
:1078E00021461A4600F090FB7B69D3F890203B6953
:1078F0009A4221D17B6903F1C003184600F050FC85
:107900000346002B0CBF00230123DBB2002B0DD05C
:107910007B6903F1C003184600F098FA03461B6820
:1079200078691946074AFFF7CDFE05E078694FF000
:107930000001044AFFF7C6FE3B69184607F16C07D1
:10794000BD4690BD0000000080B584B000AF7860F7
:107950007B6803F18403184600F0E6F90346BB6038
:1079600011E007F10803184600F030FA03461B68DF
:107970001A6802F1080212681846904707F10803D6
:10798000184600F011FA7B6803F18403184600F0F2
:10799000DDF90346FB6007F1080207F10C0310460E
:1079A000194600F0E7F90346002BDAD107F110077A
:1079B000BD4680BD90B58BB000AF78607B6803F1A9
:1079C0008403184600F0B0F90346BB6011E007F1EC
:1079D0000803184600F0FAF903461B681A6802F11A
:1079E0000C0212681846904707F10803184600F089
:1079F000DBF97B6803F18403184600F0A7F903461E
:107A0000FB6007F1080207F10C031046194600F06D
:107A1000B1F90346002BDAD17B6893F89830002B3C
:107A200027D17B689C6F07F11403184627F01EFDD1
:107A300007F1100207F11403104649F23011C0F2A9
:107A400004011A4627F0E4FF07F110032046194607
:107A500049F24412C0F2040213F02CFC07F11003A7
:107A6000184627F06FFD07F11403184627F000FDB4
:107A700081E07B6893F89830012B27D17B689C6F5D
:107A800007F11C03184627F0F1FC07F1180207F173
:107A90001C03104649F23011C0F204011A4627F0C7
:107AA000B7FF07F118032046194649F24C12C0F2FD
:107AB000040213F0FFFB07F11803184627F042FDFC
:107AC00007F11C03184627F0D3FC54E07B6893F8B9
:107AD0009830022B4ED17B689C6F07F12403184627
:107AE00027F0C4FC07F1200207F12403104649F2F5
:107AF0003011C0F204011A4627F08AFF07F1200373
:107B00002046194649F25812C0F2040213F0D2FB83
:107B100007F12003184627F015FD07F12403184646
:107B200027F0A6FC27E007F11003184627F00AFD0E
:107B3000FFE707F11403184627F09AFC28F0F2F843
:107B400007F11803184627F0FDFCFFE707F11C03B7
:107B5000184627F08DFC28F0E5F807F120031846B9
:107B600027F0F0FCFFE707F12403184627F080FC1C
:107B700028F0D8F800BF07F12C07BD4690BD00BF24
:107B800080B584B000AF786039607B6803F184030E
:107B9000184600F0C9F80346BB6030E007F108035F
:107BA000184600F013F903461A687B68D3F8903042
:107BB0009A4214BF00230123DBB2002B0DD007F142
:107BC0000803184600F002F903461B6818464FF0F8
:107BD00000013A6802F066F90CE007F10803184664
:107BE00000F0F4F803461B6818464FF001013A68AC
:107BF00002F058F907F10803184600F0D5F87B6841
:107C000003F18403184600F0A1F80346FB6007F176
:107C1000080207F10C031046194600F0ABF80346C2
:107C2000002BBBD107F11007BD4680BD80B582B0E7
:107C300000AF78607B68184600F0E8FA7B68184669
:107C400007F10807BD4680BDB0B582B000AF7860CF
:107C50007B681D687B685C687B68184600F008FBE1
:107C60000346284621461A4600F00EFB7B6818465C
:107C700000F0DAFA7B68184607F10807BD46B0BD88
:107C80007B68184600F0D0FA28F04CF880B582B036
:107C900000AF78607B68184600F012FB7B681846DE
:107CA00007F10807BD4680BD80B58AB000AF786097
:107CB00007F108031846796800F026F907F1180360
:107CC0001846796800F034F97B68184600F03EFBEE
:107CD000034607F1080107F11802786800F042FB3B
:107CE0007B68184600F006FB7B68184607F12807FA
:107CF000BD4680BD7B68184600F0FCFA28F012F8FB
:107D000080B582B000AF786039607868396827F054
:107D1000CFFB0346002B14BF00230123DBB2184620
:107D200007F10807BD4680BD80B584B000AF78601C
:107D30007B6807F10C021046194600F01FFBFB6838
:107D4000184607F11007BD4680BD00BF80B584B05E
:107D500000AF78607B6803F1040307F10C02104662
:107D6000194600F00BFBFB68184607F11007BD46EB
:107D700080BD00BF90B583B000AF7860396078688F
:107D800000F00CFB03461C68386800F007FB034654
:107D90001B689C420CBF00230123DBB2184607F18D
:107DA0000C07BD4690BD00BF80B483B000AF7860C3
:107DB0007B681B6803F104027B681A607B681846C5
:107DC00007F10C07BD4680BC704700BF80B483B08C
:107DD00000AF78607B681B68184607F10C07BD464A
:107DE00080BC704780B582B000AF78607B689A69CC
:107DF0007B68DB699A420ED07B689B69A3F1040221
:107E00007B689A617B681A467B689B6910461946B5
:107E100000F0D0FA02E0786800F0D6FA07F108071F
:107E2000BD4680BD80B582B000AF78607B6803F14D
:107E300018027B6803F108031046194600F0C4F9E4
:107E40000346184607F10807BD4680BD80B586B0D9
:107E500000AF786007F108031846796800F068F809
:107E600007F10803184600F0D7FA07F1080318468F
:107E700000F0F4FA0346184607F11807BD4680BD26
:107E800080B582B000AF786039607B685A687B68E3
:107E90009B689A420FD07B681A467B685B681046E5
:107EA00019463A6800F0E6FA7B685B6803F1040261
:107EB0007B685A6008E07868FFF748FF03467868F7
:107EC00019463A6800F0EEFA07F10807BD4680BD92
:107ED00080B483B000AF78607B684FF000021A6016
:107EE0007B684FF000025A607B684FF000029A6096
:107EF0007B684FF00002DA607B68184607F10C07D8
:107F0000BD4680BC704700BF90B583B000AF04464B
:107F1000796022467B6803F108031046194600F099
:107F20001BF82046204607F10C07BD4690BD00BF58
:107F300090B583B000AF0446796022467B6803F1B8
:107F400018031046194600F007F82046204607F1AE
:107F50000C07BD4690BD00BF80B483B000AF786011
:107F600039603B681A687B681A603B685A687B68AE
:107F70005A603B689A687B689A603B68DA687B68FD
:107F8000DA607B68184607F10C07BD4680BC704775
:107F9000B0B58EB002AF0446F960BA607B6025468A
:107FA00007F110031846F968FFF7D6FF07F1200321
:107FB0001846B968FFF7D0FFF86800F06BFB07F1CF
:107FC000100207F120038DF80010284611461A46CA
:107FD0007B6800F069FB2046204607F13007BD466C
:107FE000B0BD00BF80B582B000AF786039607868FE
:107FF000396800F0E9F8034683F00103DBB2184664
:1080000007F10807BD4680BDB0B5B4B000AF044667
:1080100079613A6107F11C0318463969FFF79CFF43
:1080200007F11C03184600F013FC07F12C03184657
:108030007969FFF769FF07F12C033869194600F0E9
:1080400029FC0346C7F8CC30D7F8CC50786900F04B
:10805000A7F803464FEA53039D422CBF0023012398
:10806000DBB2002B2FD007F13C0318467969FFF7EC
:108070004BFF07F13C0338691946FFF7B3FF03468E
:10808000002B1CD007F14C0318467969FFF73CFF21
:1080900007F15C0318463969FFF75EFF07F16C02D0
:1080A00007F11C0310461946FFF756FF384607F143
:1080B0004C0107F15C0207F16C0300F017FC7869D2
:1080C00000F046FC30E007F17C0318467969FFF7C1
:1080D0002FFF07F11C0207F17C0310461946FFF73A
:1080E00081FF0346002B1CD007F18C0207F11C0313
:1080F00010461946FFF730FF07F19C0318467969CF
:10810000FFF716FF07F1AC0318463969FFF724FFA4
:10811000384607F18C0107F19C0207F1AC0300F02F
:1081200039FC7869FFF75EFE254607F1BC03184667
:108130007969FFF7E9FE07F1BC0328461946D7F82D
:10814000CC2000F059FC2046204607F1D007BD4660
:10815000B0BD00BF80B582B000AF786039607B6889
:108160009A697B681B6AA3F104039A420FD07B686B
:108170001A467B689B69104619463A6800F07AF9FE
:108180007B689B6903F104027B689A6103E078686D
:10819000396800F04FFC07F10807BD4680BD00BFFD
:1081A00080B582B000AF78607B6803F118027B680D
:1081B00003F108031046194600F06CFB034618460D
:1081C00007F10807BD4680BD80B483B000AF78607A
:1081D00039607B681A683B681B689A4214BF0023A9
:1081E0000123DBB2184607F10C07BD4680BC70477F
:1081F00080B582B000AF78607B68184600F078FCEC
:108200007B68184607F10807BD4680BD80B582B07F
:1082100000AF78607B68184600F050FC7B68184619
:1082200007F10807BD4680BD80B582B000AF786019
:108230007B681A687B689B6819467B681B68CB1A49
:108240004FEAA303786811461A4600F05FFC7B688A
:108250001846FFF7CDFF7B68184607F10807BD46B3
:1082600080BD7B681846FFF7C3FF27F05BFD00BFAA
:1082700080B483B000AF78607B68184607F10C07C4
:10828000BD4680BC704700BF80B584B000AFF860C9
:10829000B9607A60F868B96800F04CFC07F1100723
:1082A000BD4680BD80B582B000AF78607B6818465F
:1082B00000F01EFC7B68184607F10807BD4680BD2C
:1082C00080B582B000AF78607B68184600F040FC53
:1082D00078684FF0000100F05DFC7B68184607F1FC
:1082E0000807BD4680BD7B681846FFF7DBFF27F017
:1082F00019FD00BF80B582B000AF78607B681B6855
:10830000002B13D07B685A697B685B6A03F1040316
:10831000786811461A4600F0C7FC7B681A687B68CB
:108320005B68786811461A4600F0DEFC7B681846E8
:10833000FFF7B8FF7B68184607F10807BD4680BD08
:108340007B681846FFF7AEFF27F0ECFC80B483B0E3
:1083500000AF78607B68184607F10C07BD4680BC0B
:10836000704700BF80B48DB000AFF860B9607A602C
:108370003B6007F13407BD4680BC704780B483B0D2
:1083800000AF786039603B681A687B681A607B6868
:10839000184607F10C07BD4680BC704780B483B017
:1083A00000AF78607B68184607F10C07BD4680BCBB
:1083B000704700BF80B483B000AF7860396007F1C8
:1083C0000C07BD4680BC704780B582B000AF7860B6
:1083D0007A687B68DB691046194600F0A1FC7B686F
:1083E00003F118027B685B6AA3F104031046194687
:1083F00000F0ACFC7B681B6AA3F104027B689A6105
:108400007B681A467B689B6910461946FFF7D2FFC6
:1084100007F10807BD4680BD80B582B000AF786027
:108420007B681A687B685B689A420BD17B68DB6863
:10843000A3F104037868194600F088FC7B689A6809
:108440007B681A607B681B68A3F104027B681A6072
:108450007B68184607F10807BD4680BD80B483B02D
:1084600000AF78607B681B68184607F10C07BD46B3
:1084700080BC704780B584B000AFF860B9607A60A6
:10848000BB684FF004001946FBF7F2FB03461A469F
:10849000002A02D07A6812681A6007F11007BD46F8
:1084A00080BD00BFB0B58AB000AFF860B9607A6037
:1084B000FB685A68FB689B689A4232D0FB68194691
:1084C000FB685A68FB685B68A3F104030846114621
:1084D0001A46FFF7CFFFFB685B6803F10402FB68F5
:1084E0005A607B681B683B6207F108031846FFF778
:1084F00055FF03461968FB685B68A3F10802FB6837
:108500005B68A3F10403084611461A4600F038FCE4
:1085100007F108031846FFF759FC03463A6A1A6048
:10852000B4E0F8684FF0010149F26812C0F20402A9
:1085300000F040FC0346FB61F868FFF7F5FB0346DB
:108540003B6107F1080207F110031046194600F0DD
:108550007BFC0346BB61FB681846F96900F08CFCA4
:1085600003467B617B697B62FB681A46BB694FEA05
:1085700083037969CB18104619467A68FFF77AFFAA
:108580004FF000037B62FB681D6807F10803184683
:10859000FFF704FF03461C68FB681846FFF768FEF8
:1085A0000346284621467A6900F07EFC03467B623A
:1085B0007B6A03F104037B6207F108031846FFF7A7
:1085C000EDFE03461D68FB685C68FB681846FFF714
:1085D0004FFE0346284621467A6A00F065FC0346B2
:1085E0007B62FB681D68FB685C68FB681846FFF7E8
:1085F0003FFE0346284621461A46FFF745FEF96826
:10860000FB681A68FB689B681846FB681B68C31AFE
:108610004FEAA303084611461A4600F077FAFB68B2
:108620007A691A60FB687A6A5A60FB694FEA8303C9
:108630007A69D218FB689A6028E027F075FD27F068
:1086400071FB0346184627F025FD7B6A002B0BD1F2
:10865000FB681A46BB694FEA83037969CB18104659
:108660001946FFF7A7FE09E0FB681846FFF700FE72
:1086700003467869796A1A46FFF706FEFB681846D2
:108680007969FA6900F042FA28F036F907F128070B
:10869000BD46B0BD80B483B000AF7860184607F126
:1086A0000C07BD4680BC704790B587B000AF04464C
:1086B000F960BA607B60B868F96800F0EBF80346CF
:1086C0004FEAA3037B615FE0F868FFF7C7FE03464C
:1086D0001A687B681B689A4214BF00230123DBB22F
:1086E000002B05D023461846F968FFF735FCA9E0B2
:1086F000F86800F0ADF8F868FFF7B0FE03461A68B6
:108700007B681B689A4214BF00230123DBB2002B55
:1087100005D023461846F968FFF71EFC92E0F8687A
:1087200000F096F8F868FFF799FE03461A687B6830
:108730001B689A4214BF00230123DBB2002B05D033
:1087400023461846F968FFF707FC7BE0F86800F05D
:108750007FF8F868FFF782FE03461A687B681B689B
:108760009A4214BF00230123DBB2002B05D023461D
:108770001846F968FFF7F0FB64E0F86800F068F865
:108780007B6903F1FF337B617B69002BD4BF00233E
:108790000123DBB2002B97D1B868F96800F07AF8B2
:1087A0000346022B1BD0032B02D0012B2ED044E01A
:1087B000F868FFF753FE03461A687B681B689A4205
:1087C00014BF00230123DBB2002B05D0234618463B
:1087D000F968FFF7C1FB35E0F86800F039F8F86890
:1087E000FFF73CFE03461A687B681B689A4214BF79
:1087F00000230123DBB2002B05D023461846F9687D
:10880000FFF7AAFB1EE0F86800F022F8F868FFF70F
:1088100025FE03461A687B681B689A4214BF002332
:108820000123DBB2002B05D023461846F968FFF779
:1088300093FB07E0F86800F00BF823461846B96888
:10884000FFF78AFB2046204607F11C07BD4690BD76
:1088500080B582B000AF78607B681B6803F10402CA
:108860007B681A607B681A687B689B689A420BD1A8
:108870007B68DB6803F104037868194600F066FA48
:108880007B685A687B681A607B68184607F108079E
:10889000BD4680BD80B582B000AF7860396000F021
:1088A00017FB03467A68D26811463A68D2688A1A7A
:1088B0004FEAA20202F1FF3202FB03F27B681B685F
:1088C00019467B685B68CB1A4FEAA303D2183B6852
:1088D0009B6819463B681B68CB1A4FEAA303D31861
:1088E000184607F10807BD4680BD00BFF0B597B038
:1088F00006AF0446F960BA607B60264607F11003B4
:108900001846F96800F0EEFA07F120031846B96836
:1089100000F0E8FA07F1300318467968FFF71CFB0E
:1089200001AD07F120030FCB85E80F0007F13003FD
:108930000593FB69009307F110030ECB304600F05E
:10894000EDFA2046204607F14407BD46F0BD00BFC2
:1089500080B582B000AF78607B689A687B681B69DD
:10896000A3F104039A420ED07B681A467B689B6889
:1089700010461946FFF71EFD7B689B6803F1040251
:108980007B689A6002E0786800F054FB07F1080702
:10899000BD4680BDF0B597B006AF0446F960BA6039
:1089A0007B60264607F110031846F96800F09AFA32
:1089B00007F120031846B96800F094FA07F1300374
:1089C00018467968FFF7C8FA01AD07F120030FCB0D
:1089D00085E80F0007F130030593FB69009307F169
:1089E00010030ECB304600F04BFB2046204607F12B
:1089F0004407BD46F0BD00BFB0B586B000AF044629
:108A000079603A6007F1080318467968FFF7A4FA1D
:108A1000254607F108031846396800F097FB03461E
:108A200028461946FFF798FA2046204607F118070E
:108A3000BD46B0BD90B583B000AF7860396078684E
:108A40004FF0010100F0E2FB7B685B6A03F1040474
:108A50007B68184600F0FAFB034623607B681A46E1
:108A60007B689B69104619463A68FFF703FD7B68EF
:108A700003F118027B685B6A03F104031046194690
:108A800000F064F97B68DA697B689A6107F10C078A
:108A9000BD4690BD27F048FB27F044F90346184631
:108AA00027F0F8FA7A687B685B6A03F104031B68B5
:108AB0001046194600F034F927F01EFF80B582B049
:108AC00000AF78607B68184600F0D8FB7B684FF0F9
:108AD00000021A607B684FF000025A607B684FF01A
:108AE00000029A607B68184607F10807BD4680BD02
:108AF00080B582B000AF78607B68184600F0CCFB90
:108B00007B68184607F10807BD4680BD80B584B074
:108B100000AFF860B9607A60BB68002B05D0FB68D5
:108B20001846B9687A6800F0C3FB07F11007BD4624
:108B300080BD00BF80B582B000AF786039607868D2
:108B4000396800F0C3FB07F10807BD4680BD00BFD0
:108B500080B582B000AF78607B68184600F08EFB6D
:108B60007B684FF000021A607B684FF000025A6089
:108B70007B6803F108031846FFF7AAF97B6803F145
:108B800018031846FFF7A4F97B68184607F1080791
:108B9000BD4680BD90B589B000AF786039604FF0B8
:108BA0000400FEF745FA03463A68B2FBF3F303F11B
:108BB0000103FB614FF00803FB60FB6903F1020353
:108BC0003B6107F10C0207F1100310461946FBF751
:108BD000C7FE03461A687B685A607B685B687868E2
:108BE000194600F07DFB03461A467B681A607B68D5
:108BF0001A687B685968FB69CB1A4FEA53034FEA3E
:108C00008303D318BB61FB694FEA8303BA69D318A6
:108C10007B617868B9697A6900F08AFB7B6803F147
:108C200008031846B96900F091F87B6803F118024F
:108C30007B69A3F104031046194600F087F87B68AE
:108C4000DA687B689A607B68DC694FF00400FEF7A5
:108C5000EFF902463B68B3FBF2F102FB01F29B1A0B
:108C60004FEA8303E2187B689A6107F12407BD4647
:108C700090BD27F059FA27F055F80346184627F01B
:108C800009FA7B681A687B685B68786811461A463F
:108C900000F02AF87B684FF000021A607B684FF002
:108CA00000025A6027F028FE80B586B000AFF86059
:108CB000B9607A60BB687B6109E07B691B68F86812
:108CC000194600F02DF87B6903F104037B617A6992
:108CD0007B689A422CBF00230123DBB2002BECD12E
:108CE00007F11807BD4680BD80B586B000AFF860BB
:108CF000B9607A6007F114031846F96800F04AFB7E
:108D000007F114031846B9687A6800F065FB07F1AB
:108D10001403184600F052FB07F11807BD4680BD4A
:108D200090B583B000AF786039607B681C464FF027
:108D30000400FEF77DF90346204639681A4600F024
:108D4000B7FA07F10C07BD4690BD00BF90B583B0E0
:108D500000AF786039607B683A68DA603B681A680F
:108D60007B685A607B685C6800F0B2F803464FEAA3
:108D70008303E2187B689A6007F10C07BD4690BD3B
:108D800090B585B000AFF860B9607A60F86800F01F
:108D900031FB03461C46B86800F02CFB0346204616
:108DA00019467A6800F034FB0346184607F11407A9
:108DB000BD4690BD90B587B000AFF860B9607A60ED
:108DC000F86800F055FB03461C46F86800F03EFBCF
:108DD0000346E21ABB689A422CBF00230123DBB290
:108DE000002B02D0786826F009F9F86800F02EFB15
:108DF0000446F86800F02AFB03463B6107F11002C5
:108E000007F1080310461946FBF7AAFD03461B6845
:108E1000E3187B61F86800F019FB02467B699A420F
:108E200007D8F86800F024FB03461A467B699A428B
:108E300004D2F86800F01CFB034600E07B6918468A
:108E400007F11C07BD4690BD90B583B000AF7860B8
:108E500039607868FFF7A2FA03461B681C46386839
:108E6000FFF79CFA03461B68E31A4FEAA303184670
:108E700007F10C07BD4690BD80B582B000AF7860A9
:108E800039603B68002B08D07B68184639684FF082
:108E9000000200F0FFFA034601E04FF0000318461D
:108EA00007F10807BD4680BD80B584B000AFF8600B
:108EB000B9607A603B60F868B9687A683B6800F02E
:108EC00009FB0346184607F11007BD4680BD00BFE9
:108ED00080B500AF4FF00400FEF7AAF8034618462D
:108EE00080BD00BF80B483B000AF786039603B685C
:108EF0001A687B681A603B685A687B685A603B68EE
:108F00009A687B689A603B68DA687B68DA607B689D
:108F1000184607F10C07BD4680BC704784B090B579
:108F200087B000AF044607F12C0080E80E0007F17F
:108F30003C0207F12C031046194600F0F1FA0346F3
:108F4000BB6060E0FB6B1A463B6CD31A4FEAA3038D
:108F50007B60FB6B7B61FB6C1B681A46FB6C5B6880
:108F6000D31A4FEAA3033B60FB6C1B683B617B6831
:108F7000002B0CD1FFF7ACFF03467B60BB6CA3F169
:108F800004031A687B684FEA8303D3187B613B684C
:108F9000002B0DD1FFF79CFF03463B60FB6CDB68A9
:108FA000A3F104031A683B684FEA8303D3183B61BB
:108FB00007F104023B461046194600F0DDFA03466D
:108FC00007F108021046194600F0D6FA03461B685E
:108FD000FB60FB684FEA8303C3F100037A69D3188F
:108FE000184679693A69FFF7CBFE07F13C0318464A
:108FF000F96800F0D5FAF86CF96800F0E3FABA689D
:10900000FB68D31ABB60BB68002BD4BF00230123CD
:10901000DBB2002B96D123461846F96CFEF79CFF75
:109020002046204607F11C07BD46BDE8904004B02D
:10903000704700BF80B582B000AF78607B681A4689
:109040007B689B6810461946FFF7B4F97A687B681D
:10905000DB6810461946FFF763FE7B6803F10802E0
:109060007B685B6903F1040310461946FFF76EFE47
:109070007B68DA687B689A6007F10807BD4680BDA7
:1090800084B090B585B000AF044607F1240080E8B5
:109090000E0007F1340207F124031046194600F0D0
:1090A0003FFA03463B603BE0FB6A1A467B6AD31AF1
:1090B0004FEAA3037B607B6C9B681A467B6C1B6842
:1090C000D31A4FEAA303BB6007F1040207F10803B8
:1090D0001046194600F050FA03463A461046194623
:1090E00000F04AFA03461B68FB60796A7A6AFB68FB
:1090F0004FEA8303D2187B6C1B68084611461A4658
:1091000000F072FA07F124031846F96800F086FAB5
:10911000786CF96800F01AF83A68FB68D31A3B607B
:109120003B68002BD4BF00230123DBB2002BBBD153
:1091300023461846796CFEF70FFF2046204607F1BC
:109140001407BD46BDE8904004B0704790B585B0A7
:1091500000AF786039607B681B681A467B685B6883
:10916000D31A4FEAA3031A463B68D318FB60FB6887
:10917000002B09DBFFF7ACFE03461A46FB689A4258
:1091800002DD4FF0010301E04FF00003002B08D097
:109190007B681A683B684FEA8303D2187B681A60C1
:1091A0002DE0FB68002B06DDFFF792FE0346FA6810
:1091B00092FBF3F309E0FB686FEA0304FFF788FE14
:1091C0000346B4FBF3F36FEA0303BB607B68DA6822
:1091D000BB684FEA8303D31878681946FFF7B6FDDA
:1091E0007B685C68FFF774FE0346BA6802FB03F312
:1091F000FA68D31A4FEA8303E2187B681A607B6827
:10920000184607F11407BD4690BD00BF80B582B077
:1092100000AF786039603B6803F101027B685968F0
:109220007B685B6A18467B681B68C31A4FEAA30316
:10923000CB1A9A4205D9786839684FF0000200F0DD
:109240004DFA07F10807BD4680BD00BF90B583B059
:1092500000AF78607B681C464FF00400FDF7E8FE25
:109260000346204619464FF0000200F013F903466A
:10927000184607F10C07BD4690BD00BF80B582B00F
:1092800000AF78607B68184600F0DEFA7B6818460D
:1092900007F10807BD4680BD80B483B000AF786099
:1092A0007B68184607F10C07BD4680BC704700BFBD
:1092B00080B584B000AFF860B9607A60B86826F015
:1092C000D5FC07F11007BD4680BD00BF80B483B058
:1092D00000AF7860396007F10C07BD4680BC70476D
:1092E00090B585B000AF7860396007F10C0318467F
:1092F000796800F04FF807F10C03184639684FF011
:10930000000200F0ADFA03461C4607F10C031846B4
:1093100000F054F82346184607F11407BD4690BDE7
:1093200007F10C03184600F049F826F0FBFC00BFDB
:1093300080B586B000AFF860B9607A60BB687B61C9
:109340000AE0F868FFF782FF03461A467B691A6055
:109350007B6903F104037B617A697B689A422CBFC5
:1093600000230123DBB2002BEBD10EE026F0DCFE64
:1093700026F0D8FC0346184626F08CFEF868B9683B
:109380007A69FFF791FC27F0B7FA07F11807BD4695
:1093900080BD00BFB0B582B000AF044679602546FD
:1093A000786800F07DFA03462846194600F084FAF2
:1093B0002046204607F10807BD46B0BD80B582B003
:1093C00000AF78607B68184600F086FA7B68184624
:1093D00007F10807BD4680BD80B584B000AFF860D6
:1093E000B9607A60B86826F041FC07F11007BD4605
:1093F00080BD00BF80B582B000AF7860786800F0B3
:1094000077FA0346184607F10807BD4680BD00BF3E
:10941000B0B584B000AFF860B9607A60F86800F069
:1094200073FA0546B86800F06FFA0446786800F0F1
:109430006BFA0346284621461A4600F073FA0346A3
:10944000184607F11007BD46B0BD00BF80B483B019
:1094500000AF78607B685B681A467B681B68D31A2C
:109460004FEAA303184607F10C07BD4680BC7047BE
:1094700080B582B000AF78607B68184600F066FA6D
:109480000346184600F06EFA0346184607F108072F
:10949000BD4680BD80B584B000AFF860B9607A6029
:1094A000F86800F05FFA0246BB689A422CBF0023BE
:1094B0000123DBB2002B01D025F05CFDBB684FEA35
:1094C0008303184627F0C4FA0346184607F110072D
:1094D000BD4680BD80B584B000AFF860B9607A60E9
:1094E0003B60F868B9687A6800F048FA03461846A5
:1094F00007F11007BD4680BD80B586B000AFF860AB
:10950000B9607A604FF00103FB75F868B9687A6852
:1095100000F046FA0346184607F11807BD4680BD1D
:1095200080B582B000AF7860396000F05BFA034626
:109530007A68D26811463A68D2688A1A4FEAA2025B
:1095400002F1FF3202FB03F27B681B6819467B685D
:109550005B68CB1A4FEAA303D2183B689B68194695
:109560003B681B68CB1A4FEAA303D318184607F1D0
:109570000807BD4680BD00BF80B483B000AF7860EF
:1095800039603B681A687B681B689A4201DA3B685D
:1095900000E07B68184607F10C07BD4680BC7047A9
:1095A00080B582B000AF786039603B68C3F10003DA
:1095B0007868194600F032F80346184607F10807A4
:1095C000BD4680BD80B582B000AF786039603B6831
:1095D000C3F1000378681946FFF7B8FD0346184643
:1095E00007F10807BD4680BD90B585B000AFF860B3
:1095F000B9607A60F868FFF7FDFE03461C46B8685C
:10960000FFF7F8FE0346204619467A6800F0F4F9A1
:109610000346184607F11407BD4690BD90B585B0C6
:1096200000AF786039607B681B681A467B685B68AE
:10963000D31A4FEAA3031A463B68D318FB60FB68B2
:10964000002B09DB00F0CEF903461A46FB689A426C
:1096500002DD4FF0010301E04FF00003002B08D0C2
:109660007B681A683B684FEA8303D2187B681A60EC
:109670002DE0FB68002B06DD00F0B4F90346FA6824
:1096800092FBF3F309E0FB686FEA030400F0AAF928
:109690000346B4FBF3F36FEA0303BB607B68DA684D
:1096A000BB684FEA8303D3187868194600F0C2F903
:1096B0007B685C6800F096F90346BA6802FB03F326
:1096C000FA68D31A4FEA8303E2187B681A607B6852
:1096D000184607F11407BD4690BD00BF90B58BB08A
:1096E00000AFF860B9601346FB71FB685B6A1A460D
:1096F000FB685B69D31A4FEAA30303F101033B62E2
:10970000BB683A6AD318FB61FB685A68FB694FEA89
:1097100043039A4237D9FB681A68FB685968FB69AA
:10972000CB1A4FEA53034FEA8301FB79002B03D096
:10973000BB684FEA830301E04FF00003CB18D31856
:109740007B62FB685A697B6A9A420BD9FB685A694B
:10975000FB685B6A03F10403104619467A6A00F05D
:1097600083F957E0FB685969FB685B6A03F10402FF
:109770003B6A4FEA8303786AC318084611461A46C3
:1097800000F08CF946E0FB685C68FB6803F10402BA
:1097900007F1080310461946FBF7E2F803461B6879
:1097A000E31803F10203BB61FB681846B969FFF7D0
:1097B00097FD03467B61BA69FB69D31A4FEA5303ED
:1097C0004FEA8302FB79002B03D0BB684FEA830387
:1097D00001E04FF00003D3187A69D3187B62FB686D
:1097E0005A69FB685B6A03F10403104619467A6AFA
:1097F00000F03AF9F968FB681A68FB685B6808468C
:1098000011461A46FFF770FAFB687A691A60FB681E
:10981000BA695A60FB6803F108031846796AFFF7D2
:1098200095FAFB6803F118023B6A03F1FF334FEA34
:109830008303796ACB1810461946FFF787FA07F1B8
:109840002C07BD4690BD00BF80B483B000AF7860E8
:109850007B68184607F10C07BD4680BC704700BF07
:1098600080B584B000AFF860B9607A60F86800F045
:109870002FF90246BB689A422CBF00230123DBB2BA
:10988000002B01D025F076FBBB684FEA8303184616
:1098900027F0DEF80346184607F11007BD4680BDE5
:1098A00080B483B000AF78607B68184607F10C077E
:1098B000BD4680BC704700BF80B582B000AF786005
:1098C00039607B68184600F00FF97B68184607F18D
:1098D0000807BD4680BD00BF80B483B000AF78608C
:1098E0007B68184607F10C07BD4680BC704700BF77
:1098F00080B483B000AF78607B68184607F10C072E
:10990000BD4680BC704700BF80B582B000AF7860B4
:109910007868FFF7EDFF0346184607F10807BD46D4
:1099200080BD00BF80B586B000AFF860B9607A60D6
:109930004FF00103FB75F868B9687A6800F0E0F849
:109940000346184607F11807BD4680BD80B483B0B2
:1099500000AF78607B68184607F10C07BD4680BCF5
:10996000704700BF80B483B000AF78606FF04043B1
:10997000184607F10C07BD4680BC704780B584B01F
:1099800000AFF860B9607A60F868B9687A6800F08A
:10999000E1F80346184607F11007BD4680BD00BF39
:1099A00080B586B000AFF860B9607A60BA68FB68CD
:1099B000D31A4FEAA3037B617B69002B07D07B6935
:1099C0004FEA83037868F9681A4631F013FF7B6920
:1099D0004FEA83037A68D318184607F11807BD4683
:1099E00080BD00BF80B500AF4FF00400FDF720FB45
:1099F0000346184680BD00BFB0B584B000AFF86024
:109A0000B9607A60F868FFF77FFF0546B868FFF72E
:109A10007BFF04467868FFF777FF03462846214618
:109A20001A46FFF769FD0346184607F11007BD46C1
:109A3000B0BD00BF90B583B000AF786039607B687F
:109A40003A68DA603B681A687B685A607B685C68D1
:109A5000FFF7C8FF03464FEA8303E2187B689A606A
:109A600007F10C07BD4690BD90B585B000AFF8601A
:109A7000B9607A60F86800F07FF803461C46B86861
:109A800000F07AF80346204619467A6800F082F81A
:109A90000346184607F11407BD4690BD90B585B042
:109AA00000AFF860B9607A60F86800F065F80346C6
:109AB0001C46B86800F060F80346204619467A68EC
:109AC00000F086F80346184607F11407BD4690BD1E
:109AD00080B483B000AF78606FF04043184607F160
:109AE0000C07BD4680BC704780B483B000AF78607F
:109AF0007B68184607F10C07BD4680BC704700BF65
:109B000080B586B000AFF860B9607A60BA68FB686B
:109B1000D31A4FEAA3037B617B69002B0ED07B69CC
:109B20004FEA8303C3F100037A68D2187B694FEAD6
:109B300083031046F9681A4631F05CFE7B694FEAF0
:109B40008303C3F100037A68D318184607F1180796
:109B5000BD4680BD80B584B000AFF860B9607A6062
:109B6000F868B9687A68FFF73FFD0346184607F1C1
:109B70001007BD4680BD00BF80B582B000AF7860E1
:109B8000786800F043F80346184607F10807BD4619
:109B900080BD00BFB0B584B000AFF860B9607A6036
:109BA000F86800F03FF80546B86800F03BF8044656
:109BB000786800F037F80346284621461A4600F038
:109BC0003FF80346184607F11007BD46B0BD00BF79
:109BD000B0B584B000AFF860B9607A60F86800F0A2
:109BE00021F80546B86800F01DF80446786800F0D2
:109BF00019F80346284621461A4600F035F8034670
:109C0000184607F11007BD46B0BD00BF80B483B051
:109C100000AF78607B68184607F10C07BD4680BC32
:109C2000704700BF80B582B000AF78607868FFF7FA
:109C3000EDFF0346184607F10807BD4680BD00BF8B
:109C400080B586B000AFF860B9607A604FF001036C
:109C5000FB75F868B9687A6800F01AF80346184688
:109C600007F11807BD4680BD80B586B000AFF8602B
:109C7000B9607A604FF00103FB75F868B9687A68DB
:109C800000F028F80346184607F11807BD4680BDC6
:109C900080B586B000AFF860B9607A60BA68FB68DA
:109CA000D31A4FEAA3037B617B69002B07D07B6942
:109CB0004FEA83037868F9681A4631F09BFD7B69A7
:109CC0004FEA83037A68D318184607F11807BD4690
:109CD00080BD00BF80B586B000AFF860B9607A6023
:109CE000BA68FB68D31A4FEAA3037B617B69002B38
:109CF0000ED07B694FEA8303C3F100037A68D21860
:109D00007B694FEA83031046F9681A4631F072FD09
:109D10007B694FEA8303C3F100037A68D3181846BE
:109D200007F11807BD4680BD80B483B000AF7860EE
:109D300007F10C07BD4680BC704700BF80B483B0FC
:109D400000AF786007F10C07BD4680BC704700BFCC
:109D500080B483B000AF786039607B683A68DA63BA
:109D600007F10C07BD4680BC704700BF80B582B0CC
:109D700000AF786039607B68154A1A607B683A6882
:109D80005A607B6803F10803184600F01FF97B68EE
:109D900003F11403184600F019F978680D49FFF72C
:109DA000D7FF7B684FF0000283F83A207B680A4AAD
:109DB0001A647B68184607F10807BD4680BD7B68BA
:109DC00003F10803184600F00FF925F0ABFF00BFC0
:109DD000A0910400CDCCCC3D0000000080B582B045
:109DE00000AF78607B680E4A1A607B6803F1140349
:109DF000184600F0F9F87B6803F10803184600F0F4
:109E0000F3F87B68184607F10807BD4680BD7B68FC
:109E100003F10803184600F0E7F825F083FF00BFC0
:109E2000A091040080B485B000AFF8600B467A6062
:109E3000FB7207F11407BD4680BC70470EB480B5B5
:109E400085B000AF786007F12003FB607B6803F109
:109E5000200318464FF01501FA69FB6838F038FF07
:109E600007F11407BD46BDE8804003B0704700BF4E
:109E70000EB480B585B000AF786007F12003FB60B9
:109E80007B6803F1350318464FF00501FA69FB685A
:109E900038F01EFF07F11407BD46BDE8804003B04F
:109EA000704700BF80B584B000AFF8600B467A60A1
:109EB000FB72FB7A002B09D1FB6803F1080207F162
:109EC00004031046194600F0B1F80BE0FB7A012BB1
:109ED00008D1FB6803F1140207F104031046194688
:109EE00000F0A4F807F11007BD4680BD90B587B01B
:109EF00000AF78607B6803F10803184600F0BEF8F5
:109F00000346FB6017E07B681B6803F104031C68D1
:109F100007F10C03184600F03BF903461B6878680C
:109F20004FF000011A46A0477B6803F1080318466A
:109F3000F96800F0E3F87B6803F10803184600F0C5
:109F4000AFF803463B6107F10C0207F1100310461E
:109F5000194600F0B9F80346002BD4D17B6803F111
:109F60001403184600F08AF80346BB6017E07B68CC
:109F70001B6803F104031C6807F10803184600F08E
:109F800007F903461B6878684FF001011A46A0479D
:109F90007B6803F114031846B96800F0AFF87B68DA
:109FA00003F11403184600F07BF803467B6107F1C8
:109FB000080207F114031046194600F085F803461D
:109FC000002BD4D107F11C07BD4690BD80B582B0EF
:109FD00000AF78607B68184600F002F97B6818468D
:109FE00007F10807BD4680BDB0B582B000AF78600C
:109FF0007B681D687B685C687B68184600F022F906
:10A000000346284621461A4600F028F97B68184680
:10A0100000F0F4F87B68184607F10807BD46B0BDAC
:10A020007B68184600F0EAF825F07CFE80B582B027
:10A0300000AF786039607B685A687B689B689A4299
:10A040000FD07B681A467B685B68104619463A68F1
:10A0500000F012F97B685B6803F104027B685A60C8
:10A0600008E0786800F01CF80346786819463A68FA
:10A0700000F01AF907F10807BD4680BD80B584B02D
:10A0800000AF78607B6807F10C021046194600F0BB
:10A0900003FAFB68184607F11007BD4680BD00BFF4
:10A0A00080B584B000AF78607B6803F1040307F1EA
:10A0B0000C021046194600F0EFF9FB68184607F14C
:10A0C0001007BD4680BD00BF90B583B000AF78607B
:10A0D0003960786800F0F0F903461C68386800F0D1
:10A0E000EBF903461B689C420CBF00230123DBB243
:10A0F000184607F10C07BD4690BD00BF90B587B06C
:10A1000000AF786039604FF00103FB603A4607F119
:10A110000C031046194600F0DBF90346BB60786873
:10A12000FFF7BEFF03463B6107F1080207F110038A
:10A1300010461946FFF7C8FF0346002B13D04FF017
:10A1400001037B613A4607F114031046194600F0FB
:10A15000BFF904467868FFF7A3FF03462046194677
:10A160003A6800F0D1F97B685B68A3F104027B6870
:10A170005A607B681A467B685B681046194600F097
:10A18000DDF93B68184607F11C07BD4690BD00BFCE
:10A1900080B483B000AF78607B681B68184607F115
:10A1A0000C07BD4680BC704780B582B000AF7860B8
:10A1B000786800F0CDF90346184607F10807BD4658
:10A1C00080BD00BF80B582B000AF78607B68184664
:10A1D00000F0E4F97B68184607F10807BD4680BD2A
:10A1E00080B582B000AF78607B68184600F0BCF99B
:10A1F0007B68184607F10807BD4680BD80B582B070
:10A2000000AF78607B681A687B689B6819467B683A
:10A210001B68CB1A4FEAA303786811461A4600F070
:10A22000CBF97B681846FFF7CDFF7B68184607F12E
:10A230000807BD4680BD7B681846FFF7C3FF25F0C1
:10A2400071FD00BF80B483B000AF78607B681846B2
:10A2500007F10C07BD4680BC704700BF80B584B0D5
:10A2600000AFF860B9607A60F868B96800F0B8F9D2
:10A2700007F11007BD4680BD80B584B000AFF8601F
:10A28000B9607A60BB684FF004001946F9F7F0FC3A
:10A2900003461A46002A02D07A6812681A6007F14B
:10A2A0001007BD4680BD00BFB0B58AB000AFF860F2
:10A2B000B9607A60FB685A68FB689B689A4232D042
:10A2C000FB681946FB685A68FB685B68A3F10403E6
:10A2D000084611461A46FFF7CFFFFB685B6803F19B
:10A2E0000402FB685A607B681B683B6207F1080345
:10A2F000184600F0E1F803461968FB685B68A3F1B3
:10A300000802FB685B68A3F10403084611461A467D
:10A3100000F074F907F108031846FFF739FF034608
:10A320003A6A1A60B4E0F8684FF0010149F280120D
:10A33000C0F2040200F07CF90346FB61F868FFF705
:10A340009DFE03463B6107F1080207F1100310462A
:10A35000194600F0B7F90346BB61FB681846F96976
:10A3600000F0C8F903467B617B697B62FB681A4693
:10A37000BB694FEA83037969CB18104619467A689E
:10A38000FFF77AFF4FF000037B62FB681D6807F15F
:10A390000803184600F090F803461C68FB6818464E
:10A3A000FFF750FF0346284621467A6900F0BAF9C4
:10A3B00003467B627B6A03F104037B6207F10803B7
:10A3C000184600F079F803461D68FB685C68FB6876
:10A3D0001846FFF737FF0346284621467A6A00F001
:10A3E000A1F903467B62FB681D68FB685C68FB683B
:10A3F0001846FFF727FF0346284621461A46FFF76F
:10A400002DFFF968FB681A68FB689B681846FB68B3
:10A410001B68C31A4FEAA303084611461A4600F008
:10A42000CBF8FB687A691A60FB687A6A5A60FB6944
:10A430004FEA83037A69D218FB689A6028E025F016
:10A4400073FE25F06FFC0346184625F023FE7B6A59
:10A45000002B0BD1FB681A46BB694FEA830379696D
:10A46000CB181046194600F069F809E0FB68184659
:10A47000FFF7E8FE03467869796A1A46FFF7EEFEB1
:10A48000FB6818467969FA6900F096F826F034FA04
:10A4900007F12807BD46B0BD80B483B000AF786037
:10A4A00039603B681A687B681A607B68184607F158
:10A4B0000C07BD4680BC704780B483B000AF7860A5
:10A4C0007B68184607F10C07BD4680BC704700BF8B
:10A4D00080B584B000AF786039607B681A683B68EB
:10A4E0001B684FEA8303D318FB6007F1080207F1EA
:10A4F0000C0310461946FFF7CFFFBB68184607F15B
:10A500001007BD4680BD00BF90B585B000AFF860B4
:10A51000B9607A60F86800F019F90446B86800F08C
:10A5200015F90346204619467A6800F01DF90346DE
:10A53000184607F11407BD4690BD00BF80B483B034
:10A5400000AF7860396007F10C07BD4680BC7047EA
:10A5500080B483B000AF78607B68184607F10C07C1
:10A56000BD4680BC704700BF80B582B000AF786048
:10A570007B68184600F022F97B684FF000021A60F1
:10A580007B684FF000025A607B684FF000029A60CF
:10A590007B68184607F10807BD4680BD80B582B0CC
:10A5A00000AF78607B68184600F016F97B681846A3
:10A5B00007F10807BD4680BD80B584B000AFF860E4
:10A5C000B9607A60BB68002B05D0FB681846B96893
:10A5D0007A6800F00DF907F11007BD4680BD00BF95
:10A5E00080B582B000AF786039607868396800F073
:10A5F0000DF907F10807BD4680BD00BF90B585B0D5
:10A6000000AFF860B9607A60F86800F009F90446B4
:10A61000B86800F005F90346204619467A6800F04C
:10A620000DF90346184607F11407BD4690BD00BF5B
:10A6300090B587B000AFF860B9607A60F86800F054
:10A640002FF903461C46F86800F018F90346E21A91
:10A65000BB689A422CBF00230123DBB2002B02D03F
:10A66000786824F0CBFCF86800F008F90446F86834
:10A6700000F004F903463B6107F1100207F10803FB
:10A6800010461946FAF76CF903461B68E3187B611C
:10A69000F86800F0F3F802467B699A4207D8F86838
:10A6A00000F0FEF803461A467B699A4204D2F86825
:10A6B00000F0F6F8034600E07B69184607F11C0736
:10A6C000BD4690BD90B583B000AF786039607868C2
:10A6D000FFF7F2FE03461B681C463868FFF7ECFEE6
:10A6E00003461B68E31A4FEAA303184607F10C0759
:10A6F000BD4690BD80B582B000AF786039603B68E0
:10A70000002B08D07B68184639684FF0000200F033
:10A71000D9F8034601E04FF00003184607F1080797
:10A72000BD4680BD80B584B000AFF860B9607A6086
:10A730003B60F868B9687A683B6800F0E3F8034664
:10A74000184607F11007BD4680BD00BF80B582B036
:10A7500000AF7860786800F0E7F80346184607F124
:10A760000807BD4680BD00BFB0B586B000AFF86039
:10A77000B9607A60F86800F0E3F803461D46B868EF
:10A7800000F0DEF803461C46786800F0D9F803466E
:10A79000284621461A4600F0E1F803467B6107F19E
:10A7A000100207F1140310461946FFF775FE3B69C6
:10A7B000184607F11807BD46B0BD00BF80B582B08E
:10A7C00000AF78607B68184600F0DCF87B681846BC
:10A7D00007F10807BD4680BD80B483B000AF786044
:10A7E0007B68184607F10C07BD4680BC704700BF68
:10A7F00080B584B000AFF860B9607A60B86825F0C1
:10A8000035FA07F11007BD4680BD00BF80B483B0A4
:10A8100000AF7860396007F10C07BD4680BC704717
:10A8200080B582B000AF78607868FFF791FE03468C
:10A83000184607F10807BD4680BD00BFB0B584B01B
:10A8400000AFF860B9607A60F868FFF7ADFC0346C6
:10A850001D46B868FFF7A8FC03461C467868FFF75A
:10A86000A3FC0346284621461A4600F097F8034603
:10A87000184607F11007BD46B0BD00BF80B483B0D5
:10A8800000AF78607B685B681A467B681B68D31AE8
:10A890004FEAA303184607F10C07BD4680BC70477A
:10A8A00080B582B000AF78607B68184600F08AF807
:10A8B0000346184600F092F80346184607F10807C9
:10A8C000BD4680BD80B584B000AFF860B9607A60E5
:10A8D000F86800F083F80246BB689A422CBF002358
:10A8E0000123DBB2002B01D024F044FBBB684FEA0C
:10A8F0008303184626F0ACF80346184607F1100704
:10A90000BD4680BD80B584B000AFF860B9607A60A4
:10A910003B60F868B9687A6800F06CF8034618463E
:10A9200007F11007BD4680BD80B483B000AF7860EA
:10A930007B68184607F10C07BD4680BC704700BF16
:10A9400080B582B000AF7860786800F065F80346A3
:10A95000184607F10807BD4680BD00BF80B586B028
:10A9600000AFF860B9607A604FF00103FB75F868DA
:10A97000B9687A6800F060F80346184607F11807CE
:10A98000BD4680BD80B483B000AF78607B68184658
:10A9900007F10C07BD4680BC704700BF80B586B08C
:10A9A00000AFF860B9607A604FF00103FB75F8689A
:10A9B000B9687A6800F062F80346184607F118078C
:10A9C000BD4680BD80B483B000AF78607B68184618
:10A9D00007F10C07BD4680BC704700BF80B483B050
:10A9E00000AF78606FF04043184607F10C07BD4692
:10A9F00080BC704780B584B000AFF860B9607A6001
:10AA0000F868B9687A6800F063F80346184607F1F9
:10AA10001007BD4680BD00BF80B582B000AF786032
:10AA200007F104031846FFF747FD03461B68184665
:10AA300007F10807BD4680BD80B586B000AFF8605D
:10AA4000B9607A60BA68FB68D31A4FEAA3037B61E6
:10AA50007B69002B07D07B694FEA83037868F9682C
:10AA60001A4630F0C7FE7B694FEA83037A68D31831
:10AA7000184607F11807BD4680BD00BF80B586B0F7
:10AA800000AFF860B9607A60BA68FB68D31A4FEA21
:10AA9000A3037B617B69002B0ED07B694FEA8303A4
:10AAA000C3F100037A68D2187B694FEA830310462A
:10AAB000F9681A4630F09EFE7B694FEA8303C3F1C2
:10AAC00000037A68D318184607F11807BD4680BD01
:10AAD00080B584B000AFF860B9607A60F868B96892
:10AAE0007A6800F007F80346184607F11007BD46DC
:10AAF00080BD00BF90B585B000AFF860B9607A60E6
:10AB0000F868FFF78DFE0446B868FFF789FE034634
:10AB1000204619467A6800F007F80346184607F100
:10AB20001407BD4690BD00BFB0B584B000AFF8605B
:10AB3000B9607A60F868FFF737FB03461D46B868CE
:10AB4000FFF732FB03461C467868FFF72DFB0346F0
:10AB5000284621461A46FFF701FF0346184607F12B
:10AB60001007BD46B0BD00BF90B585B000AFF8601E
:10AB70000B467A60FB7297F90B20FB6853F8223082
:10AB8000002B0FD14FF0180025F062FF03461C4642
:10AB900023461846F9F778F897F90B202146FB6809
:10ABA00043F8221097F90B20FB6853F8223018461F
:10ABB000796803F007FB07F11407BD4690BD2046F6
:10ABC00025F054F825F0AEF880B582B000AF78607B
:10ABD0007B681846796812F0C1F87B68184607F15F
:10ABE0000807BD4680BD00BF80B582B000AF786069
:10ABF0007B6803F10403184614F0CCFB03461846A7
:10AC000007F10807BD4680BD90B583B000AF04468C
:10AC1000796022467B681046194624F073FE204670
:10AC2000204607F10C07BD4690BD00BF80B483B03D
:10AC300000AF786039607B683A68DA60184607F1DF
:10AC40000C07BD4680BC7047B0B58AB002AF7860D3
:10AC50007B68D3F8A4517B68D3F8004107F1100357
:10AC6000184624F003FC07F10C0207F1100310460C
:10AC700049F2F411C0F204011A4624F0C9FE07F1AA
:10AC8000080207F10C03104621461A4610F018F985
:10AC900007F10803184624F0F9FB034618462DF087
:10ACA000EFFE02460B46104619462CF0D3F8034639
:10ACB0004FF001021446284619462CF0BDFB03460E
:10ACC000002B02D04FF000031C46E4B207F108034A
:10ACD000184624F037FC07F10C03184624F032FC28
:10ACE00007F11003184624F0C3FB002C64D04FF08A
:10ACF000080025F0DDFE0346FB617B68D3F8A43134
:10AD000018462BF099FD02460B46CDE90023F86961
:10AD10004FF0080149F21022C0F2040231F0A4FF02
:10AD20007B68D3F8004107F11803184624F09EFB16
:10AD300007F1140207F11803104649F2F411C0F2AA
:10AD400004011A4624F064FE07F114032046194654
:10AD5000FA6910F0AFFA07F11403184624F0F2FB79
:10AD600007F11803184624F083FBFB69002B25D05C
:10AD7000F86924F07FFF22E007F10803184624F069
:10AD8000E1FBFFE707F10C03184624F0DBFBFFE7CC
:10AD900007F11003184624F06BFB24F0C3FF07F102
:10ADA0001403184624F0CEFBFFE707F118031846FA
:10ADB00024F05EFB24F0B6FF00BF00E000BF07F107
:10ADC0002007BD46B0BD00BFB0B5F0B008AF07F179
:10ADD0000403186007F104031B681846FFF7F4FE2C
:10ADE0004FF48043C4F2020303F148031A6807F1E9
:10ADF00004031B68C3F83C214FF48043C4F20203F0
:10AE000003F144031A4607F104031B68C3F89021B9
:10AE10004FF48043C4F2020303F14C0207F1040330
:10AE20001B68C3F8982107F104031B6803F5D0736E
:10AE3000184618F0FDF807F104031B6803F5D073FA
:10AE40001846DFF8341B18F033F94FF000004FF0CC
:10AE5000FF314FF0000220F07DFB4FF000004FF07B
:10AE6000FF314FF0010220F075FB4FF002004FF070
:10AE7000FF314FF0000220F06DFB4FF002004FF069
:10AE8000FF314FF0010220F065FB4FF46D43CEF22D
:10AE900000034FF46D42CEF20002526A42F4E02207
:10AEA0005A624FF00C0025F0D3FD03461C462346A2
:10AEB0004FF00102009218464FF002014FF00002DD
:10AEC0004FF0010311F0BEFC224640F69C13C1F284
:10AED00000031A604FF00C0025F0BAFD03461C4633
:10AEE00023464FF00102009218464FF002014FF046
:10AEF00001024FF0010311F0A5FC224640F6A01319
:10AF0000C1F200031A6040F68C13C1F2000307F18E
:10AF1000040212681A604FF0780025F099FD03468C
:10AF20001C462346184614F0B9FC224607F10403D8
:10AF30001B68C3F8AC2062B640F22003C1F20003E4
:10AF40001A6844F6D353C1F26203A3FB02134FEA1B
:10AF5000931303F1FF33C7F83431D7F834216FF07E
:10AF60007F439A4246D84EF21003CEF20003D7F840
:10AF7000342122F07F4202F1FF325A604FF0FF038A
:10AF800087F833314FF01F03C7F82C3197F933316D
:10AF9000002B12DA4FF46D43CEF2000397F8332101
:10AFA00002F00F02A2F10401D7F82C21D2B24FEA2D
:10AFB000C202D2B25B181A760EE04FF46143CEF2B1
:10AFC000000397F93311D7F82C21D2B24FEAC2020D
:10AFD000D2B25B1883F800234EF21003CEF20003C6
:10AFE0004FF000029A604EF21003CEF200034FF0D1
:10AFF00007021A604FF4A47025F02AFD03461C4690
:10B00000234607F1040212684FF0030100914FF448
:10B01000E1310191029218464FF000014FF0020217
:10B020004FF0000311F00CFA224607F104031B68ED
:10B03000C3F8882107F104031B68D3F8882140F680
:10B040009013C1F200031A6049F21820C0F2040004
:10B0500030F0F6FE40F22003C1F200031A684DF60C
:10B060008363C4F21B33A3FB02134FEA934349F2F9
:10B070002020C0F20400194630F0BAFD04F0B2FC02
:10B0800003461D4604F0A2FC03461C4604F0B4FC33
:10B09000034649F23820C0F204002946224630F027
:10B0A000A7FD4FF00C0025F0D3FC03461C462346B9
:10B0B0004FF00002009218464FF001014FF00E02CF
:10B0C0004FF0010311F0BEFB224607F104031B6899
:10B0D000C3F8AC214FF0100025F0BAFC03461C4623
:10B0E00022464FF0110300934FF0000301934FF0FD
:10B0F0000F03029348F2A063C0F2010303931046CA
:10B100004FF000014FF012024FF0000312F06CFB01
:10B11000224607F104031B68C3F8B0204FF010006B
:10B1200025F096FC03461C4622464FF00803009388
:10B130004FF0000301934FF00703029348F2A0631E
:10B14000C0F20103039310464FF000014FF00902D3
:10B150004FF0000312F048FB224607F104031B687E
:10B16000C3F8B4204FF00C0025F072FC03461C46D7
:10B1700022464FF01C03009348F2A063C0F2010383
:10B18000019310464FF000014FF01B024FF00003F7
:10B1900018F066FA224607F104031B68C3F81C2165
:10B1A0004FF00C0025F054FC03461C4622464FF09D
:10B1B0001403009348F2A063C0F201030193104608
:10B1C0004FF000014FF013024FF0000318F048FA5F
:10B1D000224607F104031B68C3F820214FF0030047
:10B1E00025F036FC03461C46234618464FF0010165
:10B1F0004FF000024FF0010311F0D8FCC7F898415E
:10B200004FF0240025F024FC03461C46214607F19C
:10B2100004031B68D3F81C214FF4D453C0F2060377
:10B220000093084611464FF04002D7F8983117F0C6
:10B230007FFF224607F104031B68C3F824214FF067
:10B24000180025F005FC03461C46224607F10403BE
:10B250001B68D3F824314FF0010100914FF0000139
:10B2600001914FF001010291104619464FF0010281
:10B270004FF0000318F030F923461A4607F1040393
:10B280001B68C3F8C4204FF0180025F0E1FB03460B
:10B290001C46224607F104031B68D3F824314FF003
:10B2A000010100914FF0000101914FF00101029165
:10B2B000104619464FF001024FF0010318F00CF947
:10B2C00023461A4607F104031B68C3F8C8204FF051
:10B2D000180025F0BDFB03461C46224607F1040377
:10B2E0001B68D3F824314FF0010100914FF00001A9
:10B2F00001914FF001010291104619464FF00102F1
:10B300004FF0020318F0E8F823461A4607F1040349
:10B310001B68C3F8CC204FF0180025F099FB0346BA
:10B320001C46224607F104031B68D3F824314FF072
:10B33000010100914FF0000101914FF001010291D4
:10B34000104619464FF000024FF0020318F0C4F8FF
:10B3500023461A4607F104031B68C3F8D0204FF0B8
:10B36000180025F075FB03461C46224607F104032E
:10B370001B68D3F824314FF0010100914FF0000118
:10B3800001914FF001010291104619464FF0010260
:10B390004FF0040318F0A0F823461A4607F10403FF
:10B3A0001B68C3F8D4204FF0180025F051FB03466A
:10B3B0001C46224607F104031B68D3F824314FF0E2
:10B3C000010100914FF0000101914FF00101029144
:10B3D000104619464FF001024FF0030318F07CF8B5
:10B3E00023461A4607F104031B68C3F8D8204FF020
:10B3F000180025F02DFB03461C46224607F10403E6
:10B400001B68D3F824314FF0010100914FF0000187
:10B4100001914FF001010291104619464FF00002D0
:10B420004FF0010318F058F823461A4607F10403B9
:10B430001B68C3F8DC204FF0180025F009FB034619
:10B440001C46224607F104031B68D3F824314FF051
:10B45000010100914FF0000101914FF001010291B3
:10B46000104619464FF000024FF0000318F034F870
:10B4700023461A4607F104031B68C3F8E0204FF087
:10B48000180025F0E5FA03461C46224607F104039E
:10B490001B68D3F824314FF0010100914FF00001F7
:10B4A00001914FF001010291104619464FF001023F
:10B4B0004FF0050318F010F823461A4607F104036D
:10B4C0001B68C3F8E4204FF0180025F0C1FA0346CA
:10B4D0001C46224607F104031B68D3F824314FF0C1
:10B4E000010100914FF0000101914FF00101029123
:10B4F000104619464FF001024FF0060317F0ECFF1B
:10B5000023461A4607F104031B68C3F86C214FF069
:10B510000C0025F09DFA03461C4623464FF001021D
:10B52000009218464FF002014FF003024FF0000363
:10B5300011F088F9224607F104031B68C3F868215B
:10B540004FF0100025F084FA03461C462346DFF82E
:10B550002C24009218464FF001014FF01A02DFF838
:10B56000203411F00DFE224607F104031B68C3F8D6
:10B570008C214FF00C0025F06BFA03461C46234645
:10B580004FF00102009218464FF002014FF00702FF
:10B590004FF0010311F056F9C7F894414FF00C0039
:10B5A00025F056FA03461C4623464FF0010200924E
:10B5B00018464FF002014FF002024FF0000311F065
:10B5C00041F9C7F890414FF00C0025F041FA0346CD
:10B5D0001C4623464FF00102009218464FF002012C
:10B5E0004FF005024FF0010311F02CF9C7F88C4120
:10B5F0004FF00C0025F02CFA03461C4623464FF072
:10B600000102009218464FF002014FF006024FF07F
:10B61000000311F017F9C7F888414FF0340025F006
:10B6200017FA03461C46214607F104031B68D3F8AA
:10B63000B420D7F88C310093D7F88831019344F2C5
:10B640004023C0F20F03029308461146D7F8942115
:10B65000D7F89031FBF762FB224607F104031B6821
:10B66000C3F8642107F104031B68D3F86831184656
:10B670004FF0010111F0EEF907F104031B68D3F854
:10B680006C3118464FF0010111F0E4F94FF00C0055
:10B6900025F0DEF903461C4623464FF001020092D6
:10B6A00018464FF001014FF017024FF0010311F05F
:10B6B000C9F8224607F104031B68C3F8B8204FF00D
:10B6C0000C0025F0C5F903461C4623464FF0010245
:10B6D000009218464FF003014FF019024FF001039A
:10B6E00011F0B0F8224607F104031B68C3F8BC2030
:10B6F0004FF00C0025F0ACF903461C4623464FF0F2
:10B700000102009218464FF003014FF01A024FF069
:10B71000010311F097F8224607F104031B68C3F8F0
:10B72000C02007F104031B68D3F86431184649F2BE
:10B730006021C0F20401FBF735FB4FF00C0025F04F
:10B7400087F903461C4623464FF001020092184633
:10B750004FF001014FF010024FF0000311F072F8AA
:10B76000C7F884414FF0200025F072F903461C46CB
:10B77000224607F104031B68D3F8B430104619467B
:10B78000D7F8842149F28063C0F2980305F0E8FC01
:10B79000224607F104031B68C3F8FC2007F10403E9
:10B7A0001B68D3F8FC30184649F27421C0F204013A
:10B7B00005F000FD4FF01C0025F04AF903461C4639
:10B7C0002346184649F27821C0F204010FF060F9CF
:10B7D000224607F104031B68C3F8002107F10403A4
:10B7E0001B68D3F8003118460FF07AF903464FEA88
:10B7F000D373DBB2002B71D007F104031B68D3F8BD
:10B80000003118464FF000010FF088FA0346C7F8E0
:10B810008031D7F88031002B30DB40F25843C1F241
:10B8200000031B68DC6807F104031B68D3F80031D0
:10B8300007F1600210461946FFF7E6F907F16003C9
:10B84000184623F023FE03461A4649F60803C0F2C1
:10B85000040300930192204649F28821C0F20401BA
:10B8600049F2B422C0F204024FF481732DF0C4FEF9
:10B8700007F16003184623F065FE2FE040F25843BD
:10B88000C1F200031B68DC6807F104031B68D3F8EE
:10B89000003107F1640210461946FFF7B5F907F1C8
:10B8A0006403184623F0F2FD03461A4649F60803DE
:10B8B000C0F2040300930192204649F2C021C0F275
:10B8C000040149F2B422C0F204024FF483732DF054
:10B8D00093FE07F16403184623F034FE07F10403D6
:10B8E0001B68D3F8004107F17003184623F0BEFD32
:10B8F00007F16C0207F17003104649F2F421C0F21F
:10B9000004011A4624F084F807F1680207F16C0379
:10B91000104621461A460FF0D3FA07F1680318467D
:10B9200049F20831C0F20401FCF7EAF903461C466B
:10B9300007F16803184623F005FE07F16C0318466B
:10B9400023F000FE07F17003184623F091FD002C50
:10B9500018D040F25843C1F200031B689B6849F2BB
:10B960000C30C0F2040049F21C31C0F204011A4646
:10B970002EF042FA30E000BF0000204100409C471A
:10B98000A4707D3F07F104031B68D3F8004107F161
:10B990007803184623F06AFD07F1740207F1780373
:10B9A000104649F2F421C0F204011A4624F030F89E
:10B9B00007F174032046194649F22032C0F204020E
:10B9C0000FF078FC07F17403184623F0BBFD07F174
:10B9D0007803184623F04CFD07F104031B68D3F8E5
:10B9E000004107F18403184623F040FD07F180026F
:10B9F00007F18403104649F22431C0F204011A46CB
:10BA000024F006F807F17C0207F180031046214676
:10BA10001A460FF055FA07F17C03184649F23831FF
:10BA2000C0F20401FCF76CF903461C4607F17C03E5
:10BA3000184623F087FD07F18003184623F082FDA6
:10BA400007F18403184623F013FD002C29D007F1D9
:10BA500004031B68D3F8004107F18C03184623F058
:10BA600005FD07F1880207F18C03104649F22431E5
:10BA7000C0F204011A4623F0CBFF07F188032046E9
:10BA8000194649F23C32C0F204020FF013FC07F1F0
:10BA90008803184623F056FD07F18C03184623F05F
:10BAA000E7FC07F104031B68D3F8004107F1980392
:10BAB000184623F0DBFC07F1940207F198031046C7
:10BAC00049F2F411C0F204011A4623F0A1FF07F174
:10BAD000900207F19403104621461A460FF0F0F940
:10BAE00007F19003184649F23831C0F20401FCF71F
:10BAF00007F903461C4607F19003184623F022FD80
:10BB000007F19403184623F01DFD07F1980318462A
:10BB100023F0AEFC002C29D007F104031B68D3F8F6
:10BB2000004107F1A003184623F0A0FC07F19C0296
:10BB300007F1A003104649F2F411C0F204011A46BD
:10BB400023F066FF07F19C032046194649F258325C
:10BB5000C0F204020FF0AEFB07F19C03184623F07D
:10BB6000F1FC07F1A003184623F082FC07F104035F
:10BB70001B68D3F8004107F1A803184623F076FCB0
:10BB800007F1A40207F1A803104649F22431C0F2DC
:10BB900004011A4623F03CFF07F15C0207F1A403FD
:10BBA000104621461A460FF08BF907F1A4031846F8
:10BBB00023F0C8FC07F1A803184623F059FC07F14D
:10BBC0005C03184649F23C31C0F20401FCF798F8D6
:10BBD0000346002B0DD007F104031B68D3F8903106
:10BBE00007F104021268D2F890211278D2B21A70CA
:10BBF00018E107F15C03184649F26031C0F2040114
:10BC0000FCF77EF80346002B08D007F104031B68FD
:10BC1000D3F890314FF00A021A7003E107F15C0388
:10BC2000184649F27031C0F20401FCF769F8034686
:10BC3000002B08D007F104031B68D3F890314FF0B4
:10BC400000021A70EEE007F15C03184649F28031F9
:10BC5000C0F20401FCF754F80346002B08D007F1AA
:10BC600004031B68D3F890314FF001021A70D9E039
:10BC700007F15C03184649F29031C0F20401FCF769
:10BC80003FF80346002B08D007F104031B68D3F8E4
:10BC900090314FF002021A70C4E007F15C031846BD
:10BCA00049F2A031C0F20401FCF72AF80346002B48
:10BCB00008D007F104031B68D3F890314FF003025A
:10BCC0001A70AFE007F15C03184649F2B031C0F2D8
:10BCD0000401FCF715F80346002B08D007F1040314
:10BCE0001B68D3F890314FF00B021A709AE007F1FD
:10BCF0005C03184649F2C031C0F20401FCF700F8B9
:10BD00000346002B08D007F104031B68D3F89031D9
:10BD10004FF00C021A7085E007F15C03184649F2F7
:10BD2000D031C0F20401FBF7EBFF0346002B08D033
:10BD300007F104031B68D3F890314FF00D021A701D
:10BD400070E007F15C03184649F2E031C0F20401EB
:10BD5000FBF7D6FF0346002B08D007F104031B684E
:10BD6000D3F890314FF00E021A705BE007F15C03DC
:10BD7000184649F2F831C0F20401FBF7C1FF03464F
:10BD8000002B08D007F104031B68D3F890314FF063
:10BD900009021A7046E007F15C03184649F20841AF
:10BDA000C0F20401FBF7ACFF0346002B08D007F1FB
:10BDB00004031B68D3F890314FF007021A7031E08A
:10BDC00007F15C03184649F21841C0F20401FBF781
:10BDD00097FF0346002B08D007F104031B68D3F834
:10BDE00090314FF004021A701CE007F15C03184612
:10BDF00049F22841C0F20401FBF782FF0346002B01
:10BE000008D007F104031B68D3F890314FF0080203
:10BE10001A7007E007F104031B68D3F890314FF064
:10BE200009021A7007F104031B684FF0000283F83F
:10BE3000942107F104031B68D3F8004107F1B40310
:10BE4000184623F013FB07F1B00207F1B4031046C4
:10BE500049F2F411C0F204011A4623F0D9FD07F1AA
:10BE6000AC0207F1B003104621461A460FF028F83D
:10BE700007F1AC03184623F009FB034618462CF0E3
:10BE8000FFFD02460B46104619462AF0E3FF024624
:10BE900007F104031B68C3F8A42107F1AC0318469B
:10BEA00023F050FB07F1B003184623F04BFB07F1DA
:10BEB000B403184623F0DCFA4FF0200024F0C8FD4C
:10BEC00003461C462346184611F040FB224607F164
:10BED00004031B68C3F8542107F104031B68D3F85B
:10BEE000542140F69413C1F200031A6007F13003A5
:10BEF00040F2DC72DA6107F130034FF009029A6117
:10BF000007F130034FF01402DA6007F130034FF00D
:10BF100014029A6007F130034FF01D025A6007F1D6
:10BF200030034FF000021A604FF0030024F090FD40
:10BF300003461C46234618464FF002014FF00D02FF
:10BF40004FF0010310F032FEC7F87C414FF01400AF
:10BF500024F07EFD03461C46214607F104031B68BE
:10BF6000D3F81C2107F104031B6800934FF4D4534A
:10BF7000C0F206030193084611464FF03802D7F885
:10BF80007C3117F065FC224607F104031B68C3F8F7
:10BF900028214FF0030024F05BFD03461C46234696
:10BFA00018464FF001014FF009024FF0010310F065
:10BFB000FDFDC7F878414FF00C0024F049FD034621
:10BFC0001C4623464FF00102009218464FF0010133
:10BFD0004FF004024FF0000310F034FCC7F8744136
:10BFE0004FF00C0024F034FD03461C4623464FF06E
:10BFF0000102009218464FF001014FF008024FF085
:10C00000000310F01FFCC7F8704107F104031B6820
:10C01000D3F8004107F1C003184623F027FA07F1CF
:10C02000BC0207F1C003104649F23841C0F20401D6
:10C030001A4623F0EDFC07F1B80207F1BC031046E5
:10C0400021461A460EF03CFF07F1B803184623F0CC
:10C050001DFA034618464FF000014FF0000233F07E
:10C060003FFA034687F89F3107F1B803184623F0DB
:10C0700069FA07F1BC03184623F064FA07F1C0031C
:10C08000184623F0F5F997F89F31002B2FD107F1CF
:10C0900004031B68D3F8004107F1C803184623F0D6
:10C0A000E5F907F1C40207F1C803104649F2384127
:10C0B000C0F204011A4623F0ABFC07F1C40320468A
:10C0C000194649F24C42C0F204024FF000030FF04F
:10C0D000F1F807F1C403184623F034FA07F1C80356
:10C0E000184623F0C5F94FF0000387F89F3107F198
:10C0F00004031B68D3F8004107F1D403184623F06A
:10C10000B5F907F1D00207F1D403104649F25441C2
:10C11000C0F204011A4623F07BFC07F1CC0207F1C0
:10C12000D003104621461A460EF0CAFE07F1CC0392
:10C13000184623F0ABF9034618464FF000014FF0C4
:10C14000000233F0CDF9034687F89E3107F1CC03A6
:10C15000184623F0F7F907F1D003184623F0F2F957
:10C1600007F1D403184623F083F997F89E31002B8A
:10C170002FD107F104031B68D3F8004107F1DC035A
:10C18000184623F073F907F1D80207F1DC031046D3
:10C1900049F25441C0F204011A4623F039FC07F178
:10C1A000D8032046194649F24C42C0F204024FF02F
:10C1B000C6030FF07FF807F1D803184623F0C2F941
:10C1C00007F1DC03184623F053F94FF0C60387F854
:10C1D0009E314FF0100024F03BFC03461C462346E2
:10C1E00097F89F21009297F89E2101921846D7F860
:10C1F0007811D7F87421D7F87031F7F759FC224637
:10C2000007F104031B68C3F830214FF0030024F04A
:10C210001FFC03461C46234618464FF000014FF012
:10C2200006024FF0010310F0C1FCC7F86C414FF05B
:10C23000540024F00DFC03461C46224607F104037B
:10C240001B681046D7F86C111A46F8F723FE2246F1
:10C2500007F104031B68C3F8F4204FF0030024F037
:10C26000F7FB03461C46234618464FF002014FF0E9
:10C270000C024FF0010310F099FC224607F1040371
:10C280001B68C3F8F8204FF00C0024F0E1FB0346D4
:10C290001C4623464FF00102009218464FF002015F
:10C2A0004FF004024FF0010310F0CCFA224607F1E0
:10C2B00004031B68C3F850214FF4967024F0C8FBA8
:10C2C00003461C46234607F1040212684FF01D0185
:10C2D00000914FF4165101914FF002010291039227
:10C2E00018464FF004014FF01C024FF0040312F007
:10C2F000C1FD224607F104031B68C3F848214FF42F
:10C30000967024F0A5FB03461C46234607F1040261
:10C3100012684FF0090100914FF4165101914FF04E
:10C3200002010291039218464FF002014FF00802F9
:10C330004FF0020312F09EFD224607F104031B6832
:10C34000C3F84C214FF4967024F082FB03461C4640
:10C35000224607F104031B68D3F8483110461946FA
:10C360000AF0E0FA2346C7F868314FF4967024F0DB
:10C370006FFB03461C46224607F104031B68D3F8F3
:10C380004C31104619460AF0CDFA2346C7F86431FD
:10C390004FF0C40024F05CFB03461C4623461846BD
:10C3A000D7F86811D7F864210AF072FE224607F127
:10C3B00004031B68C3F8042107F104031B684FF052
:10C3C000000283F8A8214FF00C0024F041FB034643
:10C3D0001C46224607F104031B68D3F804311046BB
:10C3E00019460AF087F9224607F104031B68C3F8CF
:10C3F00008214FF00C0024F02BFB03461C4622467C
:10C4000007F104031B68D3F80431104619460AF0FB
:10C410000FF9224607F104031B68C3F80C214FF003
:10C420000C0024F015FB03461C46224607F10403CA
:10C430001B68D3F804311046194609F049FF22461B
:10C4400007F104031B68C3F810214FF00C0024F01F
:10C45000FFFA03461C46224607F104031B68D3F883
:10C4600004311046194609F0ADFF224607F10403D6
:10C470001B68C3F814214FF00C0024F0E9FA0346BE
:10C480001C46224607F104031B68D3F8043110460A
:10C4900019460AF06BF8224607F104031B68C3F83B
:10C4A00018214FF0030024F0D3FA03461C4623461C
:10C4B00018464FF002014FF00B024FF0010310F04D
:10C4C00075FB224607F104031B68C3F8E82007F157
:10C4D00054034FF001029A7007F154034FF0000229
:10C4E0001A7107F154034FF00202DA7007F1540396
:10C4F0004FF002021A7007F154034FF00B025A700A
:10C5000007F104031B6818464FF013014DF6F16262
:10C51000C0F20002FEF728FB07F1540318461FF093
:10C520000DFE1EF033FE07F150034FF001021A70AA
:10C5300007F150034FF001025A7007F150034FF01A
:10C5400001029A704FF001001EF0DAFE07F150036D
:10C5500018461EF039FE4FF00403C7F82831D7F80B
:10C56000283103F00703C7F824314FF46D43CEF2AE
:10C570000003DB68C7F82031D7F820214FF6FF030E
:10C5800002EA0303C7F82031D7F824314FEA032227
:10C59000D7F8203142EA030343F0BE6343F420237B
:10C5A000C7F820314FF46D43CEF20003D7F82021B5
:10C5B000DA604FF0130387F81F314FF00003C7F81C
:10C5C000183197F91F31002B12DA4FF46D43CEF278
:10C5D000000397F81F2102F00F02A2F10401D7F81F
:10C5E0001821D2B24FEAC202D2B25B181A760EE01C
:10C5F0004FF46143CEF2000397F91F11D7F81821C9
:10C60000D2B24FEAC202D2B25B1883F800234FF0D5
:10C61000130387F817314FF46143CEF2000397F903
:10C6200017214FEA521297F8171101F01F014FF02E
:10C63000010000FA01F143F822104FF0030024F04A
:10C6400007FA03461C46234618464FF000014FF0F8
:10C6500005024FF0010310F0A9FAC7F86041D7F8BE
:10C66000600110F00FFB4FF0340024F0F1F90346A5
:10C670001C46224607F104031B681046D7F86011D8
:10C680001A46F7F71BFB224607F104031B68C3F8A1
:10C6900038214FF0030024F0DBF903461C46234603
:10C6A00018464FF000014FF004024FF0010310F064
:10C6B0007DFAC7F85C414FF0100024F0C9F9034639
:10C6C0001C46224607F104031B681046D7F85C118C
:10C6D0001A4602F0BDFE224607F104031B68C3F8A8
:10C6E00034214FF0030024F0B3F903461C462346DF
:10C6F00018464FF001014FF011024FF0010310F006
:10C7000055FA224607F104031B68C3F8F02007F12D
:10C7100004031B68D3F8F030184610F0B3FA4FF05A
:10C720000C0024F095F903461C4623464FF0010205
:10C73000009218464FF001014FF014024FF0000331
:10C7400010F080F8C7F858414FF00C0024F080F941
:10C7500003461C4623464FF00102009218464FF054
:10C7600001014FF015024FF0000310F06BF8C7F80D
:10C7700054414FF00C0024F06BF903461C4623464D
:10C780004FF00102009218464FF001014FF01602DF
:10C790004FF0000310F056F8C7F850414FF00C006E
:10C7A00024F056F903461C4623464FF0010200923E
:10C7B00018464FF001014FF019024FF0000310F03E
:10C7C00041F8C7F84C414FF00C0024F041F9034602
:10C7D0001C4623464FF00102009218464FF001011B
:10C7E0004FF01B024FF0000310F02CF8C7F848413F
:10C7F0004FF0030024F02CF903461C46234618464C
:10C800004FF000014FF000024FF0010310F0CEF99D
:10C81000C7F844414FF0030024F01AF903461C46C0
:10C82000234618464FF000014FF001024FF001037C
:10C8300010F0BCF9C7F840414FF0030024F008F9AC
:10C8400003461C46234618464FF000014FF00A02EB
:10C850004FF0010310F0AAF9C7F83C414FF0030074
:10C8600024F0F6F803461C46234618464FF0000114
:10C870004FF00B024FF0010310F098F9C7F8384160
:10C880004FF0940024F0E4F803461C46234607F1D9
:10C8900004021268D7F84C110091D7F848110191A1
:10C8A000D7F844110291D7F840110391D7F83C1101
:10C8B0000491D7F83811059106921846D7F8581107
:10C8C000D7F85421D7F85031F8F70CFE224607F17B
:10C8D00004031B68C3F8EC2007F104031B68D3F8BA
:10C8E000EC104DF6B153C0F20003C7F8E0304FF042
:10C8F0000003C7F8E43007F10402D7F8E4300093EE
:10C90000D7F8E03008464FF00001126801F06EFCE5
:10C9100007F104031B68D3F8EC104DF6ED53C0F299
:10C920000003C7F8E8304FF00003C7F8EC3007F118
:10C930000402D7F8EC300093D7F8E83008464FF0FF
:10C940000101126801F052FC07F104031B68D3F8DF
:10C95000EC104DF60163C0F20003C7F8F0304FF061
:10C960000003C7F8F43007F10402D7F8F43000935D
:10C97000D7F8F03008464FF00201126801F036FC9B
:10C9800007F104031B68D3F8EC104DF67963C0F28D
:10C990000003C7F8F8304FF00003C7F8FC3007F188
:10C9A0000402D7F8FC300093D7F8F83008464FF06F
:10C9B0000301126801F01AFC07F104031B68D3F8A5
:10C9C000004107F58473184622F050FD07F5827286
:10C9D00007F58473104649F2F411C0F204011A46B7
:10C9E00023F016F807F5807207F58273104621468A
:10C9F0001A460EF065FA07F58073184622F046FDD8
:10CA0000034618462CF03CF802460B4610461946E1
:10CA10002AF020FA05464FF0140024F019F80346D6
:10CA20001C462346DFF8142B0092019518464FF060
:10CA300000014FF01902DFF8083B09F0FBFA22462B
:10CA400007F104031B68C3F8442107F580731846F7
:10CA500022F078FD07F58273184622F073FD07F582
:10CA60008473184622F004FD4FF0140023F0F0FF09
:10CA700003461C462346DFF8CC2A0092DFF8C82A7A
:10CA8000019218464FF000014FF01702DFF8B03A5C
:10CA900009F0D0FA224607F104031B68C3F84021CD
:10CAA0004FF0140023F0D4FF03461C462346DFF862
:10CAB000942A0092DFF8902A019218464FF0010163
:10CAC0004FF01F02DFF8783A09F0B4FA224607F176
:10CAD00004031B68C3F870214FF0140023F0B8FF63
:10CAE00003461C462346DFF85C2A0092DFF8582AEA
:10CAF000019218464FF001014FF01E02DFF8403A54
:10CB000009F098FA224607F104031B68C3F8742160
:10CB10004FF0100023F09CFF03461C4623461846A6
:10CB20004FF000014FF01A02DFF8143A16F0DEFF62
:10CB3000224607F104031B68C3F8782107F10403B8
:10CB40001B68D3F878311846DFF8FC1917F026F87F
:10CB500007F104031B68D3F8D03018460FF0E2FE4B
:10CB600007F104031B68D3F8C43018460FF0DAFE4F
:10CB700007F104031B68D3F8C83018460FF0D2FE43
:10CB800007F104031B68D3F8CC3018460FF0CAFE37
:10CB900007F104031B6803F5D073184616F0AEFACC
:10CBA0000346002B00F0868049F26840C0F2040082
:10CBB0002FF046F907F104031B68D3F864311846D7
:10CBC00049F27841C0F20401FAF708F907F10C03C1
:10CBD000184610F067FF46E007F10C03184611F005
:10CBE00097FA03461A4640F2DC539A428CBF002360
:10CBF0000123DBB2002B0CD007F104031B68D3F830
:10CC00006431184649F28041C0F20401FAF7CAF8CB
:10CC100021E007F10C03184611F07AFA03461A4690
:10CC200040F6B8339A428CBF00230123DBB2002BBD
:10CC30000CD007F104031B68D3F86431184649F29D
:10CC40009041C0F20401FAF7ADF804E007F10C03DB
:10CC5000184611F0E1F907F104031B6803F5D073DE
:10CC6000184616F041FA07F104031B68D3F8EC30BC
:10CC70001846F8F7C1FD034603F40043002B14BF28
:10CC800000230123DBB2002BA6D107F104031B68AC
:10CC9000D3F864311846FAF7BDF807F104031B68AE
:10CCA000D3F864311846FAF7C5F807F10C031846B3
:10CCB00010F0D2FF49F2A840C0F2040049F2C84186
:10CCC000C0F204012EF094FF07F104031B68D3F8AF
:10CCD0006431184649F2D041C0F2040149F2C84219
:10CCE000C0F20402FAF75EF807F104031B68D3F8F8
:10CCF0006431184649F2DC41C0F2040149F2E042D5
:10CD0000C0F20402FAF76AF840F2DC5002F09EFD2D
:10CD100007F104031B68D3F86431184649F238312F
:10CD2000C0F20401FAF73EF807F104031B68D3F8D8
:10CD30006431184649F23831C0F20401FAF74EF86E
:10CD400007F104031B68D3F8D03018460FF0FAFD42
:10CD500007F104031B68D3F8C43018460FF0F2FD46
:10CD600007F104031B68D3F8C83018460FF0EAFD3A
:10CD700007F104031B68D3F8CC3018460FF0E2FD2E
:10CD800007F104031B68DFF8BC27C3F87C214FF0D0
:10CD9000E80023F05DFE03461C46204607F104032D
:10CDA0001B68D3F8641107F104031B68D3F8EC2067
:10CDB00007F104031B68D3F80031FAF7A3F9224600
:10CDC00007F104031B68C3F82C2107F104031B6857
:10CDD000D3F8EC1007F104031B68D3F82C2147F6B5
:10CDE0008133C0F20003C7F80C314FF00003C7F8DD
:10CDF00010310846114607F586730CCB01F058FA3E
:10CE000007F104031B68D3F82C514FF0480023F0BE
:10CE10001FFE03461C46224607F10403104619680C
:10CE20001CF0B4FD234628461946FAF735FC07F1F5
:10CE300004031B68D3F82C514FF0700023F008FE58
:10CE400003461C46224607F10403104619681CF0ED
:10CE500041FC234628461946FAF71EFC07F1040355
:10CE60001B68D3F82C514FF04C0023F0F1FD034622
:10CE70001C46224607F104031046196819F084FA8B
:10CE8000234628461946FAF707FC07F104031B68F6
:10CE9000D3F82C514FF0480023F0DAFD03461C462E
:10CEA000224607F10403104619681CF011FA2346C4
:10CEB00028461946FAF7F0FB07F104031B68D3F87C
:10CEC0002C514FF0500023F0C3FD03461C46224670
:10CED00007F10403104619681BF064F8234628463E
:10CEE0001946FAF7D9FB07F104031B68D3F82C5154
:10CEF0004FF0480023F0ACFD03461C46224607F1E4
:10CF000004031046196817F021FA234628461946EB
:10CF1000FAF7C2FB07F104031B68D3F82C514FF05A
:10CF2000540023F095FD03461C46224607F10403F6
:10CF30001046196818F0FCFB234628461946FAF7F4
:10CF4000ABFB07F104031B68D3F82C514FF05000E2
:10CF500023F07EFD03461C46224607F104031046DB
:10CF6000196819F083FC234628461946FAF794FB02
:10CF700007F104031B68D3F82C514FF05C0023F039
:10CF800067FD03461C46224607F104031046196854
:10CF90001AF0E4FA234628461946FAF77DFB07F112
:10CFA00004031B68D3F82C514FF0440023F050FDCC
:10CFB00003461C46224607F10403104619681AF07E
:10CFC000FBFE234628461946FAF766FB07F10403E1
:10CFD0001B68D3F82C514FF0700023F039FD034645
:10CFE0001C46224607F10403104619681BF01CFE7C
:10CFF000234628461946FAF74FFB07F104031B683E
:10D00000D3F82C514FF0440023F022FD03461C4678
:10D01000224607F10403104619681CF0BDF82346A8
:10D0200028461946FAF738FB07F104031B68D3F8C2
:10D030002C514FF0500023F00BFD03461C462246B6
:10D0400007F104031046196816F0E4FD234628464C
:10D050001946FAF721FB07F104031B68D3F82C31BA
:10D060001846FAF771FC40F69913C1F200034FF02D
:10D0700001021A7007F15C03184622F063FA07F107
:10D0800004031B68184607F5D077BD46B0BD20469F
:10D0900022F0ECFD47E2204622F0E8FD43E2204684
:10D0A00022F0E4FD3FE2204622F0E0FD3BE2204694
:10D0B00022F0DCFD37E2204622F0D8FD33E22046A4
:10D0C00022F0D4FD2FE2204622F0D0FD2BE22046B4
:10D0D00022F0CCFD27E2204622F0C8FD23E22046C4
:10D0E00022F0C4FD1FE2204622F0C0FD1BE22046D4
:10D0F00022F0BCFD17E2204622F0B8FD13E22046E4
:10D1000022F0B4FD0FE2204622F0B0FD0BE22046F3
:10D1100022F0ACFD07E2204622F0A8FD03E2204603
:10D1200022F0A4FDFFE1204622F0A0FDFBE1204615
:10D1300022F09CFDF7E1204622F098FDF3E1204625
:10D1400022F094FDEFE1204622F090FDEBE1204635
:10D1500022F08CFDE7E1204622F088FDE3E1204645
:10D1600022F084FDDFE1204622F080FDDBE1204655
:10D1700022F07CFDD7E1204622F078FDD3E1204665
:10D1800022F074FDCFE1204622F070FDCBE1204675
:10D1900022F06CFDC7E1204622F068FDC3E107F1F3
:10D1A0006003184622F0CEF9BDE107F1640318468A
:10D1B00022F0C8F9B7E107F16803184622F0C2F976
:10D1C000FFE707F16C03184622F0BCF9FFE707F10F
:10D1D0007003184622F04CF9A5E107F174031846D4
:10D1E00022F0B0F9FFE707F17803184622F040F982
:10D1F00099E107F17C03184622F0A4F9FFE707F153
:10D200008003184622F09EF9FFE707F184031846D1
:10D2100022F02EF987E107F18803184622F092F9EF
:10D22000FFE707F18C03184622F022F97BE107F1B2
:10D230009003184622F086F9FFE707F19403184699
:10D2400022F080F9FFE707F19803184622F010F961
:10D2500069E107F19C03184622F074F9FFE707F132
:10D26000A003184622F004F95DE107F1A403184673
:10D2700022F068F905E007F15C03184622F062F934
:10D28000FFE707F1A803184622F0F2F84BE107F197
:10D29000AC03184622F056F9FFE707F1B003184631
:10D2A00022F050F9FFE707F1B403184622F0E0F846
:10D2B00033E1204622F0DAFC2FE1204622F0D6FCB2
:10D2C0002BE1204622F0D2FC27E1204622F0CEFCC2
:10D2D00023E1204622F0CAFC1FE1204622F0C6FCD2
:10D2E0001BE107F1B803184622F02CF9FFE707F11C
:10D2F000BC03184622F026F9FFE707F1C0031846E1
:10D3000022F0B6F809E107F1C403184622F01AF931
:10D31000FFE707F1C803184622F0AAF8FDE007F17D
:10D32000CC03184622F00EF9FFE707F1D0031846A8
:10D3300022F008F9FFE707F1D403184622F098F825
:10D34000EBE007F1D803184622F0FCF8FFE707F1FD
:10D35000DC03184622F08CF8DFE0204622F086FC41
:10D36000DBE0204622F082FCD7E0204622F07EFC63
:10D37000D3E0204622F07AFCCFE0204622F076FC73
:10D38000CBE0204622F072FCC7E0204622F06EFC83
:10D39000C3E0204622F06AFCBFE0204622F066FC93
:10D3A000BBE0204622F062FCB7E0204622F05EFCA3
:10D3B000B3E0204622F05AFCAFE0204622F056FCB3
:10D3C000ABE0204622F052FCA7E0204622F04EFCC3
:10D3D000A3E0204622F04AFC9FE0204622F046FCD3
:10D3E0009BE0204622F042FC97E0204622F03EFCE3
:10D3F00093E0204622F03AFC8FE0204622F036FCF3
:10D400008BE0204622F032FC87E0204622F02EFC02
:10D4100083E0204622F02AFC7FE0204622F026FC12
:10D420007BE0204622F022FC77E0204622F01EFC22
:10D4300073E0204622F01AFC6FE0204622F016FC32
:10D440006BE0204622F012FC67E0204622F00EFC42
:10D4500063E0204622F00AFCFFE707F580731846D8
:10D4600022F070F8FFE707F58273184622F06AF899
:10D47000FFE707F58473184621F0FAFF4DE02046D8
:10D4800022F0F4FB49E0204622F0F0FB45E0204684
:10D4900022F0ECFB41E0204622F0E8FB3DE007F102
:10D4A0000C03184610F0D8FB37E0204622F0DEFBD4
:10D4B00033E0204622F0DAFB2FE0204622F0D6FBB4
:10D4C0002BE0204622F0D2FB27E0204622F0CEFBC4
:10D4D00023E0204622F0CAFB1FE0204622F0C6FBD4
:10D4E0001BE0204622F0C2FB17E0204622F0BEFBE4
:10D4F00013E0204622F0BAFB0FE0204622F0B6FBF4
:10D500000BE0204622F0B2FB07E0204622F0AEFB03
:10D5100003E0204622F0AAFBFFE707F15C03184670
:10D5200022F010F8FFE707F104031B6803F5D0733E
:10D53000184615F093FD22F0F5FB00BF00000442F1
:10D5400000004040000000000000803F000000009C
:10D5500080B586B002AF786053E140F69013C1F217
:10D5600000031B6818460FF091F80346FB7340F266
:10D570005843C1F200031B68DA68F97B49F2FC7377
:10D58000C0F2040300930191104649F2E841C0F251
:10D59000040149F2B422C0F204024FF401732CF0EA
:10D5A0002BF840F6D413C1F200031B68002B59D1AD
:10D5B000FB7B1B2B07D140F6D413C1F200034FF0C5
:10D5C00001021A601DE1FB7B752B23D17B68D3F828
:10D5D000A431184629F030F902460B461046194688
:10D5E00091A3D3E9002328F0C9FF02460B46104659
:10D5F000194629F02FFC02467B68C3F8A4217B68FA
:10D60000D3F844217B68D3F8A43110461946FDF7BE
:10D610000DFBF6E0FB7B642B40F0F3807B68D3F8D6
:10D62000A431184629F008F902460B46104619465F
:10D630007DA3D3E9002328F09FFF02460B46104646
:10D64000194629F007FC02467B68C3F8A4217B68D1
:10D65000D3F844217B68D3F8A43110461946FDF76E
:10D66000E5FACEE040F6D413C1F200031B68012BAB
:10D6700019D140F6D413C1F200031B68012B0AD163
:10D68000FB7B5B2B07D140F6D413C1F200034FF0B4
:10D6900002021A60B5E040F6D413C1F200034FF065
:10D6A00000021A60ADE040F6D413C1F200031B681B
:10D6B000022B40F09F8040F6D413C1F200034FF0DC
:10D6C00000021A60FB7B412B0CD140F6A813C1F27B
:10D6D00000031B6803F1010240F6A813C1F2000326
:10D6E0001A608EE0FB7B422B0CD140F6A813C1F2EE
:10D6F00000031B6803F1FF3240F6A813C1F20003D8
:10D700001A607EE0FB7B432B38D140F20403C1F268
:10D7100000031B6803F1010240F20403C1F200039D
:10D720001A6040F20403C1F200031B68042B06DCFC
:10D7300040F20403C1F200034FF005021A6040F208
:10D740000403C1F200031B68112B06DD40F2040341
:10D75000C1F200034FF011021A6040F20403C1F25B
:10D7600000031A6840F20803C1F200039B5C1A46EA
:10D7700040F6A813C1F200031A6042E0FB7B442B81
:10D780003FD140F20403C1F200031B6803F1FF32F2
:10D7900040F20403C1F200031A6040F20403C1F234
:10D7A00000031B68042B06DC40F20403C1F20003F3
:10D7B0004FF005021A6040F20403C1F200031B6837
:10D7C000112B06DD40F20403C1F200034FF01102F9
:10D7D0001A6040F20403C1F200031A6840F2080321
:10D7E000C1F200039B5C1A4640F6A813C1F2000385
:10D7F0001A6006E040F6D413C1F200034FF00002B5
:10D800001A6040F69013C1F200031B681846FDF73A
:10D81000EBF90346002B7FF4A0AE07F11007BD46DD
:10D8200080BD00BFAFF30080FCA9F1D24D62403F44
:10D83000B0B596B000AF78607B68D3F888214DF220
:10D840005153C0F200033B654FF000037B65104667
:10D85000796807F150030CCB00F04AFD02F0C2F8E2
:10D8600003461D4602F0B2F803461C4602F0C4F817
:10D87000034649F23820C0F20400294622462EF021
:10D88000B7F949F20050C0F204002EF0D9FA7B68D3
:10D8900003F5D0731846A54915F00AFC7B6807F11B
:10D8A0002C021046194610F011F97B6807F10802A6
:10D8B0001046194610F00AF900E000BF7B6803F536
:10D8C000D073184615F010FC7B6893F8A83183F0EC
:10D8D0000103DBB2002B20D007F12C03184610F017
:10D8E00017FC03461A4640F2E7339A4294BF0023DE
:10D8F0000123DBB2002B14D007F12C03184610F0E3
:10D900008BFB7B68D3F81431184608F0BDFD034645
:10D910001A467B68C3F87C2103E07B68844AC3F81D
:10D920007C217B68D3F82C311846F9F70FFD7B6812
:10D93000D3F830311846F6F7E5F87B68D3F80431B0
:10D94000184609F075FD7B68D3F8AC30184612F024
:10D950004FF840F6A413C1F200031B78002B30D01F
:10D9600049F21850C0F204002EF06AFA7B68D3F82E
:10D970000831184608F076FF7B68D3F80C3118465A
:10D9800008F06EFE7B68D3F81031184608F0B8FC3A
:10D990007B68D3F81431184608F02CFD7B68D3F867
:10D9A0001831184608F0FAFD49F22850C0F2040078
:10D9B0002EF046FA40F6A413C1F200034FF0000225
:10D9C0001A7040F6A513C1F200031B78002B18D083
:10D9D00049F23C50C0F204002EF032FA7B68D3F8D2
:10D9E0000831184608F0EEFE49F24C50C0F204002F
:10D9F0002EF026FA40F6A513C1F200034FF0000204
:10DA00001A7040F6A613C1F200031B78002B18D041
:10DA100049F25450C0F204002EF012FA7B68D3F899
:10DA20000831184608F07EFE49F24C50C0F204005E
:10DA30002EF006FA40F6A613C1F200034FF00002E2
:10DA40001A7040F6AC13C1F200031B6803F0010327
:10DA5000002B2AD140F6AC10C1F2000022F0B4FF36
:10DA60000346002B0CBF00230123DBB2002B1CD08C
:10DA70004FF0000440F6B010C1F2000010F012F8B0
:10DA800040F6AC10C1F2000022F0C0FF4DF6594341
:10DA9000C0F2010340F6B010C1F20000194640F296
:10DAA0000002C1F2000222F043F840F69813C1F2DE
:10DAB00000031B7883F00103DBB2002B06D040F695
:10DAC000B010C1F2000010F0A7FAF7E640F6B0106F
:10DAD000C1F2000010F01CFB03461A4640F2E73387
:10DAE0009A4294BF00230123DBB2002B3FF4E5AE42
:10DAF000786800F01FF8786800F046F9DEE6002C40
:10DB000006D140F6AC10C1F2000022F07BFFFFE727
:10DB100007F10803184610F09FF8FFE707F12C0300
:10DB2000184610F099F822F0FDF800BF0000A04060
:10DB30000000000080B586B002AF786040F2584324
:10DB4000C1F200031B68DA6849F2F473C0F20403FF
:10DB50000093104649F26051C0F2040149F2B42228
:10DB6000C0F2040240F2B6232BF046FD7B68D3F8E6
:10DB70006431184649F28851C0F20401F9F712F9EC
:10DB80007868FDF761F87B68D3F82C311846F9F70F
:10DB900011FF40F69813C1F200031B7883F00103D4
:10DBA000DBB2002B40F0EA8049F2A050C0F2040042
:10DBB0002EF046F97B68D3F86431184649F2B0512B
:10DBC000C0F20401F9F7EEF87B68D3F86C3118461F
:10DBD0004FF000010EF03EFF7B68D3F86831184625
:10DBE0004FF000010EF036FF7B68D3F8B8301846CE
:10DBF0004FF000010EF02EFF7B68D3F8BC301846C2
:10DC00004FF000010EF026FF7B68D3F8C0301846B5
:10DC10004FF000010EF01EFF7B68D3F8503118461C
:10DC20004FF000010EF016FF7B68D3F8AC311846B8
:10DC30004FF000010EF00EFF7B68D3F82831184634
:10DC400015F090FE40F25843C1F200031B689B6838
:10DC500018462AF0A9FF4FF01503FB734FF46143F8
:10DC6000CEF2000397F90F204FEA5212F97B01F030
:10DC70001F014FF0010000FA01F102F1200243F808
:10DC800022104FF000004FF0FF314FF000021DF066
:10DC900061FC4FF000004FF0FF314FF001021DF02A
:10DCA00059FC4FF002004FF0FF314FF000021DF021
:10DCB00051FC4FF002004FF0FF314FF001021DF018
:10DCC00049FC4FF44043C4F20F034FF44042C4F206
:10DCD0000F02D2F8802022F00202C3F880204FF415
:10DCE0004043C4F20F034FF0AA02C3F88C204FF454
:10DCF0004043C4F20F034FF05502C3F88C204FF499
:10DD00004043C4F20F03D3F8883003F00073002BB4
:10DD10000CBF00230123DBB2002BF0D14FF44043B2
:10DD2000C4F20F034FF44042C4F20F02D2F8802035
:10DD300022F00102C3F880204FF44043C4F20F03E5
:10DD40004FF0AA02C3F88C204FF44043C4F20F03F3
:10DD50004FF05502C3F88C204FF44043C4F20F0338
:10DD6000D3F8883003F08073002B0CBF002301230D
:10DD7000DBB2002BF0D11DF081F900E000BF07F10C
:10DD80001007BD4680BD00BF80B584B000AF78608D
:10DD900072B64FF40043C1F20003FB60FB6883F3EB
:10DDA0000888F2F7A7F907F11007BD4680BD00BF4C
:10DDB00080B483B000AF78607B68D3F890311B7873
:10DDC000DBB2092B14BF00230123DBB2002B08D0E8
:10DDD0007B6893F8A83183F00103DAB27B6883F89B
:10DDE000A82107F10C07BD4680BC704780B483B002
:10DDF00000AF786007F10C07BD4680BC704700BFDC
:10DE000080B582B000AF78607B68D3F890311B7822
:10DE1000DBB2112B14BF00230123DBB2002B22D075
:10DE20007B68D3F8A431184628F006FD02460B465D
:10DE3000104619460EA3D3E9002328F09FFB0246A3
:10DE40000B461046194629F005F802467B68C3F8D0
:10DE5000A4217B68D3F844217B68D3F8A431104611
:10DE60001946FCF7E3FE07F10807BD4680BD00BF79
:10DE7000FCA9F1D24D62403F80B582B000AF78601E
:10DE80007B68D3F890311B78DBB2112B14BF0023D1
:10DE90000123DBB2002B22D07B68D3F8A4311846D3
:10DEA00028F0CAFC02460B46104619460EA3D3E9D9
:10DEB000002328F061FB02460B461046194628F065
:10DEC000C9FF02467B68C3F8A4217B68D3F84421CC
:10DED0007B68D3F8A43110461946FCF7A7FE07F17A
:10DEE0000807BD4680BD00BFFCA9F1D24D62403F8E
:10DEF00080B500AF4FF001001DF002FA40F6981314
:10DF0000C1F200034FF000021A7080BD80B500AF6F
:10DF100040F25843C1F200031B68DB68184649F21F
:10DF2000BC51C0F204014FF007022BF065FB22F058
:10DF3000E3FC00BF80B582B000AF7860396049F281
:10DF4000D050C0F2040079683A682DF051FE22F0FA
:10DF5000D3FC00BF80B500AF40F25843C1F20003CC
:10DF60001B68DB68184649F2E851C0F204014FF023
:10DF700007022BF041FB1EF0040F0CBFEFF30880EB
:10DF8000EFF3098000F032B880BD00BF80B400AF6D
:10DF90001EF0040F0CBFEFF30880EFF3098000F0D0
:10DFA00025B8BD4680BC704780B500AF49F2FC5033
:10DFB000C0F204004FF007012DF01AFE1EF0040F0E
:10DFC0000CBFEFF30880EFF3098000F00FB880BDBD
:10DFD00080B400AF1EF0040F0CBFEFF30880EFF326
:10DFE000098000F003B8BD4680BC704780B58AB098
:10DFF00000AF786049F20C60C0F204004FF00701F6
:10E000002DF0F6FD7B681B687B627B6803F10403DF
:10E010001B683B627B6803F108031B68FB617B683C
:10E0200003F10C031B68BB617B6803F110031B68E1
:10E030007B617B6803F114031B683B617B6803F120
:10E0400018031B68FB607B6803F11C031B68BB6043
:10E0500049F21C60C0F204002DF0F2FE49F24C605F
:10E06000C0F20400796A2DF0C3FD49F25860C0F295
:10E070000400396A2DF0BCFD49F26460C0F204006E
:10E08000F9692DF0B5FD49F27060C0F20400B9697C
:10E090002DF0AEFD49F27C60C0F2040079692DF0EC
:10E0A000A7FD49F28860C0F2040039692DF0A0FD97
:10E0B00049F2B860C0F20400F9682DF099FD49F208
:10E0C000DC60C0F20400B9682DF092FD4EF63853C2
:10E0D000CEF200031B6849F2E860C0F20400194662
:10E0E0002DF086FD4EF62853CEF200031B6849F250
:10E0F000F460C0F2040019462DF07AFD4EF62C5360
:10E10000CEF200031B6849F20070C0F20400194609
:10E110002DF06EFD4EF63053CEF200031B6849F22F
:10E120000C70C0F2040019462DF062FD4EF63C530F
:10E13000CEF200031B6849F21870C0F204001946C1
:10E140002DF056FD4FF46D43CEF200035B6A49F2A9
:10E150002470C0F2040019462DF04AFD22F0CCFBD9
:10E1600080B500AF40F68813C1F200031B6803F1CD
:10E17000010240F68813C1F200031A6040F69913B9
:10E18000C1F200031B78002B1BD040F68C13C1F2A8
:10E1900000031B68D3F8E8301846F5F77BFC03460C
:10E1A000002B07D040F69813C1F200034FF0000295
:10E1B0001A7006E040F69813C1F200034FF0010216
:10E1C0001A7080BD80B582B000AF786039603B685E
:10E1D000002B07D07B6803F10C023B461046194622
:10E1E00000F0C0F807F10807BD4680BD82B090B5C9
:10E1F00085B000AFF8607A607B620B46FB727B6A89
:10E20000002B04D1BB6A03F00103002B46D07B68CE
:10E21000002B45D0FB6803F13002FB7A4FEA830301
:10E22000D3181B68002B24D14FF0180022F010FCEB
:10E2300003461C4623464FF000021A604FF00002CE
:10E240005A604FF000029A604FF00002DA604FF01F
:10E2500000021A614FF000025A611846F5F714FDEA
:10E26000FB6803F13002FB7A4FEA8303D31822469E
:10E270001A60FB6803F13002FB7A4FEA8303D3187C
:10E280001B681846796807F124030CCB00F092F85C
:10E2900007E0204621F0EAFC21F044FD00BF00E049
:10E2A00000BF07F11407BD46BDE8904002B07047BB
:10E2B00080B584B000AFF860B960394681E80C00E1
:10E2C0003B68002B04D17B6803F00103002B0BD0CB
:10E2D000BB68002B08D0FB6803F178031846B968C7
:10E2E0003B460CCB00F098F807F11007BD4680BD07
:10E2F00080B584B000AFF860B960394681E80C00A1
:10E300003B68002B04D17B6803F00103002B0BD08A
:10E31000BB68002B08D0FB6803F598731846B968F2
:10E320003B460CCB00F046F807F11007BD4680BD18
:10E3300080B483B000AF78607B68184607F10C07A3
:10E34000BD4680BC704700BF80B584B000AFF860A8
:10E35000B9607A60F868B96800F0A4F807F11007AE
:10E36000BD4680BD80B582B000AF786039607B6803
:10E370005A687B689B689A420FD07B681A467B6814
:10E380005B68104619463A6800F09AF87B685B684B
:10E3900003F104027B685A6008E07868F8F72EFA07
:10E3A0000346786819463A6800F0A2F807F10807B2
:10E3B000BD4680BD90B587B000AFF860B960394602
:10E3C00081E80C00BB68002B21D03B68002B04D1F6
:10E3D0007B6803F00103002B19D04FF0100022F0EE
:10E3E00037FB03461C462346184600F079F97C614A
:10E3F0007869B9683B460CCB00F092F9FA687B6902
:10E400003B6107F1100310461946F6F7D5F807F1FE
:10E410001C07BD4690BD00BF90B587B000AFF86047
:10E42000B960394681E80C00BB68002B21D03B68FD
:10E43000002B04D17B6803F00103002B19D04FF0AF
:10E44000100022F005FB03461C462346184600F048
:10E450009BF97C617869B9683B460CCB00F0B4F954
:10E46000FA687B693B6107F110031046194600F01A
:10E47000CFF907F11C07BD4690BD00BF80B584B041
:10E4800000AFF860B9607A60BB68002B05D0FB680C
:10E490001846B9687A6800F0E3F907F11007BD463D
:10E4A00080BD00BF80B582B000AF78603960786809
:10E4B000396800F0E3F907F10807BD4680BD00BFE9
:10E4C00080B584B000AFF860B9607A60BB684FF087
:10E4D00004001946F5F7CCFB03461A46002A02D081
:10E4E0007A6812681A6007F11007BD4680BD00BF48
:10E4F000B0B58AB000AFF860B9607A60FB685A685E
:10E50000FB689B689A4232D0FB681946FB685A68E0
:10E51000FB685B68A3F10403084611461A46FFF73F
:10E52000CFFFFB685B6803F10402FB685A607B68FD
:10E530001B683B6207F108031846F8F799FA03468F
:10E540001968FB685B68A3F10802FB685B68A3F1CC
:10E550000403084611461A4600F09AF907F1080329
:10E56000184600F0AFF903463A6A1A60B4E0F8685A
:10E570004FF0010149F23872C0F2040200F0AEF926
:10E580000346FB61F868F7F749FF03463B6107F173
:10E59000080207F110031046194600F0E9F9034696
:10E5A000BB61FB681846F96900F0FAF903467B6124
:10E5B0007B697B62FB681A46BB694FEA8303796912
:10E5C000CB18104619467A68FFF77AFF4FF0000320
:10E5D0007B62FB681D6807F108031846F8F748FAE4
:10E5E00003461C68FB681846FFF7A2FE0346284650
:10E5F00021467A6900F0ECF903467B627B6A03F1FD
:10E6000004037B6207F108031846F8F731FA034662
:10E610001D68FB685C68FB681846FFF789FE0346C7
:10E62000284621467A6A00F0D3F903467B62FB68EC
:10E630001D68FB685C68FB681846FFF779FE0346B7
:10E64000284621461A46FFF77FFEF968FB681A68DC
:10E65000FB689B681846FB681B68C31A4FEAA30354
:10E66000084611461A46FFF709FFFB687A691A60E7
:10E67000FB687A6A5A60FB694FEA83037A69D218A9
:10E68000FB689A6028E021F04FFD21F04BFB034628
:10E69000184621F0FFFC7B6A002B0BD1FB681A4661
:10E6A000BB694FEA83037969CB1810461946F8F71E
:10E6B000FDF809E0FB681846FFF73AFE0346786963
:10E6C000796A1A46FFF740FEFB6818467969FA69CD
:10E6D000FFF7D4FE22F010F907F12807BD46B0BDC0
:10E6E00080B582B000AF78607B681846F5F710FF00
:10E6F0007B680A4A1A607B684FF000025A607B68A8
:10E700004FF000029A607B684FF00002DA607B688D
:10E71000184607F10807BD4680BD00BF7897040082
:10E7200080B485B000AFF860B960394681E80C006C
:10E73000BB68002B12D03B68002B04D17B6803F030
:10E740000103002B0AD0FB68BA685A60FB6803F12A
:10E7500008033A4692E8030083E8030007F1140730
:10E76000BD4680BC704700BF80B483B000AF786006
:10E770007B68044A1A607B68184607F10C07BD469F
:10E7800080BC70476897040080B582B000AF7860A5
:10E790007B681846FFF7E8FF7B680A4A1A607B68C7
:10E7A0004FF000025A607B684FF000029A607B686D
:10E7B0004FF00002DA607B68184607F10807BD4693
:10E7C00080BD00BF5897040080B485B000AFF860EA
:10E7D000B960394681E80C00BB68002B12D03B6859
:10E7E000002B04D17B6803F00103002B0AD0FB68E7
:10E7F000BA685A60FB6803F108033A4692E80300DE
:10E8000083E8030007F11407BD4680BC704700BFD2
:10E8100080B582B000AF786039607B685A687B68E9
:10E820009B689A420FD07B681A467B685B681046EB
:10E8300019463A6800F0E0F87B685B6803F104026F
:10E840007B685A6008E0786800F0E6F9034678686B
:10E8500019463A6800F0E8F807F10807BD4680BDA0
:10E8600080B584B000AFF860B9607A60B86821F014
:10E87000FDF907F11007BD4680BD00BF80B483B02D
:10E8800000AF7860396007F10C07BD4680BC704767
:10E8900090B585B000AFF860B9607A60F86800F0B4
:10E8A000CFF903461C46B86800F0CAF90346204673
:10E8B00019467A6800F0D2F90346184607F11407A2
:10E8C000BD4690BD80B483B000AF78607B681B68A4
:10E8D000184607F10C07BD4680BC704790B587B05D
:10E8E00000AFF860B9607A60F86800F0D5F90346C7
:10E8F0001C46F868F7F76EFD0346E21ABB689A42B9
:10E900002CBF00230123DBB2002B02D0786820F05B
:10E9100075FBF868F7F75EFD0446F868F7F75AFDEF
:10E9200003463B6107F1100207F108031046194640
:10E93000F6F716F803461B68E3187B61F868F7F7EB
:10E9400049FD02467B699A4207D8F86800F0A4F9AD
:10E9500003461A467B699A4204D2F86800F09CF993
:10E96000034600E07B69184607F11C07BD4690BDD1
:10E9700090B583B000AF786039607868F8F778F8C0
:10E9800003461B681C463868F8F772F803461B6894
:10E99000E31A4FEAA303184607F10C07BD4690BDE2
:10E9A00080B582B000AF786039603B68002B08D03A
:10E9B0007B68184639684FF0000200F07FF9034683
:10E9C00001E04FF00003184607F10807BD4680BD7F
:10E9D00080B584B000AFF860B9607A603B60F868D9
:10E9E000B9687A683B6800F089F90346184607F170
:10E9F0001007BD4680BD00BF80B584B000AFF86091
:10EA0000B9607A60BB684FF004001946F5F730F939
:10EA100003461A46002A02D07A6812681A6007F183
:10EA20001007BD4680BD00BFB0B58AB000AFF8602A
:10EA3000B9607A60FB685A68FB689B689A4232D07A
:10EA4000FB681946FB685A68FB685B68A3F104031E
:10EA5000084611461A46FFF7CFFFFB685B6803F1D3
:10EA60000402FB685A607B681B683B6207F108037D
:10EA7000184600F055F903461968FB685B68A3F176
:10EA80000802FB685B68A3F10403084611461A46B6
:10EA900000F052F907F10803184600F067F9034641
:10EAA0003A6A1A60B4E0F8684FF0010149F238722E
:10EAB000C0F2040200F066F90346FB61F86800F05A
:10EAC000ABF903463B6107F1080207F1100310465A
:10EAD000194600F0B3F90346BB61FB681846F969B3
:10EAE00000F0C4F903467B617B697B62FB681A46D0
:10EAF000BB694FEA83037969CB18104619467A68D7
:10EB0000FFF77AFF4FF000037B62FB681D6807F197
:10EB10000803184600F004F903461C68FB68184611
:10EB2000F7F734FD0346284621467A6900F0B6F926
:10EB300003467B627B6A03F104037B6207F10803EF
:10EB4000184600F0EDF803461D68FB685C68FB683A
:10EB50001846F7F71BFD0346284621467A6A00F05F
:10EB60009DF903467B62FB681D68FB685C68FB6877
:10EB70001846F7F70BFD0346284621461A46F7F7D5
:10EB800011FDF968FB681A68FB689B681846FB680A
:10EB90001B68C31A4FEAA303084611461A46F7F743
:10EBA000B7FEFB687A691A60FB687A6A5A60FB698B
:10EBB0004FEA83037A69D218FB689A6028E021F053
:10EBC000B3FA21F0AFF80346184621F063FA7B6AE6
:10EBD000002B0BD1FB681A46BB694FEA83037969A6
:10EBE000CB181046194600F06DF909E0FB6818468D
:10EBF000F7F7CCFC03467869796A1A46F7F7D2FC36
:10EC0000FB6818467969FA69F7F782FE21F074FE0D
:10EC100007F12807BD46B0BD80B584B000AF78606D
:10EC20007B6803F1040307F10C021046194600F05B
:10EC300053F9FB68184607F11007BD4680BD00BFB9
:10EC400080B582B000AF7860786800F055F903466F
:10EC5000184607F10807BD4680BD00BFB0B584B0B7
:10EC600000AFF860B9607A60F86800F051F90546C5
:10EC7000B86800F04DF90446786800F049F9034699
:10EC8000284621461A4600F051F90346184607F176
:10EC90001007BD46B0BD00BF80B582B000AF786040
:10ECA0007B68184600F056F90346184600F05EF9F6
:10ECB0000346184607F10807BD4680BD80B584B0FD
:10ECC00000AFF860B9607A60F86800F04FF902466A
:10ECD000BB689A422CBF00230123DBB2002B01D07A
:10ECE00020F048F9BB684FEA8303184621F0B0FED4
:10ECF0000346184607F11007BD4680BD80B584B0B5
:10ED000000AFF860B9607A603B60F868B9687A680B
:10ED100000F038F90346184607F11007BD4680BDDC
:10ED200080B483B000AF78607B68184607F10C07A9
:10ED3000BD4680BC704700BF90B585B000AFF8609D
:10ED4000B9607A60F86800F02FF903461C46B8688D
:10ED500000F02AF90346204619467A6800F032F995
:10ED60000346184607F11407BD4690BD80B483B032
:10ED700000AF78607B681B68184607F10C07BD463A
:10ED800080BC704790B587B000AFF860B9607A601A
:10ED9000F86800F035F903461C46F868F7F76AFC96
:10EDA0000346E21ABB689A422CBF00230123DBB260
:10EDB000002B02D0786820F021F9F868F7F75AFCA8
:10EDC0000446F868F7F756FC03463B6107F110026A
:10EDD00007F1080310461946F5F7C2FD03461B6804
:10EDE000E3187B61F868F7F745FC02467B699A42B5
:10EDF00007D8F86800F004F903461A467B699A427E
:10EE000004D2F86800F0FCF8034600E07B6918467D
:10EE100007F11C07BD4690BD80B584B000AF786097
:10EE20007B6807F10C021046194600F055F8FB68A4
:10EE3000184607F11007BD4680BD00BF90B583B0EE
:10EE400000AF786039607868FFF76AFF03461B6897
:10EE50001C463868FFF764FF03461B68E31A4FEA55
:10EE6000A303184607F10C07BD4690BD80B582B0DC
:10EE700000AF786039603B68002B08D07B6818468B
:10EE800039684FF0000200F0CDF8034601E04FF082
:10EE90000003184607F10807BD4680BD80B584B061
:10EEA00000AFF860B9607A603B60F868B9687A686A
:10EEB0003B6800F0D7F80346184607F11007BD4637
:10EEC00080BD00BF80B483B000AF7860396007F1C7
:10EED0000C07BD4680BC704780B483B000AF78603B
:10EEE00039603B681A687B681A607B68184607F1CE
:10EEF0000C07BD4680BC704780B483B000AF78601B
:10EF00007B68184607F10C07BD4680BC704700BF00
:10EF100080B582B000AF78607868FFF7EDFF0346F8
:10EF2000184607F10807BD4680BD00BF80B586B012
:10EF300000AFF860B9607A604FF00103FB75F868C4
:10EF4000B9687A6800F0A0F80346184607F1180778
:10EF5000BD4680BD80B483B000AF78607B68184642
:10EF600007F10C07BD4680BC704700BF80B483B07A
:10EF700000AF78606FF04043184607F10C07BD46BC
:10EF800080BC704780B584B000AFF860B9607A602B
:10EF9000F868B9687A6800F0A1F80346184607F1E6
:10EFA0001007BD4680BD00BF80B582B000AF78605D
:10EFB000786800F0A5F80346184607F10807BD4633
:10EFC00080BD00BFB0B584B000AFF860B9607A60B2
:10EFD000F86800F0A1F80546B86800F09DF804460E
:10EFE000786800F099F80346284621461A4600F052
:10EFF000A1F80346184607F11007BD46B0BD00BF93
:10F0000080B582B000AF78607B68184600F0A6F843
:10F010000346184600F0AEF80346184607F1080705
:10F02000BD4680BD80B584B000AFF860B9607A603D
:10F03000F86800F09FF80246BB689A422CBF002394
:10F040000123DBB2002B01D01FF094FFBB684FEA15
:10F050008303184621F0FCFC0346184607F110070D
:10F06000BD4680BD80B584B000AFF860B9607A60FD
:10F070003B60F868B9687A6800F088F8034618467B
:10F0800007F11007BD4680BD80B586B000AFF860BF
:10F09000B9607A60BA68FB68D31A4FEAA3037B6150
:10F0A0007B69002B0ED07B694FEA8303C3F1000319
:10F0B0007A68D2187B694FEA83031046F9681A46CA
:10F0C0002CF098FB7B694FEA8303C3F100037A6855
:10F0D000D318184607F11807BD4680BD80B584B027
:10F0E00000AFF860B9607A60F868B9687A6800F0D3
:10F0F0005FF80346184607F11007BD4680BD00BF04
:10F1000080B483B000AF78607B68184607F10C07C5
:10F11000BD4680BC704700BF80B582B000AF78604C
:10F120007868FFF7EDFF0346184607F10807BD466C
:10F1300080BD00BF80B586B000AFF860B9607A606E
:10F140004FF00103FB75F868B9687A6800F04AF877
:10F150000346184607F11807BD4680BD80B483B04A
:10F1600000AF78607B68184607F10C07BD4680BC8D
:10F17000704700BF80B483B000AF78606FF0404349
:10F18000184607F10C07BD4680BC704780B584B0B7
:10F1900000AFF860B9607A60F868B9687A6800F022
:10F1A0004BF80346184607F11007BD4680BD00BF67
:10F1B00090B585B000AFF860B9607A60F868FFF785
:10F1C0003FFD03461C46B868FFF73AFD034620465C
:10F1D00019467A6800F042F80346184607F114070A
:10F1E000BD4690BD80B586B000AFF860B9607A606A
:10F1F000BA68FB68D31A4FEAA3037B617B69002BD3
:10F200000ED07B694FEA8303C3F100037A68D218FA
:10F210007B694FEA83031046F9681A462CF0EAFA34
:10F220007B694FEA8303C3F100037A68D318184659
:10F2300007F11807BD4680BD80B584B000AFF86007
:10F24000B9607A60F868B9687A6800F025F8034612
:10F25000184607F11007BD4680BD00BFB0B584B0A9
:10F2600000AFF860B9607A60F868FFF751FE0546B4
:10F27000B868FFF74DFE04467868FFF749FE03467D
:10F28000284621461A46F7F7B5FC0346184607F10B
:10F290001007BD46B0BD00BF90B585B000AFF860A7
:10F2A000B9607A60F868FFF77FFE03461C46B868CD
:10F2B000FFF77AFE0346204619467A6800F006F802
:10F2C0000346184607F11407BD4690BDB0B584B09B
:10F2D00000AFF860B9607A60F868FFF71DFF054677
:10F2E000B868FFF719FF04467868FFF715FF034673
:10F2F000284621461A4600F007F80346184607F14B
:10F300001007BD46B0BD00BF80B586B000AFF86045
:10F31000B9607A604FF00103FB75F868B9687A68E4
:10F3200000F006F80346184607F11807BD4680BDF1
:10F3300080B586B000AFF860B9607A60BA68FB68E3
:10F34000D31A4FEAA3037B617B69002B07D07B694B
:10F350004FEA83037868F9681A462CF04BFA7B6908
:10F360004FEA83037A68D318184607F11807BD4699
:10F3700080BD00BF80B582B000AF786039607B6827
:10F380005B68002B29D07B689B68002B05D17B68CC
:10F39000DB6803F00103002B1FD07B68DB6803F000
:10F3A0000103DBB2002B0CD07B685A687B68DB68FA
:10F3B0004FEA6303D3181A687B689B68D3181B68ED
:10F3C00001E07B689B687A6851687A68D2684FEA86
:10F3D00062028A1810463968984707F10807BD4647
:10F3E00080BD00BF80B582B000AF78607B685B688D
:10F3F000002B28D07B689B68002B05D17B68DB68DD
:10F4000003F00103002B1ED07B68DB6803F00103CF
:10F41000DBB2002B0CD07B685A687B68DB684FEA54
:10F420006303D3181A687B689B68D3181B6801E0D4
:10F430007B689B687A6851687A68D2684FEA620292
:10F440008A181046984707F10807BD4680BD00BFDF
:10F4500090B58BB002AFF860B9607A60FB68BA68AB
:10F460001A60FB687A685A60FB68294ADA604FF0D4
:10F47000240021F0EDFA03461C462346184679681D
:10F480000EF024FB2246FB689A604FF25153C0F203
:10F4900000037B614FF00003BB61BB6900937B6994
:10F4A00078684FF01501FA6800F0C4F8B868F4F70E
:10F4B000C7FB03461C46B868F4F7CEFB03464FF083
:10F4C000010202FA03F3204619464FF001021BF035
:10F4D000DFFF4FF01503FB774FF46143CEF20003DB
:10F4E00097F91F204FEA5212F97F01F01F014FF0E8
:10F4F000010000FA01F143F82210FB68184607F1F9
:10F500002407BD4690BD204620F0B0FB20F00AFC49
:10F510000000000080B584B000AF78607B689B6815
:10F5200018460EF04DFE0346FB60FA6848F2804331
:10F53000C0F21E039A4202D97B68044ADA607B68F3
:10F54000DB68184607F11007BD4680BD00000000CB
:10F5500090B585B000AF78607B681B681846F4F7FB
:10F560006FFB03461C467B681B681846F4F774FB68
:10F570000346204619464FF001021CF055F8034699
:10F58000002B0CBF00230123DBB2002B46D07B688D
:10F590009B6818460EF014FE0346FB607B689B6870
:10F5A00018460EF039FD7B681B681846F4F748FBD7
:10F5B00003461C467B681B681846F4F74DFB034660
:10F5C0004FF0010202FA03F3204619461CF08CF8B2
:10F5D000FA6848F28043C0F21E039A4203D97B685E
:10F5E000104ADA601AE0F86827F03AFD03460E4840
:10F5F000194627F041FE034618460C4927F03CFE09
:10F60000034618460A4927F083FD03461846084971
:10F6100027F07EFD03461A467B68DA6007F114077F
:10F62000BD4690BD00000000002474490040934591
:10F630000000704282B090B585B000AFF8607A608B
:10F640007B620B46FB727B6A002B04D1BB6A03F022
:10F650000103002B43D07B68002B42D0FA6897F956
:10F660000B304FEA8303D3181B68002B23D14FF0D4
:10F67000180021F0EDF903461C4623464FF0000226
:10F680001A604FF000025A604FF000029A604FF08B
:10F690000002DA604FF000021A614FF000025A6176
:10F6A0001846F4F7F1FAFA6897F90B304FEA83033A
:10F6B000D31822461A60FA6897F90B304FEA830391
:10F6C000D3181B681846796807F124030CCB00F0A7
:10F6D00011F807E0204620F0C9FA20F023FB00BF14
:10F6E00000E000BF07F11407BD46BDE8904002B03E
:10F6F000704700BF90B587B000AFF860B960394679
:10F7000081E80C00BB68002B21D03B68002B04D1A2
:10F710007B6803F00103002B19D04FF0100021F09B
:10F7200097F903461C462346184600F015F87C61FD
:10F730007869B9683B460CCB00F02EF8FA687B6913
:10F740003B6107F1100310461946F4F735FF07F146
:10F750001C07BD4690BD00BF80B582B000AF786089
:10F760007B681846F4F7D4FE7B680A4A1A607B6807
:10F770004FF000025A607B684FF000029A607B688D
:10F780004FF00002DA607B68184607F10807BD46B3
:10F7900080BD00BF1898040080B485B000AFF86049
:10F7A000B960394681E80C00BB68002B12D03B6879
:10F7B000002B04D17B6803F00103002B0AD0FB6807
:10F7C000BA685A60FB6803F108033A4692E80300FE
:10F7D00083E8030007F11407BD4680BC704700BFF3
:10F7E00080B582B000AF78607B685B68002B28D062
:10F7F0007B689B68002B05D17B68DB6803F0010305
:10F80000002B1ED07B68DB6803F00103DBB2002B0A
:10F810000CD07B685A687B68DB684FEA6303D318B7
:10F820001A687B689B68D3181B6801E07B689B683B
:10F830007A6851687A68D2684FEA62028A1810467C
:10F84000984707F10807BD4680BD00BF80B584B06A
:10F8500000AF786040F69C13C1F200031B681846A5
:10F860000DF070F840F68813C1F200031B68FB60CE
:10F8700040F68813C1F200031A68FB68D21A7B684D
:10F880009A422CBF00230123DBB2002BF0D140F6BB
:10F890009C13C1F200031B6818460DF043F807F1F2
:10F8A0001007BD4680BD00BF90B583B000AF4FF4D8
:10F8B000D87021F0CDF803461C4623461846FBF7C6
:10F8C00083FA7C607868FDF7B3FF4FF000031846B9
:10F8D00007F10C07BD4690BD204620F0C7F920F087
:10F8E00021FA00BF80B58AB002AFF860B9607A60D3
:10F8F000F8682DF0FDFF034603F10103184621F0DF
:10F90000D7F80346FB61F869F9682DF09FFCF869A8
:10F9100049F65001C0F204012FF086FCB861BB69C2
:10F92000002B07D0F8694FF02F012DF0EBFA0346BA
:10F93000002B02D14FF0FF3322E0B86903F066F8E4
:10F940000346FB754FF0000049F65401C0F2040174
:10F950002FF06AFC38617A6897F91730396900919D
:10F96000B868114649F65802C0F204022DF07CF93D
:10F97000FB69002B02D0F86920F07CF94FF00003FE
:10F98000184607F12007BD4680BD00BF80B582B094
:10F9900000AF7860396029F099F803464FF01602FD
:10F9A0001A604FF0FF33184607F10807BD4680BDC7
:10F9B00080B483B000AF7860FEE700BF80B400AFD2
:10F9C0004FF001031846BD4680BC704780B400AFBD
:10F9D00040F6D813C1F200031B681846BD4680BC30
:10F9E000704700BF90B400AFEFF308842346184679
:10F9F000BD4690BC704700BF98B500AFFFF7E6FF6B
:10FA000002466FF060439A428CBF00230123DBB2B1
:10FA1000002B0AD0FFF7E6FF03461C46FFF7D6FF90
:10FA20000346E31A03F5004306E0FFF7CFFF034662
:10FA3000C3F1005303F50423184698BD90B585B073
:10FA400000AF786040F6D813C1F200031B68002BAA
:10FA500008D140F6D813C1F2000341F25042C1F27E
:10FA600000021A6040F6D813C1F200031A686FF062
:10FA700060439A4229D840F6D813C1F200031A68AD
:10FA80007B68D418FFF7AEFF03469C4294BF002367
:10FA90000123DBB2002B27D040F6D813C1F20003BC
:10FAA0001A687B68D2184FF48043C2F208039A4266
:10FAB00001D9FEF72BFA40F6D813C1F200034FF438
:10FAC0004042C2F207021A600EE040F6D813C1F2BB
:10FAD00000031A687B68D2184FF48043C2F208030F
:10FAE0009A4201D9FEF712FA40F6D813C1F2000388
:10FAF0001B68FB6040F6D813C1F200031A687B68EC
:10FB0000D21840F6D813C1F200031A60FB681846F9
:10FB100007F11407BD4690BD90B591B002AFF860F3
:10FB2000B9607A60BB6803F00103DBB2002B03D03D
:10FB30004FF002037B630BE0BB6803F00203002B72
:10FB400003D04FF003037B6302E04FF001037B63BC
:10FB5000BB6803F40073002B17D0BB6803F4006389
:10FB6000002B04D07B6B43F004037B630DE0BB6888
:10FB700003F48063002B04D07B6B43F008037B63AA
:10FB800003E07B6B43F010037B63F8682DF0B0FE5D
:10FB9000034603F10703FB62FB6A184620F088FF67
:10FBA0000346BB62F868B96AFA6AFFF79BFE034630
:10FBB000002B0CBF00230123DBB2002B0ED0BB6A4D
:10FBC000002B02D0B86A20F055F828F07FFF0346DA
:10FBD0004FF016021A604FF0FF33A7E04FF40970A0
:10FBE00020F036FF03467B617A697B6BDBB21046FF
:10FBF000B96A1A46F2F796FD034687F82730BB6AC2
:10FC0000002B02D0B86A20F035F897F82730002B87
:10FC100026D028F05BFF03461C4697F8273018468D
:10FC200002F062FF0346236040F25843C1F2000332
:10FC30001B68DC6828F04AFF03461B6818462DF055
:10FC400063FB034697F827200092204649F660019F
:10FC5000C0F20401FA6829F0CFFC4FF0FF3365E0F1
:10FC600040F6DC10C1F2000000F014FC044640F63F
:10FC7000DC10C1F2000000F01FFC02464FF0000350
:10FC8000BB6107F11803204611461A4600F028FC14
:10FC900003463B6140F6DC10C1F2000000F00CFCB2
:10FCA0000346FB6107F1100207F11C0310461946D9
:10FCB00000F02CFC0346002B1FD040F6DC10C1F2F4
:10FCC000000000F0E7FB03463B6207F1100207F17A
:10FCD00020031046194600F033FC034687F8333002
:10FCE00097F8333040F6DC10C1F20000194600F0FE
:10FCF0003FFC03467A691A6014E007F1140340F6EA
:10FD0000DC10C1F20000194600F046FC40F6DC10A1
:10FD1000C1F2000000F068FC0346DBB203F1FF33E0
:10FD200087F8333097F8333003F10303184607F1AF
:10FD30003C07BD4690BD00BF90B585B000AF786070
:10FD40007B68002B08DA28F0C1FE03464FF0090259
:10FD50001A604FF0FF3374E07B68022B02DC4FF037
:10FD600000036EE07C6840F6DC10C1F2000000F099
:10FD70003BFC034603F102039C4294BF0023012392
:10FD8000DBB2002B08D028F0A1FE03464FF0090299
:10FD90001A604FF0FF3354E07B68A3F103037B60EC
:10FDA0007B6840F6DC10C1F20000194600F0E0FB71
:10FDB00003461B681846F3F77FFA0346FB737B681C
:10FDC00040F6DC10C1F20000194600F0D1FB0346FA
:10FDD0001B6818461FF04AFF7B6840F6DC10C1F232
:10FDE0000000194600F0C4FB03464FF000021A6001
:10FDF000FB7B002B23D028F069FE03461C46FB7BCF
:10FE0000184602F071FE0346236040F25843C1F2E7
:10FE100000031B68DC6828F059FE03461B6818467F
:10FE20002DF072FA03461A46FB7B204649F68C01F8
:10FE3000C0F2040129F0E0FB4FF0FF3301E04FF086
:10FE40000003184607F11407BD4690BD80B483B087
:10FE500000AF786039603B684FF400525A604FF051
:10FE60000003184607F10C07BD4680BC704700BF71
:10FE700090B585B000AF78607B68A3F1030340F6CE
:10FE8000DC10C1F20000194600F072FB03461B684B
:10FE90001846F3F74DF90346FB73FB7B002B0CD0A0
:10FEA00028F014FE03461C46FB7B184602F01CFE9D
:10FEB000034623604FF0FF3301E04FF00003184684
:10FEC00007F11407BD4690BD80B483B000AF7860E1
:10FED0004FF00103184607F10C07BD4680BC704780
:10FEE00090B587B000AF786078682DF001FD0346CB
:10FEF00003F107037B617B69184620F0D9FD0346B7
:10FF00003B61786839697A69FFF7ECFC0346002B9E
:10FF10000CBF00230123DBB2002B0ED03B69002B6A
:10FF200002D038691FF0A6FE28F0D0FD03464FF03E
:10FF300016021A604FF0FF331CE03869F3F73EFBFE
:10FF40000346FB733B69002B02D038691FF092FE19
:10FF5000FB7B002B0CD028F0B9FD03461C46FB7B35
:10FF6000184602F0C1FD034623604FF0FF3301E065
:10FF70004FF00003184607F11C07BD4690BD00BFB7
:10FF800090B589B000AF786039604FF0FF33FB6106
:10FF900078682DF0ADFC034603F10703BB613868B8
:10FFA0002DF0A6FC034603F107037B61BB691846ED
:10FFB00020F07EFD03463B617B69184620F078FD0A
:10FFC0000346FB6078683969BA69FFF78BFC034622
:10FFD000002B0CBF00230123DBB2002B14D03B69A4
:10FFE000002B02D038691FF045FEFB68002B02D0C1
:10FFF000F8681FF03FFE28F069FD03464FF0160237
:020000021000EC
:100000001A604FF0FF334EE03868F9687A69FFF7FD
:1000100069FC0346002B0CBF00230123DBB2002B3D
:1000200014D03B69002B02D038691FF023FEFB6817
:10003000002B02D0F8681FF01DFE28F047FD034694
:100040004FF016021A604FF0FF332CE0F8684FF0C3
:100050002F012CF057FF034638691946F3F780FB50
:100060000346FB72FB7A002B03D14FF00003FB61C8
:100070000CE028F02BFD03461C46FB7A184602F0E4
:1000800033FD034623604FF0FF33FB613B69002BD8
:1000900002D038691FF0EEFDFB68002B02D0F86833
:1000A0001FF0E8FDFB69184607F12407BD4690BD27
:1000B00090B587B000AFF860B9607A60FB68002B3C
:1000C00008DA28F003FD03464FF009021A604FF0EA
:1000D000FF336BE0FB68022B02DC4FF0000365E0AE
:1000E000FC6840F6DC10C1F2000000F07DFA034627
:1000F00003F102039C4294BF00230123DBB2002BD7
:1001000008D028F0E3FC03464FF009021A604FF0D4
:10011000FF334BE0FB68A3F10303FB607B68012B1B
:1001200003D0022B10D0002B1DE0FB6840F6DC1042
:10013000C1F20000194600F01BFA03461B689A68DA
:10014000BB68D318BB600EE0FB6840F6DC10C1F260
:100150000000194600F00CFA03461B68DA68BB6819
:10016000D31ABB6000BFFB6840F6DC10C1F2000090
:10017000194600F0FDF903461A68BB681046194697
:10018000F3F7B0F80346FB75FB7D002B0CD028F08D
:100190009DFC03461C46FB7D184602F0A5FC034669
:1001A00023604FF0FF3301E04FF00003184607F1E2
:1001B0001C07BD4690BD00BF90B587B000AFF8608A
:1001C000B9607A60FB68002B08DA28F07FFC0346F0
:1001D0004FF009021A604FF0FF3347E0FB68022B33
:1001E00002DC4FF0000341E0FC6840F6DC10C1F295
:1001F000000000F0F9F9034603F102039C4294BFAA
:1002000000230123DBB2002B08D028F05FFC03465B
:100210004FF009021A604FF0FF3327E0FB68A3F1AB
:100220000303FB60FB6840F6DC10C1F200001946D6
:1002300000F09EF9034619687A6807F11003084632
:10024000B968F2F75FFC0346FB75FB7D002B0CD011
:1002500028F03CFC03461C46FB7D184602F044FC9B
:10026000034623604FF0FF3300E03B69184607F177
:100270001C07BD4690BD00BF90B587B000AFF860C9
:10028000B9607A6040F25843C1F200031B68DB6832
:10029000184628F0C1FE03461A46FB689A420ED162
:1002A00040F25843C1F200031B689B68184628F0CF
:1002B000B3FE0346012B02D04FF0010301E04FF0E3
:1002C0000003002B0AD040F25843C1F200031B6820
:1002D0009B68184628F0A0FE0346FB6040F2584396
:1002E000C1F200031B689B68184628F095FE034680
:1002F0001A46FB689A420DD040F25843C1F20003FF
:100300001B68DB68184628F087FE03461A46FB6820
:100310009A4202D14FF0010301E04FF00003002B9D
:1003200011D040F69013C1F200031B68002B0AD0D5
:1003300040F69013C1F200031A687B681046B96852
:100340001A460CF08FF9FB68002B08DA28F0BEFB88
:1003500003464FF009021A604FF0FF3387E0FB6855
:10036000022B01DC7B6882E0FC6840F6DC10C1F205
:10037000000000F039F9034603F102039C4294BFE8
:1003800000230123DBB2002B08D028F09FFB03469B
:100390004FF009021A604FF0FF3368E0FB68A3F1E9
:1003A0000303FB60FB6840F6DC10C1F20000194655
:1003B00000F0DEF8034619687A6807F11003084672
:1003C000B968F2F711FD0346FB75FB7D002B23D0C6
:1003D00028F07CFB03461C46FB7D184602F084FB9C
:1003E0000346236040F25843C1F200031B68DC68F7
:1003F00028F06CFB03461B6818462CF085FF03466B
:100400001A46FB7D204649F6A801C0F2040129F0F6
:10041000F3F84FF0FF332AE0FB6803F10303FB60BE
:1004200040F25843C1F200031B689B68184628F04D
:10043000F3FD03461A46FB689A420DD040F258433A
:10044000C1F200031B68DB68184628F0E5FD03468F
:100450001A46FB689A4202D14FF0010301E04FF0C7
:100460000003002B02D0F868FFF702FD3B69184635
:1004700007F11C07BD4690BD80B582B000AF786023
:100480007B68184600F0D0F87B68184607F108072B
:10049000BD4680BD80B584B000AF78607B6807F151
:1004A0000C021046194600F0F1F8FB68184607F1F7
:1004B0001007BD4680BD00BF80B584B000AF786036
:1004C0007B6803F1040307F10C021046194600F0A3
:1004D000DDF8FB68184607F11007BD4680BD00BF78
:1004E00080B584B000AFF860B9607A6007F10C03A2
:1004F000184600F0DBF8F868B9687A6800F0E0F8B0
:100500000346184607F11007BD4680BD90B583B07D
:1005100000AF78603960786800F0AAF903461C687B
:10052000386800F0A5F903461B689C420CBF002305
:100530000123DBB2184607F10C07BD4690BD00BF92
:1005400090B583B000AF78603960786800F090F9BA
:1005500003461B681C46386800F08AF903461B688E
:10056000E31A4FEAA303184607F10C07BD4690BDF6
:1005700080B582B000AF786039607868396800F083
:1005800083F97868396800F09BF90346184607F14B
:100590000807BD4680BD00BF80B582B000AF78605F
:1005A00039607B685A687B689B689A420FD07B6889
:1005B0001A467B685B68104619463A6800F092F963
:1005C0007B685B6803F104027B685A6008E0786826
:1005D000FFF772FF0346786819463A6800F09AF907
:1005E00007F10807BD4680BD80B483B000AF7860D6
:1005F0007B685B681A467B681B68D31A4FEAA303C3
:10060000184607F10C07BD4680BC704780B582B024
:1006100000AF78607B68184600F08EFA7B68184659
:1006200007F10807BD4680BD80B582B000AF786095
:100630007B68184600F066FA7B68184607F10807E1
:10064000BD4680BD80B582B000AF78607B681A6817
:100650007B689B6819467B681B68CB1A4FEAA3032B
:10066000786811461A4600F075FA7B681846FFF75D
:10067000CDFF7B68184607F10807BD4680BD7B6843
:100680001846FFF7C3FF1FF04DFB00BF80B483B0D7
:1006900000AF786039603B681A687B681A607B68D5
:1006A000184607F10C07BD4680BC704780B483B084
:1006B00000AF7860184607F10C07BD4680BC704754
:1006C00080B586B000AFF860B9607A603B7007F122
:1006D000080207F10C0310461946FFF731FF0346E5
:1006E0004FEAA3037B615FE007F10C03184600F0BB
:1006F00045FA03461A687B681B689A4214BF0023B8
:100700000123DBB2002B01D0FB68ABE007F10C0347
:10071000184600F03FFA07F10C03184600F02EFAD5
:1007200003461A687B681B689A4214BF00230123A2
:10073000DBB2002B01D0FB6894E007F10C031846F4
:1007400000F028FA07F10C03184600F017FA0346E8
:100750001A687B681B689A4214BF00230123DBB22E
:10076000002B01D0FB687DE007F10C03184600F078
:1007700011FA07F10C03184600F000FA03461A6854
:100780007B681B689A4214BF00230123DBB2002B55
:1007900001D0FB6866E007F10C03184600F0FAF997
:1007A0007B6903F1FF337B617B69002BD4BF00239E
:1007B0000123DBB2002B97D107F1080207F10C03EC
:1007C00010461946FFF7BCFE0346022B1BD0032B35
:1007D00002D0012B2ED044E007F10C03184600F0A4
:1007E000CDF903461A687B681B689A4214BF002340
:1007F0000123DBB2002B01D0FB6833E007F10C03CF
:10080000184600F0C7F907F10C03184600F0B6F9D6
:1008100003461A687B681B689A4214BF00230123B1
:10082000DBB2002B01D0FB681CE007F10C0318467B
:1008300000F0B0F907F10C03184600F09FF90346E9
:100840001A687B681B689A4214BF00230123DBB23D
:10085000002B01D0FB6805E007F10C03184600F0FF
:1008600099F9BB68184607F11807BD4680BD00BF5F
:1008700080B483B000AF78607B68184607F10C073E
:10088000BD4680BC704700BF80B582B000AF7860C5
:1008900039607868FFF7A8FE02463B689A428CBF31
:1008A00000230123DBB2002B05D049F6C400C0F2BF
:1008B00004001EF0D5FB07F10807BD4680BD00BF50
:1008C00080B483B000AF786039607B681A683B6899
:1008D0004FEA8303D318184607F10C07BD4680BCC6
:1008E000704700BF80B584B000AFF860B9607A602F
:1008F000BB684FF004001946F3F7BAF903461A46ED
:10090000002A02D07A6812681A6007F11007BD4603
:1009100080BD00BFB0B58AB000AFF860B9607A6042
:10092000FB685A68FB689B689A4232D0FB6819469C
:10093000FB685A68FB685B68A3F10403084611462C
:100940001A46FFF7CFFFFB685B6803F10402FB6800
:100950005A607B681B683B6207F108031846FFF783
:1009600087FF03461968FB685B68A3F10802FB6810
:100970005B68A3F10403084611461A4600F01CF90F
:1009800007F10803184600F0F9F803463A6A1A60BE
:10099000B4E0F8684FF0010149F6DC02C0F204024D
:1009A00000F024F90346FB61F868FFF773FD034686
:1009B0003B6107F1080207F1100310461946FFF7E3
:1009C000BFFD0346BB61FB681846F96900F058F9A2
:1009D00003467B617B697B62FB681A46BB694FEA11
:1009E00083037969CB18104619467A68FFF77AFFB6
:1009F0004FF000037B62FB681D6807F1080318468F
:100A0000FFF736FF03461C68FB68184600F050F9F4
:100A10000346284621467A6900F056F903467B6270
:100A20007B6A03F104037B6207F108031846FFF7B2
:100A30001FFF03461D68FB685C68FB68184600F0F2
:100A400037F90346284621467A6A00F03DF9034605
:100A50007B62FB681D68FB685C68FB68184600F0F9
:100A600027F90346284621461A4600F04BF9F96853
:100A7000FB681A68FB689B681846FB681B68C31A0A
:100A80004FEAA303084611461A4600F063F8FB68D4
:100A90007A691A60FB687A6A5A60FB694FEA8303D5
:100AA0007A69D218FB689A6028E01FF03DFB1FF0BE
:100AB00039F9034618461FF0EDFA7B6A002B0BD17B
:100AC000FB681A46BB694FEA83037969CB18104665
:100AD000194600F00DF909E0FB68184600F0E8F847
:100AE00003467869796A1A4600F00CF9FB681846E3
:100AF0007969FA6900F02EF81FF0FEFE07F1280769
:100B0000BD46B0BD80B582B000AF78607B68184646
:100B100000F006F97B684FF000021A607B684FF026
:100B200000025A607B684FF000029A607B681846AA
:100B300007F10807BD4680BD80B582B000AF786080
:100B40007B68184600F0FAF87B68184607F108073A
:100B5000BD4680BD80B584B000AFF860B9607A60F2
:100B6000BB68002B05D0FB681846B9687A6800F0AE
:100B7000F1F807F11007BD4680BD00BF80B483B017
:100B800000AF78607B681B68184607F10C07BD460C
:100B900080BC704780B483B000AF78607B681B680E
:100BA00003F104027B681A607B68184607F10C07A2
:100BB000BD4680BC704700BF90B585B000AFF860FF
:100BC000B9607A60F86800F0D3F803461C46B8684C
:100BD00000F0CEF80346204619467A6800F0D6F8B1
:100BE0000346184607F11407BD4690BD90B587B07F
:100BF00000AFF860B9607A60F86800F0E5F8034685
:100C00001C46F868FFF7F0FC0346E21ABB689A42FC
:100C10002CBF00230123DBB2002B02D078681EF02A
:100C2000EDF9F868FFF7E0FC0446F868FFF7DCFC34
:100C300003463B6107F1100207F10803104619460D
:100C4000F3F78EFE03461B68E3187B61F868FFF735
:100C5000CBFC02467B699A4207D8F86800F0B4F8EA
:100C600003461A467B699A4204D2F86800F0ACF851
:100C7000034600E07B69184607F11C07BD4690BD9E
:100C800080B582B000AF786039603B68002B08D037
:100C90007B68184639684FF0000200F0A7F8034659
:100CA00001E04FF00003184607F10807BD4680BD7C
:100CB00080B483B000AF78607B68184607F10C07FA
:100CC000BD4680BC704700BF80B584B000AFF860FF
:100CD000B9607A603B60F868B9687A683B6800F090
:100CE000A5F80346184607F11007BD4680BD00BFB2
:100CF00080B483B000AF7860396007F10C07BD465F
:100D000080BC704780B584B000AFF860B9607A608D
:100D1000F868B96800F09CF807F11007BD4680BD7F
:100D200080B582B000AF78607B68184600F09EF80E
:100D30007B68184607F10807BD4680BD80B483B0C4
:100D400000AF78607B68184607F10C07BD4680BC91
:100D5000704700BF80B584B000AFF860B9607A60BA
:100D6000B8681EF083FF07F11007BD4680BD00BFC5
:100D700080B582B000AF7860786800F083F80346F1
:100D8000184607F10807BD4680BD00BFB0B584B066
:100D900000AFF860B9607A60F86800F07FF8054647
:100DA000B86800F07BF80446786800F077F80346EE
:100DB000284621461A4600F07FF80346184607F1F8
:100DC0001007BD46B0BD00BF80B582B000AF7860EF
:100DD0007B68184600F084F80346184600F08CF84B
:100DE0000346184607F10807BD4680BD80B584B0AC
:100DF00000AFF860B9607A60F86800F07DF80246EC
:100E0000BB689A422CBF00230123DBB2002B01D028
:100E10001EF0B0F8BB684FEA830318461FF018FEB7
:100E20000346184607F11007BD4680BD80B584B063
:100E300000AFF860B9607A603B60F868B9687A68BA
:100E400000F066F80346184607F11007BD4680BD5E
:100E500080B582B000AF786039607868396800F09A
:100E600069F807F10807BD4680BD00BF80B483B0B4
:100E700000AF78607B68184607F10C07BD4680BC60
:100E8000704700BF80B483B000AF78607B681846BD
:100E900007F10C07BD4680BC704700BF80B582B02B
:100EA00000AF78607868FFF7EDFF0346184607F15A
:100EB0000807BD4680BD00BF80B586B000AFF860B2
:100EC000B9607A604FF00103FB75F868B9687A6819
:100ED00000F03AF80346184607F11807BD4680BDF2
:100EE00080B483B000AF78607B68184607F10C07C8
:100EF000BD4680BC704700BF80B483B000AF78604F
:100F00006FF04043184607F10C07BD4680BC7047A0
:100F100080B584B000AFF860B9607A60F868B968ED
:100F20007A6800F03BF80346184607F11007BD4603
:100F300080BD00BF80B483B000AF7860396007F136
:100F40000C07BD4680BC704780B586B000AFF86026
:100F5000B9607A60BA68FB68D31A4FEAA3037B6171
:100F60007B69002B0ED07B694FEA8303C3F100033A
:100F70007A68D2187B694FEA83031046F9681A46EB
:100F80002AF038FC7B694FEA8303C3F100037A68D7
:100F9000D318184607F11807BD4680BD80B584B048
:100FA00000AFF860B9607A60F868B9687A6800F0F4
:100FB00007F80346184607F11007BD4680BD00BF7D
:100FC00090B585B000AFF860B9607A60F868FFF757
:100FD000CFFE03461C46B868FFF7CAFE034620460C
:100FE00019467A6800F006F80346184607F1140718
:100FF000BD4690BDB0B584B000AFF860B9607A600E
:10100000F868FFF74BFF0546B868FFF747FF04464F
:101010007868FFF743FF0346284621461A4600F04A
:1010200007F80346184607F11007BD46B0BD00BFDC
:1010300080B586B000AFF860B9607A604FF0010308
:10104000FB75F868B9687A6800F006F80346184638
:1010500007F11807BD4680BD80B586B000AFF860C7
:10106000B9607A60BA68FB68D31A4FEAA3037B6160
:101070007B69002B07D07B694FEA83037868F968A6
:101080001A462AF0B7FB7B694FEA83037A68D318C4
:10109000184607F11807BD4680BD00BF80B582B075
:1010A00000AF786039607B68012B19D13A684FF640
:1010B000FF739A4214D140F6DC10C1F20000FFF732
:1010C000DBF941F2E903C0F2010340F6DC10C1F2A2
:1010D0000000194640F20002C1F200021EF028FD95
:1010E00007F10807BD4680BDB0B582B000AF78609B
:1010F0007B681D687B685C687B681846FFF7D8FDD5
:101100000346284621461A46FFF7FCFD7B68184631
:10111000FFF798FA7B68184607F10807BD46B0BD8F
:101120007B681846FFF78EFA1EF0FCFD80B500AF15
:101130004FF001004FF6FF71FFF7B0FF80BD00BF19
:1011400080B483B000AF78607B68044A1A607B6823
:10115000184607F10C07BD4680BC7047609B040031
:1011600080B584B000AFF860B9607A603B60FB681E
:101170001846FFF7E5FFFB680D4A1A60FB68BA687E
:101180009A60FB687A68DA60FB6803F1100318461E
:101190001EF072F9FB683A68DA61FB684FF00002F2
:1011A0001A76FB68184607F11007BD4680BD00BFE0
:1011B000409B040080B586B002AF786039607B68E0
:1011C0001B7E002B02D04FF0FF3333E07B681846C4
:1011D000396801F0D5F90346FB73FB7B002B1CD06B
:1011E00040F25843C1F200031B68DA68F97B49F604
:1011F000F433C0F2040300930191104649F6F40160
:10120000C0F2040149F61C12C0F204024FF095032B
:1012100028F0F2F96FF001030CE07B684FF0010257
:101220001A767B6803F11003184639681EF0A0FA9D
:101230004FF00003184607F11007BD4680BD00BF00
:1012400080B588B002AF78607B689B68184648F22A
:10125000A061C0F201010CF06FFB7B689B6818462F
:101260004FF001010CF0A4FB7B68DB6818464FF0DF
:1012700001010BF0EFFB4FF000037B610AE07B689C
:101280009B6818464FF0FF010CF0D8FB7B6903F117
:1012900001037B617B690F2BCCBF00230123DBB2F1
:1012A000002BECD14FF002033B6178684FF0000156
:1012B0004FF0000200F052FA0346FB60FB68012B7E
:1012C00008D1786800F00EFC0346BB60BB68012BB8
:1012D00023D027E03B69002B1AD140F25843C1F2DA
:1012E00000031B68DA6849F6E433C0F20403009394
:1012F000104649F65811C0F2040149F61C12C0F21A
:1013000004024FF0D50328F077F94FF000032BE0EB
:101310003B6903F1FF333B61C7E7786800F07CF875
:10132000034621E0BB68052B04D1786800F022F861
:10133000034619E040F25843C1F200031B68DA6823
:1013400049F6E433C0F204030093104649F6A011B5
:10135000C0F2040149F61C12C0F204024FF0E1038E
:1013600028F04AF94FF00003184607F11807BD4668
:1013700080BD00BF80B586B002AF78604FF000033B
:10138000FB6020E078684FF037014FF0000200F07A
:10139000E5F978684FF029014FF0000200F0DEF91E
:1013A0000346002B14BF00230123DBB2002B06D021
:1013B0007B684FF400725A614FF0010327E0FB682D
:1013C00003F10103FB60FA6840F257239A42CCBF55
:1013D00000230123DBB2002BD4D140F25843C1F2E9
:1013E00000031B68DA6849F6D033C0F204030093A7
:1013F000104649F6E811C0F2040149F61C12C0F289
:1014000004024FF0F20328F0F7F84FF000031846FB
:1014100007F11007BD4680BD80B586B002AF786089
:101420004FF00003FB602AE04FF03200FEF70EFAA7
:10143000786800F09DFA78684FF037014FF00002AD
:1014400000F08CF978684FF029014FF0804200F0ED
:1014500085F90346002B14BF00230123DBB2002BC8
:1014600009D0786800F084FA7B684FF001025A6175
:101470004FF0020327E0FB6803F10103FB60FA6809
:1014800040F257239A42CCBF00230123DBB2002B4A
:10149000CAD140F25843C1F200031B68DA6849F62A
:1014A000BC33C0F204030093104649F61821C0F281
:1014B000040149F61C12C0F204024FF4837328F0B1
:1014C0009BF84FF00003184607F11007BD4680BD9A
:1014D00080B586B002AF78607868FFF7B1FE03464A
:1014E000FB60FB68002B02D14FF0030332E0786809
:1014F00000F0F6FC03461A467B685A6078684FF0A5
:1015000010014FF4007200F029F90346002B0CBFC4
:1015100000230123DBB2002B1AD040F25843C1F262
:1015200000031B68DA6849F6AC33C0F20403009389
:10153000104649F64821C0F2040149F61C12C0F2D7
:1015400004024FF48C7328F057F84FF0010301E0C8
:101550004FF00003184607F11007BD4680BD00BFDD
:1015600080B582B000AF78607B689A687B68DB6981
:10157000104619460CF0E0F978684FF010014FF46E
:10158000007200F0EBF80346002B0CBF0023012390
:10159000DBB2002B02D04FF0030301E04FF0000359
:1015A000184607F10807BD4680BD00BF80B586B06C
:1015B00000AFF860B9607A603B60FB689A68FB68CE
:1015C000DB69104619460CF0B7F94FF000037B6158
:1015D0003DE04FF000033B613B69642B01D17B6927
:1015E00042E0FB685B697A6802FB03F3F8684FF03E
:1015F00018011A4600F0B2F80346002B0CBF002376
:101600000123DBB2002B1AD1F868B9684FF40072DD
:1016100000F07AFB0346002B0CBF00230123DBB252
:10162000002B0ED17B6903F101037B617B6803F121
:1016300001037B60BB6803F50073BB6007E000BF7C
:1016400000E000BF3B6903F101033B61C4E73B6875
:10165000002B0CBF00230123DBB23A6802F1FF32FA
:101660003A60002BB5D17B69184607F11807BD46D3
:1016700080BD00BF80B586B000AFF860B9607A6009
:101680003B60FB689A68FB68DB69104619460CF002
:1016900053F94FF000037B613DE04FF000033B61E5
:1016A0003B69642B01D17B6942E0FB685B697A6826
:1016B00002FB03F3F8684FF011011A4600F04EF8F0
:1016C0000346002B0CBF00230123DBB2002B1AD1F1
:1016D000F868B9684FF4007200F09EFA0346002BD8
:1016E0000CBF00230123DBB2002B0ED17B6903F179
:1016F00001037B617B6803F101037B60BB6803F539
:101700000073BB6007E000BF00E000BF3B6903F16E
:1017100001033B61C4E73B68002B0CBF002301239E
:10172000DBB23A6802F1FF323A60002BB5D17B6937
:10173000184607F11807BD4680BD00BF80B485B0CC
:1017400000AFF8600B467A60FB724FF0000318465A
:1017500007F11407BD4680BC704700BF80B586B056
:1017600000AFF860B9607A60FB68DB6818464FF03C
:1017700000010BF06FF9FB689A68BB68DBB243F0BD
:101780004003DBB2DBB2104619460CF057F9FB6898
:101790009A687B684FEA2363DBB2104619460CF067
:1017A0004DF9FB689A687B684FEA2343DBB2104629
:1017B00019460CF043F9FB689A687B684FEA2323CB
:1017C000DBB2104619460CF039F9FB689A687B6861
:1017D000DBB2104619460CF031F9FB689B681846DD
:1017E0004FF095010CF02AF94FF000037B6121E0E6
:1017F000FB689B6818464FF0FF010CF01FF9034689
:101800003B613B6903F08003002B0FD1FB68DB6871
:1018100018464FF001010BF01DF9FB689B68184654
:101820004FF0FF010CF00AF93B691DE07B6903F101
:1018300001037B617A6940F257239A42CCBF0023AF
:101840000123DBB2002BD3D1FB68DB6818464FF0D5
:1018500001010BF0FFF8FB689B6818464FF0FF0191
:101860000CF0ECF84FF0FF33184607F11807BD46AF
:1018700080BD00BF80B586B000AFF860B9607A6007
:10188000FB68DB6818464FF000010BF0E3F8FB68DB
:101890009A68BB68DBB243F04003DBB2DBB21046B0
:1018A00019460CF0CBF8FB689A687B684FEA236313
:1018B000DBB2104619460CF0C1F8FB689A687B68E9
:1018C0004FEA2343DBB2104619460CF0B7F8FB6829
:1018D0009A687B684FEA2323DBB2104619460CF066
:1018E000ADF8FB689A687B68DBB2104619460CF0CD
:1018F000A5F8FB689B6818464FF095010CF09EF820
:101900004FF000037B6113E0FB689B6818464FF0C3
:10191000FF010CF093F803463B613B6903F0800341
:10192000002B01D13B691DE07B6903F101037B6161
:101930007A6940F257239A42CCBF00230123DBB2DD
:10194000002BE1D1FB68DB6818464FF001010BF07A
:1019500081F8FB689B6818464FF0FF010CF06EF8A9
:101960004FF0FF33184607F11807BD4680BD00BF92
:1019700080B586B000AF78607B68DB6818464FF0B2
:1019800000010BF067F84FF000033B617B689B6838
:1019900018464FF07A010CF051F87B689A683B6961
:1019A0004FEA2363DBB2104619460CF047F87B6818
:1019B0009A683B694FEA2343DBB2104619460CF0A4
:1019C0003DF87B689A683B694FEA2323DBB21046F7
:1019D00019460CF033F87B689A683B69DBB2104615
:1019E00019460CF02BF87B689B6818464FF0950160
:1019F0000CF024F84FF000037B6154E07B689B6897
:101A000018464FF0FF010CF019F80346FB60FB6825
:101A100003F08003002B42D17B689B6818464FF08F
:101A2000FF010CF00BF803464FEA0363BB607B68D1
:101A30009B6818464FF0FF010CF000F803464FEA90
:101A40000343BA6842EA0303BB607B689B6818469D
:101A50004FF0FF010BF0F2FF03464FEA0323BA6891
:101A600042EA0303BB607B689B6818464FF0FF01A6
:101A70000BF0E4FF0346BA6842EA0303BB607B68ED
:101A8000DB6818464FF001010AF0E4FF7B689B68B1
:101A900018464FF0FF010BF0D1FFFB681DE07B699A
:101AA00003F101037B617A6940F257239A42CCBF6C
:101AB00000230123DBB2002BA0D17B68DB68184632
:101AC0004FF001010AF0C6FF7B689B6818464FF093
:101AD000FF010BF0B3FF4FF0FF33184607F1180773
:101AE000BD4680BD80B586B000AF78607B68DB689E
:101AF00018464FF000010AF0ADFF7B689B6818465E
:101B00004FF048010BF09AFF7B689B6818464FF036
:101B100000010BF093FF7B689B6818464FF00001B3
:101B20000BF08CFF7B689B6818464FF001010BF0AF
:101B300085FF7B689B6818464FF0AA010BF07EFF7B
:101B40007B689B6818464FF087010BF077FF4FF0DA
:101B500000037B613FE07B689B6818464FF0FF0104
:101B60000BF06CFF03463B723B7ADBB25BB2002B9F
:101B70002DDB4FF001033B6111E07B689B68184649
:101B80004FF0FF010BF05AFF03461A4607F1080118
:101B90007B69CB181A703B6903F101033B613B6918
:101BA000042BCCBF00230123DBB2002BE5D17B68E3
:101BB000DB6818464FF001010AF04CFF7B689B6818
:101BC00018464FF0FF010BF039FF3B7A1FE07B69AD
:101BD00003F101037B617A6942F2BF73C0F209032A
:101BE0009A42CCBF00230123DBB2002BB3D17B6828
:101BF000DB6818464FF001010AF02CFF7B689B68F8
:101C000018464FF0FF010BF019FF4FF0FF33184655
